:020000040800F2
:10000000005000203DA9000883A9000885A9000828
:1000100087A9000889A900088BA900080000000032
:100020000000000000000000000000008DA9000892
:100030008FA900080000000091A90008050A000827
:1000400097A9000899A900089BA900089DA9000884
:100050009FA90008A1A90008A3A90008A5A9000854
:10006000A7A90008A9A90008ABA90008ADA9000824
:10007000A5990008B1A90008B3A90008B5A900080E
:10008000B7A90008B9A90008BBA90008BDA90008C4
:10009000BFA90008C1A90008C3A90008C5A9000894
:1000A000C7A90008C9A90008CBA90008CDA9000864
:1000B00071760008D1A90008D3A90008D5A90008C5
:1000C000D7A90008D9A90008DBA90008DDA9000804
:1000D000DFA90008DD7400081D390008E5A9000843
:1000E000E7A90008E9A90008EBA9000810B5054C2C
:1000F000237833B9044B13B10448AFF300800123D4
:10010000237010BDB8020020000000006CE200085F
:1001100008B5064B1BB106480649AFF300800648F8
:10012000036813B1054B03B1984708BD00000000F8
:100130006CE20008BC020020B802002000000000B1
:10014000154B002B08BF134B9D46A3F5803A0021A9
:100150008B460F461348144A121A0AF076FD0F4BCD
:10016000002B00D098470E4B002B00D09847002062
:10017000002104000D000D48002802D00C48AFF308
:1001800000800AF015FD2000290007F0A1FB0AF00D
:10019000FBFC00BF00000800005000200000000031
:1001A00000000000B80200207826002000000000B7
:1001B0000000000070B5354D86B02C681CB10123DD
:1001C0002B6006B070BD684609F0C6FF01A809F0B3
:1001D000CDFD4FF400400AF01FF9112001210AF073
:1001E00087F94FF400602023C4F201006946ADF89E
:1001F00000308DF8034009F04BFF4FF400700121EF
:100200000AF076F94FF4105001264FF46023C4F23F
:10021000010001A9039301948DF808408DF809406D
:1002200004948DF8146009F07BFD4FF41050C4F273
:10023000010005213246234609F0CAFD4FF4105053
:10024000C4F20100314609F09BFD4FF41050C4F296
:10025000010009F09FFD4FF41050C4F2010009F0B5
:100260009FFD0028F7D14FF41050C4F2010009F0AF
:100270009BFD4FF41050C4F2010009F09BFD0028D3
:10028000F7D1034B01221A6099E700BFD802002082
:100290008C2500204FF4105008B5C4F20100012154
:1002A00009F08CFD40F2D423C2F2000301221A604F
:1002B00008BD00BF38B50D4C054623680BB90020BA
:1002C00038BD4FF41050C4F20100022109F0D0FDF6
:1002D0000028F4D04FF41050C4F2010009F0C4FD1E
:1002E000002328802360012038BD00BFD4020020F5
:1002F00070B448F6396301EB4104951EC3F6E3037D
:100300000229C1EBC40183FB014348F21F54D8BF4B
:100310001546C5F2EB14D8BF013A84FB0264C91735
:10032000C1EB630128180818D51CD317043032EA32
:10033000220228BF2A46A3EB641100EBA202C3EB02
:10034000E413521842F29340D218C9F2492080FBBC
:100350000230D3178018C3EBA000C0EBC000101A06
:1003600070BC704770B40646002922D00078F0B106
:1003700000231846F25CA2F13004E4B2092CA2F189
:1003800041050DD9052DA2F161049CBFA2F13704EE
:10039000E4B205D9052C9ABFA2F15704E4B20024B7
:1003A0000133DDB204EB0010A94280B2E2D870BC88
:1003B00070470846FBE700BF4FF48050C4F20100CD
:1003C0004FF40051002209F0D5BE00BF4FF4805019
:1003D000C4F201004FF40051012209F0CBBE00BF6E
:1003E00000B583B001A809F0B7FE102001210AF082
:1003F0007FF84FF40053ADF804304FF480500223DF
:10040000C4F2010001A98DF8063010238DF80730E1
:1004100009F03EFEFFF7DAFF03B000BD00B583B080
:1004200001A809F099FE042001210AF061F8402397
:100430004FF40060ADF80430C4F20100482301A974
:100440008DF8073009F024FE03B000BD4FF40060C2
:10045000402108B5C4F2010009F086FED0F1010088
:1004600038BF002008BD00BFF0B4114A0346106831
:10047000D8B110490E68104964360D680F49013D26
:100480000C680F495E610F680E491D610968DF60E5
:1004900099600D49096859600021072C08BF0C4676
:1004A0009C610F2419621C601160F0BC704700BF92
:1004B00004030020DC02002018030020F0020020CA
:1004C000E002002014030020EC02002070B582B08E
:1004D00001A809F041FE4FF44064082001210AF010
:1004E00007F8C4F201044FF4807301A902262046E4
:1004F000ADF8043004238DF807308DF8066009F05C
:10050000C7FD01A809F028FE0820012109F0F0FF2D
:100510004FF40075204601A91023ADF804508DF862
:1005200006608DF8073009F0B3FD20462946012208
:1005300009F020FE02B070BDF8B5A44C2368FF2B73
:1005400056D04FF44060C4F201004FF4807109F0BE
:100550000BFE0546002833D0FFF72EFF236801204D
:10056000012B9A4D33D04AD3022B4DD0984B1A68A9
:10057000904200F08680974E022132682960911FD8
:100580001229186063D9052A94BF9348934806F04E
:100590006FFF934F934806F06BFF002323603B6887
:1005A0000F2B00F0CC81102B6ED0FF2B3AD00133F3
:1005B0003B2B3B6000F0CE8134D90023236031E037
:1005C000FFF704FF23682846012B804DCBD1804BD9
:1005D0001A68824229D01860002814BF0322022220
:1005E0007F4B2260FF221A607A4B00221A60F8BD0E
:1005F0007D4B1A68642A19D001321A60F8BD0123B4
:100600002B60734B1860F8BD714B1A68904238D05C
:10061000704E032132682960782A186012D9704B15
:1006200000221A6000233360F8BDF8BD4FF440602B
:10063000C4F201004FF40071002209F09BFD002379
:100640002360F8BD4A2AEDD800232B60EAE7644F07
:100650000F2A3B6834D8232B00F097813A2B00F007
:1006600085811C2B9CD1614A1268D0079FD56048B8
:1006700006F0FEFE5B4806F0FBFE002323603B68AD
:100680008EE7544B1A68B7E75A4A002313605A4A58
:100690001360564A1360594A1360594A1360594A05
:1006A0001360594A1360594A1360594A1360594AF2
:1006B0001360594A1360594A136011233B60B1E734
:1006C000A3F11102292A3FF66BAF01A151F822F0E4
:1006D00037090008A1050008A1050008A1050008C8
:1006E000310900082B090008250900081F09000826
:1006F00019090008130900080D090008FD08000881
:10070000F7080008F1080008EB080008E5080008F1
:10071000DF080008D9080008C9080008C308000855
:10072000BD080008B7080008B3080008AF080008B3
:10073000AB080008A50800089F08000899080008F1
:10074000930800088D08000887080008830800083F
:100750007F0800086D0800085B08000849080008C9
:100760003708000825080008BB070008A90700088B
:100770009707000879070008214A126812F001055E
:100780007FF415AF264806F073FE164806F070FE9B
:1007900025603B6804E72149194A0D681068503507
:1007A00001300D601060FEE61C49154A0D681068A6
:1007B000283501300D601060F5E61849104A0D68C3
:1007C0001068143501300D601060ECE62000002048
:1007D00000030020E8020020F0BC000810BD000863
:1007E0001C00002028C70008E40200201C03002091
:1007F00030BD000804030020F4020020FC020020A9
:100800001003002008030020EC0200201403002045
:10081000F0020020E002002018030020DC0200208B
:1008200078BD00086549664A0D6810680A350130D0
:100830000D601060B7E66149614A0D6810680835BF
:1008400001300D601060AEE65C495D4A0D681068CD
:10085000043501300D601060A5E65849584A0D680E
:100860001068023501300D6010609CE65349544A0F
:100870000D681068013501300D60106093E6514934
:10088000D1E75049D8E74F494D4ADFE74D494C4A37
:10089000E5E74C494A4AEBE74B49494AD6E74A491A
:1008A000474ADCE74849464AE2E7484986E747497C
:1008B000B9E74649C0E74549414AC7E74349404A85
:1008C000CDE742493E4AD3E7414A126812F001059A
:1008D0007FF46DAE3F4856E73F493D4A6FE73E49DA
:1008E0003B4AA1E73C493A4AA7E73B49384AADE7CA
:1008F0003949374AB3E73849354AB9E7374A1268C0
:1009000012F001057FF453AE35483CE73549334AD0
:100910004CE73449314A52E73249304A84E7314999
:100920002E4A8AE72F492D4A90E72E492B4A96E70F
:100930002C492A4A9CE72C4A0121116033E62B4BB3
:100940001A6822B12A4A0121116000221A6010237C
:100950003B6067E6274B204A196812689142264996
:1009600022D0204800681A6008605BE6144A1268CA
:10097000D2077FF51CAE214806F07AFD204806F02C
:1009800077FD00223B682A600AE6114A1268D10707
:100990007FF50DAE0F4806F06BFD194806F068FDB7
:1009A00000232B603B68FBE50E480C6800680134AF
:1009B0008442D8D10D4C01252560D4E7DC0200200B
:1009C0001003002018030020F0020020E0020020A5
:1009D000FC02002054BD0008140300201C0300206A
:1009E00030BD0008EC02002008030020F4020020C3
:1009F00004030020F80200200C03002078BD00084A
:100A000028C70008034B1A6812B11A68013A1A6025
:100A1000704700BF90250020064B074A1B68012B3A
:100A20001EBF064B1B68B0FBF3F010601368002B71
:100A3000FCD17047200300209025002028000020D2
:100A4000044B054A1B6803FB00F010601368002B81
:100A5000FCD170472400002090250020084B4FF463
:100A60007A711B6810F1FF3001FB03F1054A06D3D0
:100A700011601368002BFCD110F1FF30F8D27047E1
:100A80002400002090250020012810B423D0022843
:100A90002CD01C4B64221A601B4B0A221A6042F2B3
:100AA00010710320194A4EF210031468CEF20003AD
:100AB000B4FBF1F101394FF46D425960CEF20002FE
:100AC000F02182F8231000229A6007221A60104B4E
:100AD000186010BC70470B4B44F2402118600A4B61
:100AE0004FF47A721A60C0F20F01DBE7054B0A225D
:100AF0001A60054B48F2A06164221A60C0F201013D
:100B0000D0E700BF280000202400002004020020BD
:100B1000200300202DE9F00140F2901240F25C1316
:100B200040F26411C2F20003C2F20001C2F20002FC
:100B3000D2F8008093F800C05F789E780D784C78EA
:100B400040F2581040F2700240F274038978C2F209
:100B50000002C2F20003C2F20000C0F8008082F876
:100B600000C0577096701D705C709970BDE8F00100
:100B7000704700BF722008F023BF00BFF0B5214AC4
:100B800083B01160204A002310608DF804308DF886
:100B900005308DF8063000282AD04CF6CD45CCF62D
:100BA000CC451A48A5FB01250478194A8678477870
:100BB00032F8144032F81700AD0832F8162005EB71
:100BC00085058DF800408DF801008DF802204D1B41
:100BD0001C46A542204601A988BF6946013408F099
:100BE00075FF042CF5D1042008F0EAFE03B0F0BD37
:100BF0000446204601A9013408F068FF042CF8D10E
:100C0000F1E700BF9C0300203003002064010020B6
:100C10009CC10008AE2008F0D3BE00BF70B50546E9
:100C20000E46722420462946013408F04FFFAE2CB0
:100C3000F8D106B970BDBDE87040FFF7EBBF00BF4B
:100C400070B540F27402C2F20002957814785678BA
:100C50004CF29C13C0F6000382B033F8144033F812
:100C6000162033F81530014601A88DF804408DF8A0
:100C700005208DF80630FFF7D1FF02B070BD00BF30
:100C800000B583B00023014601A88DF804308DF82B
:100C900005308DF80630FFF7C1FF03B000BD00BF7F
:100CA0000E2A30B436D81F4B0C789B5C48F689026C
:100CB00004FB03F4C8F68802A2FB0452C2F3C70285
:100CC00002700C7814B10AB9012202704C7848F60F
:100CD000890204FB03F4C8F68802A2FB0452C2F3A3
:100CE000C70242704C7814B10AB9012242708C7864
:100CF00048F6890204FB03F3C8F68802A2FB03420C
:100D0000C2F3C70282708B7813B10AB901238370D2
:100D100030BC70470B7803704B7843708B788370CE
:100D2000F6E700BF94C2000810B5104B104C1A68CB
:100D300082B020460F49FFF7B3FF0F4B1B689BB1F2
:100D40000E4BA1782078627833F8104033F81220E7
:100D500033F8113001A801218DF804408DF80520E9
:100D60008DF80630FFF75AFF02B010BD5801002081
:100D70007400002070000020600100209CC1000869
:100D80000E4B1B68032B18D8DFE803F013100A0280
:100D90000B4B00223F2119705A709A70FFF7C4BFA5
:100DA000084B012200201A60FFF76ABF0020FFF7FE
:100DB00067BF054B1868FFF743BF7047A8030020C3
:100DC00070000020000400206001002030B5234B9B
:100DD0008DB01B68002B20D0214D00242A462346CD
:100DE00011691432890741BF0CA800EB840141F856
:100DF0002C3C013401330B2BF2D1002C1FD1194AAA
:100E00002346146003EB830305EB83056B68984767
:100E1000154B00221A600DB030BD1249124A096804
:100E20000F4801EB8101156800EB81008468691CA3
:100E3000A1421160EFD3416813608847EBE70AF0E5
:100E400099F9B0FBF4F303FB14000CAA02EB800346
:100E500053F82C3C034A1360D4E700BFFC03002086
:100E60007C000020E8030020B40300202DE9F00FEF
:100E70000C0682B04DD4DFF810C1424C01276FEA56
:100E8000020904EBC10BC2F1040A3D46CDF80490FF
:100E9000ACF10B060021042A1AD854460BEB0708C4
:100EA00001460A290DD818F8019C49FA04F933B310
:100EB00019F0010F05D01CF8019049F002090CF857
:100EC0000190013C0131B4F1FF3FEAD101990631B3
:100ED00063B909180A2909D807EB870807EB4808FE
:100EE00008EB010401310A293555F9D90137092FD9
:100EF0000CF10B0CCED102B0BDE8F00F704719F029
:100F0000010F1ABF4FF004090CF801900CF80150C2
:100F1000D7E7B0394C292AD8DFE801F02B29292955
:100F20002929292929292929292929292929292931
:100F30002D2929292929292929292929292929291D
:100F400029292F2929292929312929272929292905
:100F50002D292929292929292929292929292929FD
:100F600029292F29292929293100052183E7202131
:100F700081E701217FE702217DE703217BE704214F
:100F800079E700BF9CBD0008A32500206D2812D87A
:100F900048F6A333CBF62E23A3FB0023DB08DA07A6
:100FA00041BF03EB830203EB4203C0EB43000A3073
:100FB000043008F08BBD704770B52B4B82B01A68B7
:100FC00006460AB901261E60284A294B1178547832
:100FD000907833F8111033F8142033F810300024CF
:100FE000244D8DF800108DF801208DF802308DF819
:100FF00004408DF805408DF806400AE0FFF7C6FF73
:1010000015F8013C013443F001036E2C05F8013C56
:1010100015D015F8013B204603F00203DBB2694608
:10102000002BEBD1204601A9FFF7B0FF15F8013CDA
:10103000013423F001036E2C05F8013CE9D10E4B7D
:1010400018680E4B1968FFF799FD16B10C4B1B6819
:1010500033B1FFF78FFD0B4B01221A6002B070BD58
:101060000120FFF7EDFDF6E7DC030020640100201E
:101070009CC1000898250020300300209C0300201C
:10108000A80300209425002008B5064B1A6822B159
:10109000002210461A60FFF78FFF034B01221A60EF
:1010A00008BD00BFFC0300209425002008B50D4BAF
:1010B0000D481A680D49FFF7F3FD0D4B1B68032B14
:1010C00003D00C4B1B68990708D40B4B1B6803B962
:1010D00008BD0120BDE80840FFF76EBFFFF71AFD0D
:1010E000F3E700BF90010020640100205C010020B4
:1010F000A803002078000020600100202DE9F041C5
:10110000854B84B01A683AB984490B68002B00F00B
:10111000E28004B0BDE8F081814A4CF6CD401678FB
:10112000CCF6CC40A0FB06107C49002400091C60D2
:101130000C60DFF8048200F0B380C8F80000557836
:101140004CF6CD43CCF6CC43A3FB05031B09DFF8DB
:10115000ECC102D1002D40F0BC80CCF80030947876
:101160004CF6CD43CCF6CC43A3FB04231B096D4FB7
:1011700002D1002C40F0AB806B4A3B606B4B0020EF
:101180001070507090701E705D709C70D8F80030B8
:101190001C4693B1654A1478A34240F2948014B17E
:1011A000002010700124604A5D4815780078EB1823
:1011B000834200F2A08013700124DCF800308BB170
:1011C0005A48427893427AD912B1002242700124DF
:1011D000554A534855784078EB18834200F2908086
:1011E000537001243868002861D0504B9A7890429F
:1011F00061D912B100229A7001244B4D484AAF7850
:1012000096783818B0429CBFC0B2A87003D9B742D4
:101210004DD0AE703046464992F800C092F801E0D9
:101220006C782F785A781D789B7831F81C8031F8CB
:10123000177031F81EC031F8122031F816E031F87D
:10124000133031F8146031F8104031F815008DF882
:101250000A40384D8DF804808DF805C08DF806E001
:101260008DF808708DF809608DF80C008DF80D2050
:101270008DF80E30002406E0012B32D0032B35D040
:1012800001346E2C09D0635D022BF5D1204602A9F2
:101290000134FFF77BFE6E2CF5D1FFF76BFC38E7CE
:1012A000002E3FF44AAF0123C8F8003047E764BB83
:1012B00001230B602DE7121A9A7001249DE7D21AC0
:1012C0004270012484E7E41A147001246BE70123BF
:1012D00052E7012341E7DFF86080DFF860C0114F7B
:1012E00054E7204603A9FFF751FEC9E7204601A9AC
:1012F000FFF74CFEC4E785421CBF107001245CE779
:1013000085421CBF507001246CE7054A064D967853
:10131000A878064B7FE700BFFC030020942500203F
:1013200064010020380400204C03002050030020FA
:101330009CC100089825002088030020700300202D
:1013400070B5154A154B94781178557833F811100B
:1013500033F8152033F8143082B00024104E0546BF
:101360008DF800108DF801208DF802308DF80440C2
:101370008DF805408DF80640A35D20462B4201A95B
:1013800018BF69460134FFF701FE6E2CF4D1FFF758
:10139000F1FB02B070BD00BF640100209CC10008D9
:1013A000982500202DE9F843584B594E1A682AB960
:1013B0003768002F00F09B80BDE8F883DFF8588184
:1013C00000221A603260C8F80020524C4FF0000E24
:1013D0007746A4460EEB8E050EEB45050B230CEB72
:1013E00005095A1EA918605C611810F0010F47D05A
:1013F0000A2A05EB03074CD01CF8077020F0010007
:10140000FF0741D40870002A48D0023B0127002B77
:10141000E7D10EF1010EBEF10A0FDBD10120FFF77B
:101420008FFF002F5FD0D8F800300127012B08BFB5
:10143000384CC1D1DFF8DCE04FF0000CF1460CEB8A
:101440008C050CEB4505002309EB0508EA18A15CA7
:10145000A21801F00600022827D001330A2BF5D983
:101460000CF1010CBCF10A0F0EF10B0EE7D10420B8
:10147000FFF766FF002F9FD101233360BDE8F8839B
:101480001346002BADD1C4E713460127002BA8D18A
:10149000BFE720F0010089F80A00B6E70EF1010E5F
:1014A0000127BEF10A0F95D1B8E73BB301F0040064
:1014B000C0B20028D1D141F004010A2B117022D012
:1014C0000133EA18A25C02F00202D2B24AB10A2B3E
:1014D00019D001331EF8032002F00202D2B2002A12
:1014E000F5D10127BAE70123C8F80030A2E7DFF8F9
:1014F0002880D8F80030002B98D166E741F004012D
:1015000088F80010DCE70127AAE700BFFC030020F1
:1015100094250020982500205C0300202DE9F00F81
:101520006C4B1A6832B96C4A1368002B6BD0BDE85B
:10153000F00F704700201860674A684E684B012121
:1015400010603160196033688BB166480A256C1EE3
:101550000023C25C02F00301012938D001330B2BB8
:10156000F7D10B382546002CF1D1346043E0DFF889
:1015700070A1DAF80010002942D0DFF87CB1DBF866
:101580000020002A41D0584C58492268086802EBD4
:101590008205574902EB450501322D1802EB820600
:1015A0004F5D02EB46063018524E27F004074F55A8
:1015B00036680D5CB24245F0040708BF45F00505EA
:1015C0000F54226004BF0D54CBF8003013E004EB3D
:1015D0008400474904EB4000C01822F00102092CA6
:1015E0000A5408D005EB850205EB4205EB18CA5CEE
:1015F00042F00102CA540520BDE8F00FFFF7A0BE7B
:101600000123136093E7354E9DE740F28431C2F227
:1016100000010F6840F2F43340F298313148C2F2D1
:101620000003C2F20001D3F80090D1F80080944684
:101630000A25A0F163066C1ED30749D40023C25CBF
:1016400002F00301022905D001330B2BF7D14B46E1
:10165000002211E0ACB112F0010217D005EB8502B7
:1016600005EB4202D218B15CA84641F00401B15426
:101670004FF0010C2746012225460B388CB19946C4
:10168000D9E7F25C42F00502F254F3E7BCF1000F37
:10169000F0D1F15C4FF0010C41F00401F15490469F
:1016A000E8E740F28431C2F200010F6040F2F43109
:1016B000C2F200010B6040F29833C2F20003C3F89B
:1016C0000080CBF800C0002A95D1CAF8002092E72C
:1016D0004B46D1E7FC03002094250020A003002006
:1016E00094030020FB25002098030020F403002031
:1016F00098250020840300206C0300202DE9F84386
:101700006B4B1A6832B96B4D2B68002B00F0A6802A
:10171000BDE8F88300201860674C664B20601860B5
:101720004FEA8008654B08EB0007C0F10B0600EBA1
:10173000400200EB470703EB8202F7191D4699466A
:10174000DF191346197841F0040103F8011BBB426D
:10175000F8D1C0F1090E431C73454FEA8E0C18D224
:1017600008EB000300EB09070CEB0E0105EB43034C
:101770000B3F0EEB41010A337F18D17A41F004018F
:1017800002F80B1FD97ABA4241F0040103F80B1F8B
:10179000F3D10CEB0E020EEB420252190346D15C60
:1017A00041F00401D1540133B342F8D300284DD0A5
:1017B000421EC0F10C07BA4210D202EB820102EBCA
:1017C00041010B185B197E19013B761813F8011BB8
:1017D00021F00401B34203F8011CF7D1C0F10A085B
:1017E000404528BF4FEA880920D200EB80034FEA2A
:1017F000880900EB430309EB08019B1802EB050C79
:1018000008EB4101C0F10B065B198C4493F800E032
:10181000991A2EF0040E83F800E011F806E00B335D
:101820002EF0040E634501F806E0EFD109EB080342
:1018300008EB43031B185B19013B13F8011B013232
:1018400021F00401BA4203F8011CF6D30420FFF78B
:1018500077FD236801332360BDE8F883164C2068C8
:1018600004287FF65DAF05281CBF144B03F16E04FE
:1018700004D119E0A34203F8010C0ED013F8012B98
:1018800002F00201C9B242F0040022F00402002971
:10189000F0D1A34203F8012CF0D10420FFF750FD52
:1018A00001232B60BDE8F88304220727034D84E75A
:1018B000FC0300209425002024030020982500200C
:1018C00070B5254A254813681BB90368002B39D029
:1018D00070BD00231360224D224A03602B60136009
:1018E0002E6886B9204B03F16E011A7822F00402AB
:1018F00003F8012B8B42F8D10420FFF721FD2B6860
:1019000001332B6070BD174A136801331360DA0787
:10191000DED5741EA4B26D2C0FD813490B5D03F0F5
:101920000202D2B22AB10FE00B5D03F00202D2B282
:1019300052B90134A4B26E2CF6D1012303600136F2
:101940002E6070BD064DCBE743F0040304200B5519
:10195000661CFFF7F5FCF2E7FC030020942500204D
:101960002C03002034030020982500202DE9F00FDF
:101970008F4B86B01A6842B98E4B1A68002A00F065
:101980000D8106B0BDE8F00F704700221A608A4C46
:10199000884B22601A600292DFF820C2002000EB20
:1019A000800200EB4202624400231178013321F0EF
:1019B00004010B2B02F8011BF7D101300A28EED1EC
:1019C000029A029B0132C3F1040305922260009344
:1019D000002000EB0C0200231178013321F00801F4
:1019E0000B2B02F8011BF7D10B306E28F1D1009FB1
:1019F000724C7F42DDF800B00197BA460027BAF179
:101A0000050F2CBFD1464FF005099DE806000023C5
:101A1000BBF1040F34BFD8464FF004081AE0042984
:101A200034BF0D460425042B404603D9052A2CBF9C
:101A30001546052500EB800600EB460040191CF812
:101A4000005045F008050CF8005001330131013217
:101A50000B2B15D0E05C00F00200C0B20028F4D0DF
:101A6000042FDCD9042B05D8042934BF0D460425E6
:101A70004846DFE7042A8CBF154605254846D9E7C6
:101A800001370B340A2F0AF1010A0BF1010BB6D111
:101A9000029A6FF015036FF0090909FB02F9DDF8EE
:101AA00008A003FB02F2DDF814B053460020DB432C
:101AB0000190049280460393CDF800B0039F0298F2
:101AC00007EB080303EB83050AEB8A020AEB4202E9
:101AD00003EB4505019B16182D18D21903EB0C01D9
:101AE0006644624465445C4600231EE0042B30D803
:101AF000C34509D89B4507D8049FD01910F80B7C23
:101B000047F0040700F80B7C11F8010B00F0080700
:101B1000FFB21FB140F0040001F8010C013301369F
:101B20000132013501340B2B25D002EB090040783E
:101B3000C007E9D5B8F1040FD8D9042B009811D803
:101B40000928E1D89B45DFD8D07A40F00400D07254
:101B5000DAE7C345D8D80A2CD6D8687840F0040014
:101B60006870D1E70928CFD80A2C9EBF307B40F09F
:101B700004003073C8E7019A009B08F101080B329A
:101B80000133B8F10A0F01920AF1010A009395D1CD
:101B9000042006B0BDE8F00FFFF7D2BB064C20686A
:101BA000042802907FF6F8AE01221A60E9E600BF31
:101BB000FC03002094250020F0030020982500203D
:101BC000F8B59F4C2368002B40F0A2809D4B1B680A
:101BD000032B11D8DFE803F0724211022368002BB7
:101BE00040F0C280984A136833B998490B686D2B4E
:101BF00040F2C18001231360F8BD2368002B00F080
:101C00009D808F4900220A60914B8F491A600A60BB
:101C1000904802F10B0500F10B071D600021BF1A6F
:101C20008B1A1B187C180DE013F80B6C16F0010FC3
:101C30009E5C00F0E28046F004069E5401339C4214
:101C400000F0E2808D42EFD993F8636006F002065F
:101C5000F6B2002E00F0D0809E5CECE72368002BEB
:101C600076D0774900230B607B4A774913600B607D
:101C70005F1C78481E46176003F16E0C594203F151
:101C80000C0433183A460DE05D7815F0010F5D5CE9
:101C900000F0C48045F0040501325D540133A242D6
:101CA00000F0C4800A2AEFD913F80A5C05F0020597
:101CB000EDB2002D00F0B1805D5CEBE72368002BF6
:101CC00031D05F4A00211160644B5F4A1960116096
:101CD0004C1C60481C604E42C1F16E073318002254
:101CE0000CE013F8015C15F0010F5D5C78D045F055
:101CF000040501325D5401330B2A78D09442F0D9A7
:101D00009D7A05F00205EDB2002D68D05D5CEEE72E
:101D100009F030FAC217920F831803F003039B1ADD
:101D2000484A136054E7484A1368002B7FF464AFB5
:101D30004A4B19680A293FF65DAFC9E742490B686B
:101D4000002B7FF459AF424B1A686D2A09D85FE720
:101D50003D490B68002B7FF44FAF3F4A13680A2BB5
:101D600086D901230B60F8BD354A0023136037493B
:101D7000354A0B601360374803F10B021B180A60E9
:101D800003F1160C002113180CEB010410E01E786F
:101D90009D1AF60755BFC2EB03056E5C6E5C46F0FC
:101DA000040658BF26F004066E5401339C4211D03D
:101DB0006D2AECD913F86E7C9E1A07F00207FFB269
:101DC0003546002F37D0755C013345F004059C4241
:101DD0007554EDD10B310B326E29D4D118E05D5C16
:101DE00025F0040501325D5401330B2A86D10B36F0
:101DF000BE427FF473AF0BE09E5C26F004069E5457
:101E000001339C427FF41EAF0B316E297FF408AF83
:101E10000420BDE8F840FFF793BA5D5C25F00405A7
:101E200001325D540133A2427FF43CAF0B3666456C
:101E30007FF427AFECE7765C26F004066E54B4E737
:101E4000FC0300205403002094250020AC03002054
:101E50003C03002098250020900300204003002030
:101E60002DE9F04FB54A85B01368B54E33B93368E4
:101E7000002B00F0978005B0BDE8F08F00231360C1
:101E8000B04AB14C1360B14AB14D1360B14A3360EE
:101E900023602B6013602368002B44D1AE4A117875
:101EA0001F2960D951781F2900F2C8803F228DF880
:101EB00008308DF809208DF80A30A84B03A802A934
:101EC0001A68FEF7EDFE9F4F2968A54E9DF80C801D
:101ED0009DF80DC09DF80EE0A24B386801EB81091A
:101EE000A14A36F8188036F81CC036F81EE001EB1F
:101EF000490100260818194683F8008083F801C0BC
:101F000083F802E0167056709670FFF73FF823686A
:101F10002D6896493868CD5495495A1CC85422609A
:101F2000FEF728FEA7E72A680F2A24D9914B03F170
:101F30006E0403E0A34203F8010C0ED013F8012B4A
:101F400002F00201C9B242F0040022F004020029AA
:101F5000F0D1A34203F8012CF0D10420FFF7F0F9EF
:101F60000123336087E73F228DF808208DF8093080
:101F70008DF80A30A1E7DFF8D4C1724FDCF80030E9
:101F8000D7F800809A4279D0724B1B6802F00109A1
:101F9000B9F1000F4BD143452ED908F101033B6045
:101FA0002A6830E0684C6A4D75E7BBF10A0F1AD811
:101FB0005B460EEB8E000EEB400042F29858C018C4
:101FC000C2F2000818F8008018F0010FDDF8008058
:101FD00004D0E5E0C85CC00700F1E28001330B2BC0
:101FE000F8D1CDF800800EF1010E0B31BEF10A0FD1
:101FF00067D11023CCF80030DCF800309A4228D3A7
:1020000001232A683360092A2ED92368DFF85C810E
:10201000062B7BD0564E29683A68052B08F803102A
:10202000F25401D801332360FEF7A4FD23E74345B2
:10203000E2D208F1FF333B602A68E4E792781F2A76
:102040000AD88DF808308DF809303F238DF80A3012
:1020500033E701322A60D6E73F228DF808308DF849
:1020600009208DF80A2028E702EB8201386802EB8C
:10207000410210183B49FEF789FFC6E740F2803065
:10208000C2F200000368984580D112F0010900F007
:102090008F8008F1FF3B9246B8F1000F02D102F1A8
:1020A000010AC346BAF1090FA3D80AEB8A0142F22A
:1020B00098530AEB4101C2F200035918D646CDF8F5
:1020C0000080D64562D01EF001033FF472AF0A23B0
:1020D0000EEB8E000EEB400042F29858C2F2000860
:1020E000C01818F80000DDF80080C00706D4002BE7
:1020F0003FF477AF013BC85CC007F8D540F28030B1
:10210000C2F20000CCF800E0036041E798F800302C
:10211000174E092B30D90023013318F803E0F15C86
:1021200008EB0300F218052B00F801EC02F8011C83
:10213000F2D12368013B23606DE700BFFC03002060
:10214000942500205803002028030020EC030020E1
:10215000B8030020800300205C01002090010020D3
:102160009CC10008F803002038030020640300200D
:10217000300400209825002003EB8301307803EB26
:10218000410318180F49FEF701FFC4E71EF0010FC5
:102190003FF40BAFBBF1FF3F18BF5B4698D122E77E
:1021A00040F28031C2F20001CCF800E00B60EFE6B3
:1021B000B8F1090F9CBF08F1010B92467FF672AF90
:1021C0006DE700BF380300202DE9F04F874B85B045
:1021D0001A68874D002A40F09B802B68002B58D14D
:1021E000DFF820A2DAF800201D2A55D8DFF80CB25B
:1021F000DFF818829BF800009BF801109BF8022082
:102200008DF80C008DF80D108DF80E209946D8F839
:1022100004400F2C2ED9A4F10F05012D64D0A4F198
:102220001103092B69D9092D5ED904EB840304EB52
:102230004303103CA9F1BB070126A51E092C1F442E
:1022400009D9082D45D90136163F6B1C2C460FD0F5
:10225000A51E092CF5D89BF8013007F10B00B3FB44
:10226000F6F303A98DF80D30FEF790FE002CE8D1AF
:10227000D8F8044009F101090134B9F10B0F48F80D
:10228000044FC4D1FEF776FCDAF800300133CAF807
:10229000003005B0BDE8F08F564B03F16E0403E04B
:1022A000A34203F8010C0ED013F8012B02F0020137
:1022B000C9B242F0040022F004020029F0D1A34286
:1022C00003F8012CF0D10420FFF73AF801232B602A
:1022D000DFE79BF801303846B3FBF6F303A98DF82E
:1022E0000D30FEF753FEAEE705EB850005EB400031
:1022F00048444149FEF74AFE97E705EB850005EBA8
:102300004000A9F11603C0183C49FEF73FFE8AE7DA
:102310003B4A002617681E603A4B3F243A4602A803
:1023200069461E6010238DF806308DF800408DF848
:1023300001408DF805402E608DF802608DF8046034
:10234000FEF7AEFC3A4603A801A9FEF7A9FC2E4B06
:102350009DF808809DF80E709DF809C09DF80AE070
:102360009DF80C409DF80D002349244A33F818903D
:1023700033F8144033F81CC033F81EE033F8100073
:1023800033F8173046F267671470DFF8848081F8FD
:10239000009081F801C081F802E0507093703446DB
:1023A000C6F2666711E008F0E5FE87FB0032C3174E
:1023B000C3EBA20303EB8303A0EB430048F8060042
:1023C000013404360B2C3FF408AFE207EBD408F0DD
:1023D000D1FE87FB0032C317C3EBA20303EB8303D9
:1023E000A0EB4300053048F80600E9E7FC030020B5
:1023F0009425002098250020D8030020B003002059
:1024000090010020480300209CC100080004002027
:1024100004040020704700BF074B012003F16E0148
:1024200013F8012B12F0020214BF03F8010C03F899
:10243000012C8B42F4D17047982500202DE9F84FEC
:102440009246814688460AB9BDE8F88F0020FEF71B
:10245000B3FD1AF0080F40F095801AF0100F40F00D
:102460008D80DFF87CB14146DBF80000FEF786FB8B
:102470004CF6CD42CCF6CC42A2FB08324F4B920830
:10248000197802EB420201EBC101C9004C4B01EB90
:1024900042021AF0040F02EB0301D05CD4D0494A87
:1024A000494F00249460D4601461546114605460F6
:1024B000148394763B4607F16E05012613F8014B11
:1024C00014F0020414BF03F8016C03F8014CAB4292
:1024D000F4D1DBF80030002B62D03C4B1B68DC07EA
:1024E00062D501235370937000230125CC18A47882
:1024F000013314B1042B1555F8D1B9F10B0F4B78FA
:1025000088BFA9F10C099944B9F10B0F304B88BF72
:10251000A9F10C0900EB400009EB800913F8191030
:1025200003EB490329B15B78012050540BB1254AD4
:10253000D054284CDFF8ACC004F11B06002514F879
:10254000013F9BB105EB0C03987815F80C205B78E4
:1025500060B102EB820102EB41021818D219D15C82
:1025600041F00201D15401338342F8D10335B44222
:10257000E5D1194B01221A60BDE8F88F0120FEF762
:102580007FFB6EE706F02AFDC820FEF759FA134BD1
:102590001B68002B7FF465AF0120FEF751FB60E75D
:1025A0001AF0100FE5D14FE7B8F1040F99D9A8F14F
:1025B0001E08B8F1040F97D893E700BF7C030020F2
:1025C000A4C20008BC030020982500207800002049
:1025D000B8C40008BB030020FC030020A8030020AF
:1025E0006001002064C4000840F27803C2F20003D6
:1025F0001868704738B50B4B04461B680A4D032B0F
:1026000004D0820702D52B689B0707D5FEF7B8FBDD
:10261000064B01222C601A60204638BDFEF77AFA7C
:10262000F4E700BFA803002078000020FC0300208E
:1026300040F2A833C2F2000318687047032810B5AF
:1026400009D8074C2368834203D02060FEF798FB2B
:102650002368184610BD024B1B68184610BD00BF0A
:10266000A803002040F26C13C2F200031868704700
:102670003B28024B88BF3C20186070476C0100204B
:1026800040F29813C2F20003186870473A28024BD0
:1026900088BF0020186070479801002040F27C330A
:1026A000C2F20003186870470328044B04D818606E
:1026B000034B01221A607047186870477C030020A2
:1026C000FC030020064B1868022805D9002018607A
:1026D000044B01221A60704701301860F8E700BF10
:1026E0007C030020FC030020054B186828B101384A
:1026F0001860044B01221A60704703201860F8E745
:102700007C030020FC03002040F2E433C2F200030B
:1027100018687047074B10B5186000B110BD064B24
:102720000F241C60FEF7C2FC044B1C60BDE8104087
:10273000FEF7FABAE40300209001002058010020BF
:1027400040F29413C2F2000318687047024B0A2843
:102750008CBF18681860704794010020044B1868FB
:10276000092802D9002018607047013018607047AE
:1027700094010020044B186810B1013818607047AC
:102780000A201860704700BF94010020064B1B68A8
:10279000012B00D07047054B00223F2119705A7061
:1027A0009A70FEF783BC00BF8C0300205C01002000
:1027B00040F28C33C2F2000318687047012810B54C
:1027C000034602D9054B186810BD044C2068984296
:1027D00003D02360FFF7DAFF206810BD8C030020D0
:1027E000F0B5574B83B01B680446012B41D0022B38
:1027F00001D003B0F0BD20B9524B1A68002A78D03E
:1028000018600020FEF73CFA4F4B1B683B2B2DD87D
:102810001D2B71D967081E254C4A4D4B10785178F5
:10282000927833F8100033F8111033F81220454B2A
:102830008DF804001B688DF805108DF80620002B1C
:1028400045D1AF423CBF434E3C4605D338E07230E1
:1028500007F03CF9AC4233D2306801A920180134AA
:10286000A842F4D33C383B28F4D8F0E727463C256F
:10287000D2E70020FEF704FA334B1B683B2B47D905
:10288000344A3C231268A418304AA34298BFC3EBD1
:10289000040411782E4B9078557833F8111033F8E2
:1028A000152033F810303B2C8DF804108DF80520DE
:1028B0008DF8063004D804F1720001A907F006F97A
:1028C000254B1B68002B94D0FEF7A4F991E7214E0D
:1028D000002404E0723007F0F9F8BC42F0D8336805
:1028E00001A9E0180134A842F4D33C383B28F4D8BD
:1028F000F0E701221A6084E7132B7FF67AAF4AF6DD
:10290000AB27CAF6AA27A7FB043714257F0883E75D
:102910001D2B0ED8132B7FF66CAF4AF6AB23CAF6ED
:10292000AA23A3FB04240B4A1423126802EB5404C9
:10293000AAE7084A1E23126802EB5404A4E700BF6A
:10294000A8030020000400206C0100207400002077
:102950009CC10008980100206001002038B5874B19
:102960001B680A2B1DD8864A864C126892B9864D80
:102970002A68DAB9042B00F0E280844A844803EB29
:102980008303116800EB8303986801318142116071
:1029900045D238BD7E4A03EB830302EB83035B68B9
:1029A0009847794B1B68002BF3D0764C794B1B680A
:1029B000012B1FD0784B1B68032B06D02368002BFC
:1029C000E7D1BDE8384006F025BB744B74491A685E
:1029D000496B0132B2EB411F1A60EFD3714A0020FC
:1029E000116818604B1E052B3AD8DFE803F050A1A0
:1029F0009A938C856C4B6D491A6849690132B2EB28
:102A0000411F1A60D6D36A4A0020116818604B1E15
:102A1000052B0CD8DFE803F069625B544D440021BC
:102A20005B68116098472B68002BBED1B1E7614904
:102A30000B680133072B00F09E800B605E4913602A
:102A40000A685B4801320D2A0A6000F08B800E2A6A
:102A5000B0D1013B08BF0623036000230B60A9E748
:102A600056490B680133072B7AD00B605449136029
:102A70000A684C4801320D2A0A6068D00E2A9DD19E
:102A8000013B08BF0623036000230B6096E74D4B14
:102A900059783E29E4D801315970FEF745F98DE7A0
:102AA000494B99780029C2D001399970FEF7FEFA96
:102AB00080E7454B19783E29B9D801311970F5E7FF
:102AC000414B59780029B2D001395970EEE73E4B9D
:102AD00099783E29ABD801319970E7E73A4B1978DC
:102AE0000029A4D001391970E0E7374B59783E2905
:102AF0009DD801315970D9E7324B99780029AFD070
:102B000001399970C9E72F4B19783E29A8D80131AE
:102B10001970C2E72B4B59780029A1D0013959709F
:102B2000BBE7284B99783E299AD801319970B4E7D0
:102B3000244B1978002993D001391970ADE7144B53
:102B40005B6D98472B68002B7FF42FAF21E7013393
:102B5000072B18BF03607FF431AF012303602DE71B
:102B6000012382E70133072B18BF03607FF422AFF4
:102B7000012303601EE701235FE700BF94010020EB
:102B8000FC0300206001002094250020E0030020C9
:102B90007C0000208C030020A8030020600300209C
:102BA0002C00002078030020400400207001002049
:102BB000A40300203C0400206801002044030020FE
:102BC0006C000020700000205C010020064B1A7889
:102BD0003E2A07D803D13F221A70FEF767BA0232A5
:102BE0001A70FAE7704700BF5C010020064A1378AC
:102BF00043B1012B03D100231370FEF757BA023BF8
:102C00001370FAE7704700BF5C010020064B5A784A
:102C10003E2A07D803D13F225A70FEF747BA023244
:102C20005A70FAE7704700BF5C010020064A5378EB
:102C300043B1012B03D100235370FEF737BA023B97
:102C40005370FAE7704700BF5C010020064B9A788A
:102C50003E2A07D803D13F229A70FEF727BA0232E4
:102C60009A70FAE7704700BF5C010020064A93782B
:102C700043B1012B03D100239370FEF717BA023B37
:102C80009370FAE7704700BF5C01002040F25C13CC
:102C9000C2F200031A7802705A7842709B788370EF
:102CA000704700BF10B404784178827840F25C131A
:102CB000C2F200033F2C34BF20463F203F2928BFEB
:102CC0003F213F2A28BF3F22187059709A7010BCCC
:102CD000FEF7ECB940F27003C2F200031A780270FA
:102CE0005A7842709B788370704700BF10B40478A4
:102CF0004178827840F27003C2F200033F2C34BF67
:102D000020463F203F2928BF3F213F2A28BF3F229E
:102D1000187059709A7010BCFEF706B840F2901304
:102D2000C2F20003186870470F2803D8034B1860DD
:102D3000FEF7BCB9014B0F221A60F9E790010020A1
:102D4000034B1A6802B97047013A1A60FEF7AEB930
:102D500090010020044B1A680E2A00D970470132F6
:102D60001A60FEF7A3B900BF9001002040F258138B
:102D7000C2F20003186870470F2803D8034B18608D
:102D8000FDF7D2BF014B0F221A60F9E7580100206E
:102D900030B5012583B015F0010F0CBF002139219A
:102DA00015F0020F0CBF0022392215F0040F0CBFE2
:102DB000002339238DF804108DF805208DF8063096
:102DC0000024204601A9013406F080FEAE2CF8D183
:102DD000204606F0F5FD01350320FDF73FFE082DE6
:102DE000D9D10020FEF7E8F803B030BD284B2DE91B
:102DF000F04103F16E01012413F8012B12F00202DD
:102E000014BF03F8014C03F8012C8B42F4D1017874
:102E100000293AD080460746013705260020C6F132
:102E200005020346FEF722F898F8011059B30A2E5E
:102E300018D83D46344601E00A2C13D8002220461B
:102E40001346FEF713F815F8011F06340029F3D1D5
:102E500006E000222046202113460634FEF706F83D
:102E60000A2CF6D90420FEF76BFA3220FDF7E8FDB4
:102E7000013E02D017F8011CD0E718F8011F002905
:102E8000CAD1BDE8F0813446EAE7BDE8F08100BF71
:102E90009825002070B51B4D82B02B6804460BB9F5
:102EA00002B070BD4208184901A808F0AFF900202F
:102EB000FEF782F8154B04F0010603F16E000124C1
:102EC00013F8012B12F0020214BF03F8014C03F8AF
:102ED000012C8342F4D1002002469DF80410012306
:102EE000FDF7C4FF0022012306209DF80510FDF721
:102EF000BDFF28687100FDF741FE054B01221A60F5
:102F0000CEE700BF600100201CC200089825002009
:102F1000FC0300202DE9F04FBA4B04461B6893B028
:102F2000184613B913B0BDE8F08F3F268DF8346012
:102F30003C2603258DF82360162600230CA92A467B
:102F4000A4208DF824600F268DF835308DF83630AA
:102F50008DF825308DF826308DF82B308DF82750E0
:102F60008DF8296000F0B0FB01220DF12101A720AE
:102F700000F0AAFB01220DF12501A82000F0A4FB1E
:102F800001220AA9BD2000F09FFBBE2001220DF105
:102F90002A0100F099FBB4F5843F80F0A4809DF8ED
:102FA00021809DF822C0B8F1030F88BF4FF00008C0
:102FB0009DF825E088BF8DF82180BCF1030F84BF08
:102FC0004FF0000C8DF822C09DF82610BEF10A0FBC
:102FD00084BF4FF0000E8DF825E0012902D90021B1
:102FE0008DF826109DF828700F2F02D90F278DF825
:102FF00028709DF829600F2E71D89DF82A000128AD
:1030000002D000208DF82A009DF823203C2A00924F
:1030100003D93C258DF8235000959DF824303B2B97
:1030200002D916238DF82430774C07932568774B07
:1030300001959DF827509DF834B002959DF83050C9
:103040009DF835A003959DF831509DF83690049574
:103050009DF8325083F800B005959DF82B5083F809
:1030600001A0069540F27C35C2F20005C5F800804B
:10307000DFF8C481029DC8F800C0DFF8C0C183F842
:103080000290CCF80050DFF8B8C1614BCCF800E0FA
:10309000DFF8B0E15F4ACEF800101F6003995E4B85
:1030A0001170049D05991E605C4B557091701860FD
:1030B000009A5B4B079D1A605A4B06991D605A4B4C
:1030C000196000232360FDF72FFEFDF7EFFF019A43
:1030D0002260FFF75BFBFDF753FE012022E70F267E
:1030E0008DF8296089E7A92001220DF1260100F061
:1030F000EBFA40F6FF03C0F201039C427FF64FAFAC
:1031000001220DF12701BC2000F0DEFA0DA92A46AC
:10311000D72000F0D9FA01220DF12901DA2000F0C0
:10312000D3FADB2001220DF1220100F0CDFAB4F533
:10313000003FFFF434AF01220DF12301DC2000F049
:10314000C3FADD20012209A900F0BEFAFF23C0F274
:1031500002039C427FF623AF0DF12B010122E020F8
:1031600000F0B2FA0FA90B22E52000F0ADFA0EAE86
:103170000BA9022240F2251000F0A6FA40F2351009
:103180003146042200F0A0FA0DF14605274B0DF15F
:103190003B0005E042F002021A611433A84212D04B
:1031A00010F8012FFF2AF8D002F01001C9B202F086
:1031B0000F029A601A690029ECD122F002021A610A
:1031C0001433A842ECD19DF82C301948FF2B1EBFB8
:1031D000184A03F00F0353609DF82D30FF2B1EBFDC
:1031E000144A03F00F0353610023F25C00EB031158
:1031F0000133FF2A1CBF02F00F024A60042BF4D1F6
:10320000CDE600BF640400206001002070000020B3
:10321000900100205C01002058010020E403002000
:103220006C01002098010020740300207C00002025
:103230002C00002070010020A8030020780000204E
:10324000940100208C0300202DE9F04F854BA3B0A2
:103250001B68002B00F08C80834B844A93F800801D
:1032600093F801C093F802E0814B92F800B01F6818
:10327000804B92F801A01E687F4B92F802901D6867
:103280007E4B8DF819501C687D4B8DF81A401B68D9
:103290008DF820B000937B4B009C1B688DF81B4081
:1032A0000193794B019C1B688DF821A00293774B09
:1032B0008DF822901B688DF824800393744B8DF851
:1032C00025C01868734B8DF826E01968724B8DF88D
:1032D00015701A688DF816608DF81C40029C6F4BB3
:1032E0008DF81D40039C8DF817008DF81E408DF859
:1032F000181000208DF81F2012ACFF250A2888BF67
:10330000255409D89A68196902F00F0289072254D6
:1033100044BF42F010022254013014334028EDD152
:103320005F4800230AAEFF22012B9BBF00EB031175
:103330004968F25401F00F0198BFF1540133102B8A
:10334000F2D1584800230EADFF21032B9BBF00EBA9
:1033500003125268E95402F00F0298BFEA54013395
:10336000102BF2D1A42008A9032200F0C7F918B944
:10337000002023B0BDE8F08FA7200DF11501012238
:1033800000F0BCF90028F3D0BC200DF11901012296
:1033900000F0B4F90028EBD0A8200DF11A010122A9
:1033A00000F0ACF90028E3D0A9200DF11B010122A7
:1033B00000F0A4F90028DBD0BD2007A9012200F00D
:1033C0009DF90028D4D0BE200DF11E01012200F08D
:1033D00095F90028CCD0D72009A9032200F08EF956
:1033E0000028C5D0DA200DF11D01012200F086F978
:1033F0000028BDD0DB200DF11601012200F07EF97E
:103400000028B5D0DC200DF11701012200F076F97B
:103410000028ADD0DD2006A9012200F06FF90028B8
:10342000A6D0E0200DF11F01012200F067F900286D
:103430009ED0E5202146402200F060F9002897D078
:1034400040F225103146102200F058F900288FD0A4
:10345000102240F23510294600F050F9003018BF14
:10346000012086E764040020700000205C01002039
:103470007C030020A8030020780000209401002095
:103480008C0300209001002058010020E40300205C
:103490006C01002098010020740300207C000020B3
:1034A000700100202C00002006F03ABB2DE9F84303
:1034B00081468846174605F029FC10B90020BDE872
:1034C000F883552005F0CAFC2E48082105F002FDBE
:1034D000442005F0C3FC002443F2144505F080FCB1
:1034E0000134AC4298BF002814BF00260126F5D055
:1034F00043F214439C4227D805F008FC0028DDD095
:10350000552005F0ABFC204C08211E4805F0E2FCDC
:10351000BE2005F0A3FC0921204605F091FC05F032
:10352000F5FB1A4B1B68222B13D0282B11D0092333
:10353000C9F8003094F901300120DB0FC8F80030E1
:1035400023783B60BDE8F88305F0E0FB3046BDE83A
:10355000F88323796278C3F341132578093302F0A5
:103560000704C3F10C00191F45FA00F004FA01F139
:10357000D2090143C9F800300120C8F800203960A1
:10358000BDE8F883580400204404002054040020BF
:10359000F8B5A0F10905032D044602D900263046EE
:1035A000F8BD05F0C7FC05F0B1FB0028F6D02E4FA2
:1035B000384605F09DFC3B782C4A012113602C4ACB
:1035C000222B0646116001D0282BE8D105F09EFB86
:1035D0000028E4D0552005F041FC264F0821224860
:1035E00005F078FCBE2005F039FC0921384605F0CD
:1035F00027FC3B79C3F341130933A342CFD005F035
:1036000085FB0028CBD0552005F028FC0821164862
:1036100005F060FC4E2005F021FC7F2005F01EFC2B
:10362000802005F01BFC680100F0E00005F016FCAE
:1036300005F06CFB05F06AFB0028B0D0552005F0C2
:103640000DFC0948082105F045FC482005F006FC62
:10365000002405F0C5FB0134F92C98BF0028F8D0F0
:1036600005F054FB9BE700BF5804002054040020E1
:1036700050040020440400202DE9F04184B003F000
:1036800027F8DFF8408000240127650045F0A005F9
:10369000012600972846002132460DF10F03A41998
:1036A000C8F8005003F04CF830B1082CEDD1044BB1
:1036B000186804B0BDE8F081014B30461E60F8E7A1
:1036C000640400206004002010B50A4B82B01C681E
:1036D0000B4614B9204602B010BD0092064A0146BE
:1036E00012681046012203F02BF8D0F1010038BF18
:1036F0000020F0E764040020600400202DE9F0477A
:10370000144B82B01B68174603B3EAB1DFF84CA034
:10371000114C0646C0EB01094FF001080025DAF80C
:103720000000CDF800803146012209EB060303F0CA
:1037300085F858B910202368002BFCD0013825608B
:10374000F9D10136013FEAD1012000E0002002B0AA
:10375000BDE8F087640400200826002060040020F3
:1037600030B53A4B87B01A68044682426BD068463F
:103770001C6006F0F1FC02A807F066F804200121A5
:1037800006F0B6FE0420012106F0B2FE4FF4003030
:10379000012106F0BBFE04234FF400600325C4F2B0
:1037A00001006946ADF8003018238DF803308DF81C
:1037B000025006F06DFC08234FF40060C4F20100D3
:1037C0006946ADF8003048238DF803308DF802507B
:1037D00006F05EFC4FF48840C4F20000012107F0BF
:1037E00071F800234FF488401D46C4F2000002A97E
:1037F000ADF80C30ADF80E30ADF81030ADF8143037
:103800000C23ADF81230029406F0B8FF4FF4884054
:10381000C4F20000012107F023F84FF48840C4F2FD
:10382000000040F22551012207F028F826238DF8E8
:10383000043001A801238DF805508DF806508DF84D
:10384000073006F02FFA07B030BD00BF6804002033
:1038500030B40F4A13687F2BFCD80E490E4D0B680D
:103860005C1C7F2C45F8230098BF0C6001D9002315
:103870000B6072B613680133136062B64FF4884070
:10388000C4F2000040F22771012230BC06F0F6BFFE
:10389000780600207C0600207004002010B5044645
:1038A000007828B1FFF7D4FF14F8010F0028F9D1F0
:1038B00010BD00BF40F26C43C2F200031868003034
:1038C00018BF0120704700BF30B40D4B1A6882B199
:1038D0000C490D4D0A68541C802C55F8225018BF15
:1038E0000C6009D072B61A68013A1A6062B60122F9
:1038F0000560104630BC704700220A60F2E700BF46
:103900006C0400207006002080060020024A136824
:10391000002BFCD1704700BF780600204FF4884090
:1039200038B5C4F2000040F2255106F0D9FF002856
:103930002BD14FF48840C4F2000040F2277106F00A
:10394000CFFF00B938BD4FF48840C4F2000040F208
:10395000277106F0EBFF234B1A68002A38D0224A61
:10396000224C1168481C802808BF002054F8211000
:1039700010601A684FF48840013AC4F2000089B21E
:103980001A60BDE8384006F095BF4FF48840C4F295
:10399000000040F2255106F0C9FF4FF48840C4F200
:1039A000000006F08BFF124B1A687F2AC1D811491C
:1039B000114D0A68C0B2541C7F2C45F8220098BFF4
:1039C0000C6001D900220A601A6801321A60B0E75F
:1039D0004FF48840C4F2000040F22771BDE838403F
:1039E00006F04CBF780600208008002070040020FC
:1039F0006C0400207406002080060020F0B583B01F
:103A000001A84FF40065C4F2010506F0A5FB0420EF
:103A1000012106F06DFD012402271026284601A988
:103A2000ADF804408DF806708DF8076006F030FBA5
:103A30000420214606F05CFD284601A9ADF804707B
:103A40008DF806708DF8076006F022FB04202146F1
:103A500006F04EFD284601A9ADF804608DF8067009
:103A60008DF8076006F014FB28462146224606F032
:103A700081FB28463946224606F07CFB2846314623
:103A8000224606F077FB03B0F0BD00BFF8B5094D44
:103A900004460F46002601E02B6833B92046FFF7A5
:103AA00013FF0028F8D00120F8BD0136BE4228607F
:103AB000F4D3F8BD0C2600202DE9F04F85B0054663
:103AC00003F004FDFFF722FFFFF7F4FE002843D0C8
:103AD0000024624FDFF888A10126A346294603A8E7
:103AE000FFF7D4FFDFF874914FF001080346002878
:103AF00035D0039B3E600A2B07D00D2BEED0FF2C58
:103B0000ECD80AF804300134E8E70AF804B0002CD5
:103B100032D103F0DBFCE1E7514852491A4607F085
:103B2000C0FB00284CD04E484F49032207F0B9FB98
:103B300000284FD04A484D49052207F0B2FB002823
:103B400055D14B484B49022207F0ABFB002849D125
:103B50000123C9F80830062005B0BDE8F08F4648BB
:103B6000019303F085FC454803F082FC444803F0D0
:103B70007FFC019B1846EFE73F48019303F078FC78
:103B8000374803F075FC3E4803F072FC34483D4969
:103B9000022207F086FB38B131483B49052207F085
:103BA00080FB18B90220D7E74046D5E72C483749B3
:103BB000022207F076FB019B0028ADD10320CBE762
:103BC00009F13C0032490F2207F084FBC9F8048058
:103BD0000420C1E709F11C002E491F2207F07AFBDF
:103BE0000520B9E70023C9F808300620B4E71C48CF
:103BF0002949052207F055FB98B1194827490922A0
:103C000007F04FFB10B316482549042207F049FB83
:103C1000A8B113482349092207F043FB40B1FF2014
:103C20009AE7214812490F2207F054FB072093E737
:103C30001E481F49FF2207F04DFB0A208CE71D4854
:103C40001D491F2207F046FB092085E71B4818493C
:103C50000F2207F03FFB08207EE700BF840800200A
:103C6000540A002008C5000814C5000818C500083B
:103C7000590A002020C50008E8C40008ECC4000868
:103C8000F4C40008F8C40008FCC4000804C5000817
:103C90005E0A0020570A002024C500082CC5000831
:103CA00038C5000840C50008F0090020D0080020F1
:103CB0005D0A0020D0090020580A0020900800204A
:103CC000F0B583B0074607F0E4FA06461A4803F059
:103CD000CFFBBEB13C46F61904E0184603F0A2FB48
:103CE000B4420FD014F8013B6846A3F120055E2DC5
:103CF00012491A46F1D907F089FA684603F0B8FB71
:103D0000B442EFD10E4803F0B3FB03F0DFFB3846BB
:103D1000FFF7C4FD0B48FFF7C1FDFFF7F7FD02E019
:103D2000022807D020B10A20FFF7C6FE0128F7D1EC
:103D300003B0F0BD0020FBE74CC5000860C50008DB
:103D400054C5000828C7000838B539B104464518DD
:103D500014F8010BFFF77CFDAC42F9D1BDE8384007
:103D6000FFF7D4BD40F68400C2F20000704700BFE8
:103D700010B54FF40060C4F201000121002282B0AE
:103D800006F0F8F90C4A0521144600201368002BB0
:103D9000FCD001392060F9D101214FF40060C4F258
:103DA00001000A4606F0E6F901A83221FFF76EFE8F
:103DB0000028F9D102B010BD0C26002008B502463B
:103DC0000B460748074907F021FA0548FFF778FF37
:103DD00020B1054B002283F83C205A6008BD00BF8B
:103DE000000A002068C500088408002008B50246C3
:103DF0000B460748074907F009FA0548FFF760FF37
:103E000020B1054B002283F83C205A6008BD00BF5A
:103E1000000A002078C500088408002008B5024682
:103E200008B1037823B90748BDE80840FFF748BF49
:103E30000549064807F0EAF90448BDE80840FFF7DD
:103E40003FBF00BFA4CB000888C50008000A0020BF
:103E500030B54FF4E13083B003F0D2FBFFF7CEFD75
:103E60004FF4E130FFF77CFC4FF40060C4F2010036
:103E70001021002206F07EF91F4C4FF40060002252
:103E8000C4F20100012106F075F905252246002340
:103E900021680029FCD0013D1360F9D101214FF4C4
:103EA00000600A46C4F2010006F064F912493222A9
:103EB0002368002BFCD0013A0D60F9D14FF400606B
:103EC000C4F201001021012206F054F903E001A818
:103ED00003F0DAFA60B901A8FFF7F6FC0028F6D083
:103EE000019803F09FFA01A803F0CEFA0028F2D05F
:103EF0000198FFF7ADFCEEE70C26002008B50B4B50
:103F00001A6802B108BD01224FF4E1301A6003F0D3
:103F100077FB074803F0ACFAFFF770FD4FF4E13090
:103F2000FFF71EFCBDE80840FFF722BF500A002043
:103F300094C5000810B403781649FBB1002208604C
:103F40001446013005E001300E2A14DC10F8013C63
:103F50008BB13D2B02BF01EBC20300F8014C58604E
:103F6000F1D0262BEFD1013200F8014C41F832009C
:103F700001300E2AEADD531C0F2B08DC002201EB76
:103F8000C30011460133815008320F2BFADD10BCFB
:103F9000704700BF6C0B0020F8B50A4D06460024A0
:103FA00055F83430E70031461846013423B107F0A4
:103FB0005EF918B1102CF3D10348F8BD014BDF199D
:103FC0007868F8BD6C0B0020B0C6000808B5FFF794
:103FD000E3FF4CF28C61C0F6000107F048F9D0F124
:103FE000010038BF002008BD00B50B4685B04CF27B
:103FF00094610246C0F60001684607F007F968467A
:10400000FFF7CAFF05B000BD10B5044607F041F93F
:10401000014600B910BD2046BDE81040FFF794BE30
:1040200010B504464CF29C60C0F60000FFF7ECFFB0
:104030004CF2AC60C0F60000FFF7E6FF4CF2B46053
:10404000C0F60000FFF7E0FF4CF2C060C0F60000D1
:10405000FFF7DAFF4CF2CC60C0F60000FFF7D4FFA8
:104060002046FFF7D1FF4CF2D460C0F60000FFF706
:10407000CBFF4CF2E060C0F60000FFF7C5FF4CF24A
:10408000EC60C0F60000FFF7BFFF4CF2F860C0F62E
:104090000000FFF7B9FF2046FFF7B6FF4CF20070B3
:1040A000C0F60000BDE81040FFF7AEBF38B50446CB
:1040B0004CF20870C0F600000D46FFF7A5FF204641
:1040C000FFF7A2FF4CF21470C0F60000FFF79CFF50
:1040D0002846FFF799FF4CF21870C0F60000BDE8C3
:1040E0003840FFF791BF00BF4CF2B0604CF22C712A
:1040F00008B5C0F60000C0F60001FFF7D7FF4CF28C
:1041000034704CF23C71C0F60000C0F60001FFF7BD
:10411000CDFF4CF648704CF24471C0F60000C0F67A
:104120000001FFF7C3FF4CF250704CF25471C0F61F
:104130000000C0F60001FFF7B9FF4DF2C0004CF2DD
:104140005871C0F60000C0F60001FFF7AFFF4CF257
:1041500060704CF26C71C0F60000C0F60001FFF711
:10416000A5FF4CF278704CF28471C0F60000C0F6E6
:104170000001FFF79BFF4CF290704CF29871C0F673
:104180000000C0F60001FFF791FF4CF2A070C0F6EE
:104190000000BDE80840FFF737BF00BF054A1368BD
:1041A00001331360DB0702D40348FFF72DBF034838
:1041B000FFF72ABF380C0020BCC70008A4C70008BE
:1041C00010B504464CF2C470C0F60000FFF71CFFA7
:1041D0002046FFF719FF4CF2CC70C0F60000BDE896
:1041E0001040FFF711BF00BF70B584B00C46054604
:1041F0001B49164668461A4607F008F802A81849EF
:10420000089A07F003F83CB123782BB12046FFF75A
:10421000FBFE1448FFF7F8FE1348FFF7F5FE2846AB
:10422000FFF7F2FE1148FFF7EFFE2846FFF7ECFE1E
:104230000F48FFF7E9FE3046FFF7E6FE0D48FFF7AF
:10424000E3FE6846FFF7E0FE0B48FFF7DDFE02A83D
:10425000FFF7DAFE0948FFF7D7FE04B070BD00BFD4
:10426000DCD2000874CE0008D4C70008ECC70008F0
:10427000F8C7000804C8000814C8000814C70008DC
:1042800010B504464CF62000C0F60000FFF7BCFE57
:104290002046FFF7B9FE4CF65400C0F60000FFF7C9
:1042A000B3FE4CF66400C0F60000BDE81040FFF716
:1042B000ABBE00BF70B505460F480E46FFF7A4FE23
:1042C0000E48FFF7A1FE002E0EDD043D00240C4831
:1042D000FFF79AFE55F8040FFFF796FE01340948E0
:1042E000FFF792FEB442F2D10748FFF78DFE074B6D
:1042F00000221A6070BD00BF6CC80008BCC700086F
:1043000088C80008A0C8000880C80008380C002031
:104310004CF6B000C0F60000FFF776BE38B5044694
:104320004CF6C000C0F600000D46FFF76DFE2046BB
:10433000FFF76AFE4CF21470C0F60000FFF764FE4F
:104340002846FFF761FE4CF6EC00C0F60000BDE821
:104350003840FFF759BE00BF4CF6FC0008B5C0F668
:104360000000FFF751FE4CF60810C0F60000BDE853
:104370000840FFF749BE00BFF0B5044683B01F48B0
:104380001E460D461746FFF73FFE2046FFF73CFE50
:104390001B48FFF739FE2046FFF736FE1948FFF7A6
:1043A00033FE002E24DD043D00240BE01648FFF709
:1043B0002BFE55F8040FFFF727FE1448FFF724FEE5
:1043C000B44215D02246124901A806F01FFF114839
:1043D000FFF71AFE01A8FFF717FE0F48FFF714FEBC
:1043E000BC4204F10104E1D10C48FFF70DFEDDE70A
:1043F0000B48FFF709FE03B0F0BD00BF14C9000869
:10440000ECC7000824C9000820CA000854C90008E5
:10441000DCD2000838C9000800C8000848C90008F4
:104420002CC9000870B50E4605460E481446FFF725
:10443000EBFD3046FFF7E8FD0B48FFF7E5FD2846AA
:10444000FFF7E2FD0948FFF7DFFD14B10848FFF769
:10445000DBFD0848FFF7D8FD0748BDE87040FFF7CF
:10446000D3BD00BFC4C7000860C9000884C90008E4
:1044700098C9000820CA0008CCC700082DE9F041FF
:10448000069F044616469846079D11B10B78002BEF
:1044900049D12848FFF7B8FD2046FFF7B5FD26486B
:1044A000FFF7B2FD2046FFF7AFFD2448FFF7ACFD54
:1044B0003046FFF7A9FD2248FFF7A6FD4046FFF76B
:1044C000A3FD2048FFF7A0FD3846FFF79DFD55B13D
:1044D0002B7843B11C48FFF797FD2846FFF794FD62
:1044E0001A48FFF791FD1A48FFF78EFD2046FFF7A7
:1044F0008BFD1848FFF788FD2046FFF785FD16481D
:10450000FFF782FD1548FFF77FFD2046FFF77CFD92
:104510001348FFF779FD3046FFF776FD1148BDE8F7
:10452000F041FFF771BD0846FFF76EFD0E48FFF73B
:104530006BFDAEE7A0C90008ECC70008F8C700088B
:10454000BCC90008C4C90008CCC90008DCC90008FF
:10455000E0C90008ECC90008FCC9000808CA000846
:1045600018CA000824CA000874CE00084CF630208F
:10457000C0F600000321FFF7E7BB00BF10B50446FB
:104580004CF2C470C0F60000FFF73EFD4CF634213B
:104590002046C0F60001FFF7C1FE4CF66400C0F6ED
:1045A0000000BDE81040FFF72FBD00BF70B5064604
:1045B0004CF2C47082B0C0F600000D461446FFF7FE
:1045C00023FD4CF2B0614CF63C23C0F60001C0F66E
:1045D00000033046009301912A462346FFF74EFF21
:1045E0004CF66400C0F6000002B0BDE87040FFF772
:1045F0000BBD00BF38B505460C46FFF7CFFD28467A
:10460000FFF7DEFD2046FFF7DBFD4CF2B060C0F6A1
:104610000000FFF7D5FD4CF68000C0F60000BDE8B5
:104620003840FFF7F1BC00BF10B504464CF64020FF
:10463000C0F60000FFF7E8FC2046FFF7E5FC4CF66B
:104640002410C0F60000BDE81040FFF7DDBC00BF3D
:1046500010B50446FFF7A2FD2046BDE81040FFF765
:10466000E3BF00BF4CF66020C0F60000FFF7CCBCF3
:1046700008B5FFF7F7FF4CF68000C0F60000BDE874
:104680000840FFF7C1BC00BFF0B50E4683B014462A
:104690001F46089DFFF7DCFF3046FFF791FD4CF207
:1046A000C470C0F60000FFF7AFFC4CF2B061C0F67A
:1046B00000013A462B4620460095FFF795FD4CF247
:1046C000CC70C0F60000FFF79FFC2046FFF7D8FD36
:1046D00003B0BDE8F040FFF7CBBF00BFF8B5069DC3
:1046E0000E4614461F46FFF7B3FF3046FFF768FD3E
:1046F000204639462A46FFF795FE2046FFF7C0FDC3
:10470000BDE8F840FFF7B4BF2DE9F0410F4614466D
:104710009846069E079DFFF79BFF3846FFF750FD22
:104720004CF2C470C0F60000FFF76EFC4146324602
:104730002B462046FFF720FE4CF2CC70C0F600005E
:10474000FFF762FC2046FFF79BFDBDE8F041FFF755
:104750008FBF00BF2DE9F04F83B08B46924699463C
:104760000C9D0D9FFFF774FF1148FFF729FD1148BD
:10477000FFF74AFCDFF8488000242E595BF804005C
:1047800033463E595AF8041059F804208DE8400188
:10479000FFF774FE04340848FFF736FC0C2CECD10C
:1047A0000648FFF76DFD03B0BDE8F04FFFF760BFAF
:1047B0006CCA000874CA000880CA000828D1000822
:1047C0007CCA00082DE9F04F05460E46C5B0854865
:1047D0002946934602F004FF33781BB3741C4FF054
:1047E0002008002706E02B2B08BF04F8018C14F8E2
:1047F000013BBBB1252BF6D120460221FBF7B2FDD0
:10480000A27804F8010C002A00F04485234603F83E
:10481000012B9A781946002AF9D10F7014F8013B40
:10482000002BE7D13146704802F0DAFE3046FFF740
:1048300081FB28466D4906F01AFD002842D0284623
:104840006B4906F014FD0446002800F0CF8328468B
:10485000684906F00CFD002800F07484284666497B
:1048600006F005FD0446002800F0868128466349CD
:1048700006F0FDFC002800F06D852846604906F032
:10488000F6FC002800F0EA8728465E4906F0EFFCB7
:10489000002800F04D8228465B4906F0E8FC00281D
:1048A00000F000875948FFF7AFFB5948FFF7ACFB12
:1048B0005848FFF7A9FB0026FFF758FE304645B0E1
:1048C000BDE8F08F544C18AF3CAD04F1080694E8F5
:1048D0000300039587E803000FCE0FC596E8030099
:1048E00023AA04F12006914685E8030007920FCE23
:1048F000A9E80F00366828AD04F1480C06970DF1C1
:10490000C8082DAFC9F80060049504F1340EE246E2
:104910002E4644463D46BEE80F000FC6BCE80F00D9
:104920000FC5BAE80F000FC4DCF80030DEF8002035
:1049300005942B6016AC059D13A90894326037943A
:1049400014AA12A81AAC0DF1440A2B603A913B92BA
:104950000594CDF8E0A0399002F096FF814602F070
:1049600099FF2E49C0F30742C0F30723059806F0CC
:104970004DFC02F095FF42690446002A54DB0369AE
:10498000002B51DBC16800294EDB806800284BDB1F
:104990006568002D48DBB2F5966F45DC0C2B43DCD7
:1049A0001F2941DC17283FDC3B2D3DDC02F26C72F5
:1049B00008981B4906F02AFC226950460132194921
:1049C00006F024FCE26812A8164906F01FFCA26853
:1049D00013A8144906F01AFC14A81249626806F0DC
:1049E00015FC2CE014CC000828CC000840CC0008B2
:1049F00068CD0008DCCE0008C0CF000844D0000815
:104A00007CD1000838D20008E0D200082CD300087E
:104A1000ACC6000844D30008A8C5000844CC000870
:104A200050CC000854CC000800238DF858308DF885
:104A300044308DF848308DF84C308DF85030964821
:104A4000FFF7AAFA0546002801F05B80934906F0BB
:104A50000EFC002841F01E80914C49269148FFF73A
:104A6000DFFADFF8C8A2FFF73FFB06980221FFF745
:104A700021FC8D484946FFF7BDFDDAF800308B4A2E
:104A80008B498C48002B18BF1146FFF7B3FDDAF8AD
:104A90000030002B40F0F887FFF73AFC039806211E
:104AA000FFF708FC8448FFF7D3FD4FF00009059598
:104AB000DDF820A00394079DDDF810B002E037ABCD
:104AC00059F803A07D48FFF79FFA58F8094055F8B8
:104AD00009005BF8091057F8093052460094FFF7B7
:104AE00083FB09F104097648FFF78EFAB9F1140F38
:104AF000E5D17448039C059DFFF7C2FBFFF7B8FDA5
:104B0000FFF706FC06980221FFF7D4FB6A481E2730
:104B100003466D4A6D490097FFF7B6FDFFF7F8FBB6
:104B20006548FFF781FD6A486A49FFF7F7FB6A4865
:104B30006A49FFF7F3FB59486949FFF7EFFB6948FA
:104B40006949FFF7EBFBFFF78DFD44B16748FFF7BD
:104B50005BFA2046FFF758FA6548FFF755FA2846F2
:104B6000604906F084FB0446002800F0EF84FFF75C
:104B7000F3FBFFF7FBFCA1E65E4B3CAD93E80300C3
:104B8000039585E80300FDF7BFFD80464248FFF727
:104B900003FA0546002801F00782574906F067FB33
:104BA0000646002801F04E812846544906F05FFB76
:104BB0000646002801F025802846514906F057FB9B
:104BC0000546002841F0EC814E48FFF7FFF910F14F
:104BD000000818BF4FF00108CBF800804C260023D6
:104BE0008DF8B4300A24FBF755FB0DF13200FBF7CA
:104BF00061FB002841F010810A20FBF721FF013CF6
:104C0000F3D144AF3F2327F85C3D02F05DFA3E4903
:104C100082B232A806F0FAFA02F05CFA3A4982B29D
:104C200037A806F0F3FA3948FFF7FAF9FFF75CFA0C
:104C300003980221FFF73EFB35483946FFF7DAFCBF
:104C4000344832A9FFF7D6FC334837A9FFF7D2FC26
:104C50002C4A324B2E493248CDF80080FFF73EFDFA
:104C6000FFF756FB2E48FFF7DFFC23482D49FFF7DF
:104C700055FB22482C49FFF751FBFFF7F3FC002DB1
:104C80003FF475AF1948FFF7BFF92846FFF7BCF9A5
:104C90001748FFF7B9F96AE75CCC000864CC000854
:104CA00098CA0008B4CC0008C0CC000848DB000853
:104CB000E8CA0008C8CC0008B0C60008C4C700088D
:104CC000CCC7000884CC0008ACCC0008E0CC0008BD
:104CD0006CCC0008E8CC000874CC0008F4CC0008C8
:104CE00000CD000818CD000824CD000830CD000804
:104CF000D0CE0008A8C50008C8CF0008D0CF000853
:104D0000D8CF0008DCCF00081CC20008E4CF0008A0
:104D100054C70008F4CF0008F8CF0008FCCF000803
:104D200050C7000814D000082CD0000864040020EC
:104D30003CAD039523AD924A079528AD0495039D9C
:104D400002F150031EAC02F1180702F10C0E02F141
:104D5000240602F1300A07CA84E807000FCB85E871
:104D60000F009EE80700079DDFF878C285E807007E
:104D700097E80700049D0DF1C80885E8070096E84C
:104D8000070088E807009AE80700DCF800300DF11A
:104D9000DC0989E807007B4F53B97B4D3B6A3968D2
:104DA0003A69386B85E80E000123E860CCF80030E2
:104DB000FDF73EFC0690FDF755FC0590FDF760FC05
:104DC0000890FDF711FC00F002000990FDF7CEFFFE
:104DD0008246FDF799FC0A900DA8FDF77BFF6B4812
:104DE000FFF7DAF80546002800F01087684906F05A
:104DF0003EFA0346002801F07E802846654906F009
:104E000036FA0346002801F0F6802846624906F08B
:104E10002EFA0346002801F0B98128465F4906F0C2
:104E200026FA0646002801F0008328465C4906F071
:104E30001EFA0646002801F0DD822846594907225D
:104E400006F02FFA0646002801F0CB822846564984
:104E5000042206F026FA0646002801F05A83284666
:104E6000524906F004FA0026B34610B9DFF878B1CB
:104E700053267A6B4E4913A806F0C8F94C49059A97
:104E800014A806F0C3F94A49089A16A806F0BEF914
:104E9000524647490EA806F0B9F90DF1400A4449B7
:104EA0009DF834200FA806F0B1F911AF40499DF8E4
:104EB0003520504606F0AAF99DF836203C49384680
:104EC00006F0A4F903250FA93A482D91CDF8B8A012
:104ED0002F97FFF7A5F8FFF707F920462946FFF7B8
:104EE000E9F935483549364A14AB0095FFF7CCFB54
:104EF000009531483349344A16ABFFF7C5FB099C8E
:104F00005CB90A9D002D01F01B818DE800032A4841
:104F10000799049A2DABFFF71DFC069F04242B4A2A
:104F2000194B25482A4901940097FFF7EDFBFFF73D
:104F3000EFF921460398FFF7BDF9264D00242B68B1
:104F4000DA0700F18F8601341035042CF7D1FFF712
:104F5000DFF91948FFF768FB14481F49FFF7DEF92E
:104F6000FFF780FBBBF1000F3FF401AE1B48FFF7DA
:104F70004BF85846FFF748F81948FFF745F8F6E5AB
:104F80000CC600082C0000205C0B00205CCC000844
:104F90006CD000087CD0000844D2000854D200082D
:104FA00064D2000874D2000884D20008C8D0000877
:104FB000DCD200088CD2000878C70008A0D2000814
:104FC00058D20008A8D2000868D2000848D20008C9
:104FD000C0D200083800002070D1000830CD000891
:104FE000D0CE0008340C0020F4CB0008AB4A3CAD16
:104FF00002F108030DF1DC0992E80300039589E84A
:10500000030093E8070085E80700FEF7ABFE0546BE
:10501000A348FEF7C1FF05F10C088246AF680028DF
:1050200000F0E4879F4906F022F90646002800F0C8
:10503000448650469C4906F01AF90646002800F0BE
:10504000F4865046994906F012F90646002800F009
:1050500008875046964906F00AF9002800F0558561
:105060002646B24604F010FC9249024632A806F0E9
:10507000CDF89148FEF7D4FFFFF736F803980321E7
:10508000FFF718F905F13C018C48FFF7B3FA4146E8
:105090008B48FFF7AFFA8B48FFF7DAFA8A48FFF739
:1050A0008FF88A48FEF7B0FF4FF00F08884849464E
:1050B0003A460223FFF760F905F11C0285492023D7
:1050C0008548CDF80080FFF78FF814258348FEF758
:1050D0009BFF8349834A402383480095FFF784F868
:1050E0008248FEF791FF8248FFF7CAF8FFF7C0FA3F
:1050F00004F0ECFB032503467E4972487E4ACDF856
:105100000080FFF7C1FA7D497D4A32AB6D480095BA
:10511000FFF7BAFAFFF7FCF86A48FFF785FA644828
:105120007849FFF7FBF8FFF79DFA002C00F0FF81AC
:105130007548FEF769FF2046FEF766FF7348FEF7E5
:1051400063FF14E5724B0DF1C80893E8030088E88B
:1051500003005348FEF720FF0446002800F0E884CF
:105160006C4906F084F80646002800F04B8620467D
:10517000694906F07CF80646002800F09F86204624
:10518000664906F074F8002840F0D284644D572632
:10519000644B1B68002B00F05C8504F091FA0DF164
:1051A000DC09044662084846424906F02FF8E70742
:1051B00000F1AF86484606F06CF85B4B09EB000245
:1051C00001469C8818689B7949F801009480937186
:1051D000564B1B68002B00F0338504F091FA3CAF6E
:1051E0000446620838463349039706F00FF8E4078F
:1051F00000F19C86039806F04CF8039C4A4B221859
:10520000039F01469C8818689B797850948093711D
:1052100004F046FA0246002840F0718544AF07F8D2
:105220005C0D04F0BDFA0246002840F0608544ACF5
:1052300004F8700D04943E48FEF7F2FEFEF754FFAA
:1052400040460221FFF736F83A484946FFF7D2F9BF
:10525000022439480399FFF7CDF938483849394ACB
:105260003B460094FFF710FA3749384A049B33480D
:105270000094FFF709FAFFF74BF83048FFF7D4F92D
:1052800026483349FFF74AF8FFF7ECF9002D7FF481
:10529000F9AC6CE421460F70FFF7C0BA04C60008F1
:1052A0005CCC000874CD000810CE000820CE0008A9
:1052B00030CE0008DCD2000894CD000838CE0008BB
:1052C00044CE000834C7000858CE0008C4C7000800
:1052D00080CD000860CE00088CCD000868CE0008A4
:1052E0007CCE0008B0C6000854DC0008CCC700081B
:1052F00078CD000880CE000814CE00088CCE0008BF
:1053000024CE0008A0CE0008B0CE0008CCCE000805
:10531000A8C50008ECCE0008FCCE00080CCF0008A1
:10532000ACCB0008DC12002024CF00085004002081
:105330002CCF000844CF000854CF000848CF000805
:105340005CCF0008F0CE000884CF000800CF000832
:10535000ACCF0008AB4B23AC07943CA803F10C0E78
:1053600003F1240503F13004039003F1180693E8D8
:10537000070028AF079B049783E807009EE8070013
:10538000049B2DAF0DF1DC0983E8070096E80700C8
:1053900087E8070095E8070089E8070094E8070018
:1053A000039C84E80700FDF779F90990FDF71CF9E3
:1053B0000546FDF7FDF90A90FDF7B0FC8046FDF7C4
:1053C000A3F9914C0B9014A8FDF760FC236805F03D
:1053D0000102C5F3400A0692002B00F068838B4857
:1053E000FEF7DAFD0446002800F0F885884905F04C
:1053F0003EFF002800F063832046864905F037FF12
:10540000002840F09E858448FEF7E0FD002800F06B
:105410001686012045F002050590CBF8005047267E
:1054200020467E4905F023FF0546002800F05785F9
:1054300020467B4905F01BFF002840F0A085DFF8DF
:105440005CA2DFF85CB2582616AC424675490DF1F5
:105450006008204608941AAD05F0D8FE71499DF801
:105460005020404605F0D2FE1CAC6E499DF85120FC
:10547000284605F0CBFE9DF852202046694905F0EC
:10548000C5FEDBF80020CDF8C88033953494002A9F
:1054900040F01E8544AC04F8982D6348FEF7C0FD2B
:1054A000FEF722FE07980321FEF704FF069D5F48E2
:1054B0005F49604A604B0095FFF710F9099D5B4812
:1054C000009504255D495E4A5E4B0195FFF71CF986
:1054D000059D564800955C494F4A5C4BFFF7FEF826
:1054E0000B9D002D00F0CC840A9D002D00F0DA8485
:1054F00023460224564A57494C480094FFF7C4F803
:10550000FEF706FF4948FFF78FF853485349FEF767
:1055100005FF53485349FEF701FF41485249FEF742
:10552000FDFE52485249FEF7F9FEFFF79BF8BAF12B
:10553000000F3FF41CAB4F48FEF766FD5046FEF7E8
:1055400063FD4D48FEF760FDFFF711BB4B48FEF7CA
:105550005BFDA0461CAD1EAC42464949284605F0FD
:1055600055FE2846FEF750FD4648FEF74DFD4046E5
:1055700021461022FEF7A8F800283DD000270DE0B4
:10558000E25D4149284605F041FE2846FEF73CFD14
:1055900001373E48FEF738FD102F0AD007EB08030D
:1055A000B3F5A27F3A48EBD90137FEF72DFD102F56
:1055B000F4D13648FEF728FD002320212E2003EBEE
:1055C0000802B2F5A27F88BFE15404D8E25C203A19
:1055D0005E2A88BFE0540133102BF0D1002320460F
:1055E0008DF8883008F11008FEF70EFD2948FEF707
:1055F0000BFDB8F5A87FAFD12748FEF705FDFFF7F3
:10560000B6BA00BF0CC60008EC0B00205CCC00084A
:1056100050D000085CD0000860D00008ACD0000872
:10562000BCD00008DCD20008D0D00008C0D00008F0
:10563000E4D0000854D00008ECD000080CD10008D9
:10564000A0D00008240C002084C700081CD100084A
:10565000B0D0000848D100086CCC0008E8CC0008A5
:1056600074CC0008F4CC000860D10008C8D0000851
:1056700070D1000830CD0008D0CE000848CD000819
:1056800050CD000858CD000830DA000894C9000851
:1056900064CD000828C700085CCD0008E0CB0008F6
:1056A00074030020B44D3CAC03940FCD0FC495E8B7
:1056B0000F0084E80F00B148FEF76EFC044630B1DD
:1056C000AF49062205F0EDFD002800F03582DFF835
:1056D00034B30DF1DC09AB48FEF7A2FC23ACFEF7B6
:1056E00003FD03980821FEF7E5FD18AD07941AACF9
:1056F0004FF0000A0695059428AD1EAC0495564659
:105700002DAF0DF1C8081CAD03940BEB0A0CDCF8AF
:10571000042048F68904C8F68804A4FB02029A49CA
:1057200052090598CDF808C005F070FDDDF808C0F5
:105730009549DCF80420A4FB02035B09C3EB0313C7
:10574000A2EB8302284605F061FD9048FEF780FF3A
:1057500032468F49069805F059FD32468D49039827
:1057600005F054FD32468C49079805F04FFD32464E
:105770008A49049805F04AFD32468949384605F0C1
:1057800045FD32468749404605F040FD0698FEF744
:1057900017FD5BF80A2007988349C2F3C012FEF791
:1057A00041FE5BF80A208049C2F380120498FEF79C
:1057B00039FE32467D49484605F028FD5BF80A204F
:1057C0007B48C2F3C204FEF71FFC07232246794937
:1057D0004846FEF7D1FD7848FEF716FC3246774979
:1057E000484605F013FD5BF80A20714802F00704F3
:1057F000FEF70AFC224607236E494846FEF7BCFD29
:105800006D48FEF701FC02246948FEF7FDFB66497E
:10581000059A234638460094FEF7E6FC6648FEF7F4
:10582000F3FB6348FEF7F0FB5F492A4623464046F8
:105830000094FEF7D9FC6048FEF7E6FB01360398BA
:10584000FEF71EFDFEF714FF082E0AF1080A7FF48A
:105850005CAFFEF75DFD0026FFF789B9DFF8A8E130
:105860003CAF3E460EF13C040DF1C8089EE807002F
:1058700088E807000FCC0FC6514D039724682F68A6
:105880000DF1DC090EF1500E9EE80F00346089E83E
:105890000F00002F00F023814A4EFCF751FF07460E
:1058A000FCF786FF05463548FEF776FB04460028E0
:1058B00000F0C283444905F0DAFC8246002800F07B
:1058C000C6822046414905F0D2FC8246002800F0FD
:1058D000758320463E49032205F0E3FC82460028FA
:1058E00000F0728420463B49062205F0DAFC83462C
:1058F000002800F0AF8420463749072205F0D1FC8C
:105900000646002800F09C8420463449042205F015
:10591000C8FC0646002800F056852046304905F0B0
:10592000A6FC0026B24610B9DFF8E0A053262D48A9
:10593000FEF776FB0B24FEF7D7FB40460321FEF76C
:10594000B9FC294829492A4A2A4B01940097022484
:10595000FEF7DAFE2849294A294B2348009501948D
:10596000FEF7D2FEFEF7D4FC03980521FEF7A2FC59
:10597000144D002451E000BF6CC600085CCC000848
:10598000E8D2000800D3000854CC000890C70008F3
:10599000DCD2000814D300081CD3000820D3000870
:1059A00024D3000828D30008B0C60008F8D20008A5
:1059B000C4C7000800000020CCC70008FCD20008C3
:1059C000580B00207C00002088D1000898D10008E6
:1059D000ACD10008B0D10008C8D10008D8D1000867
:1059E000C8D00008E0D1000860C70008F8D100085E
:1059F0008CD10008F00B002004D200089CD10008D4
:105A00001C0C0020342600200CC60008F4CB000833
:105A1000013414350B2C00F0FD802B69D807F7D525
:105A20002246BA4918A805F0F1FB2246B8491AA83F
:105A300005F0ECFB2246B7491CA805F0E7FB22461F
:105A4000B5491EA805F0E2FBAA68B44916A805F0FE
:105A5000DDFBB348FEF7FCFD2868FEF7B1FB16A995
:105A60001AA8B04AFEF7A2FD1CA8FEF787FD2A6916
:105A7000AD49C2F340021EA8FEF7D4FC18A8FEF7F9
:105A8000FFFBFEF7F5FDC3E7A8480599FEF7B2FD59
:105A9000FFF702B82846A64905F0E9FB00283AD1ED
:105AA0000123CBF800305026A24CFEF7D7BFA24B03
:105AB000A24E0FCB86E80F00012323608FE4A0489D
:105AC000FEF784FA002800F05682012345F0010514
:105AD0000693CBF80050CDF814A04726A0E4994ACD
:105AE000994E3B4699591433DC2B42F8041FF9D1E7
:105AF000964B97491A681B6981E80C0001232B60BB
:105B0000CBE606460446FEF7A9BFDFF89CA24E2668
:105B10000446FFF7A7BA28468E4905F0A8FB0028DF
:105B200040F02083CBF8000050268B4CFEF796BF48
:105B300000263546FFF72CBBA01D05F021F80728ED
:105B400004463FF6C4AD01468448FEF74DFA844949
:105B500005F08DFB002800F05D83DFF850B25BF8A4
:105B6000343023F080034BF8343021467D48FEF773
:105B70003BFA7B4905F07BFB002800F044835BF88F
:105B8000343023F040034BF834300DF1DC09224669
:105B90007549484605F03AFB4846FEF7FDF904F022
:105BA000EFFF224671490546484605F02FFB48465F
:105BB000FEF7F2F904F0E4FF5BF83430ED0000F09A
:105BC000070023F03F0340EA030205F038031343C4
:105BD0004BF8343021466648FEF706FA04F0D0FF51
:105BE000214605466348FEF7FFF904F0C9FFC5EBFF
:105BF00005150BEBC40400EB8500606003F01EF894
:105C000069E501F089FA5C4DFEF7E9BF0646834677
:105C1000FFF72FB9FEF77CFB48460421FEF74AFB4D
:105C2000564D00242B68D90700F1C280013410358D
:105C3000022CF7D1FEF76CFB3948FEF7F5FC70E457
:105C40004F4B3CAC93E80300039484E80300FFF758
:105C5000DFBA4B4B0DF1DC0993E8030089E8030040
:105C6000FFF7B6BA2246474918A805F0CFFA2246F0
:105C700045491AA805F0CAFA224644491CA805F06D
:105C8000C5FA55F8082C254912A805F0BFFA404876
:105C9000FEF7DEFC55F80C0CFEF792FA12A93D4A0D
:105CA0001AA8FEF783FC1CA8FEF768FC18A8FEF7EC
:105CB000E7FAFEF7DDFCFFF746B93748FEF76CF967
:105CC00004F05EFF07463548FEF766F98246344821
:105CD000FEF762F90446002F00F0B68105F0D9FA0C
:105CE000092800F2CB812F4CB246FFF7BBB928AC94
:105CF00020460A49049405F089FAFFF79CBA2DAFB3
:105D00003846064905F082FAFFF78BBA14D200082C
:105D1000B8D100081CD20008C0D10008DCD20008AD
:105D200060C7000824D20008B0C60008D0CC000824
:105D30006CCC0008B8CA00089C010020240C00208C
:105D400054D00008EC0B00207C00002070010020E3
:105D50001C0C002074CC0008D0CA0008F0D2000847
:105D60008CC60008F4D20008F8D20008FCD2000863
:105D70009CCC00082CD60008C8CB00087C01002071
:105D8000E8CA0008D0D200087CD20008D8D20008A7
:105D900078C7000844D1000880CD00088CCD0008E9
:105DA00054DC0008F0CA000898CB00083426002014
:105DB0002246BF4923A805F029FA2246BD4928A852
:105DC00005F024FA2246BC492DA805F01FFA55F823
:105DD000082CBA4914A805F019FAB948FEF738FC9E
:105DE00055F80C0CFEF7ECF914A9B64A28A8FEF7F2
:105DF000DDFB2DA8FEF7C2FB23A8FEF741FAFEF754
:105E000037FC13E7B048FEF7C7F804F0B9FE03F01B
:105E10004DFC3546FFF7BCB92DAF3846AB49BDF850
:105E2000322005F0F3F9FEF7F0BEA948FEF7B4F80A
:105E300003F052FD002800F0BB803446DFF8E8A2F2
:105E4000FFF710B901F04CF9A24DFEF7C8BEA24809
:105E5000FEF7A2F804F094FE41260746CBF80000B6
:105E600065E59E48FEF798F804F08AFE03F012FDFF
:105E7000002800F0AD803446DFF8B0A2FFF7F2B89A
:105E80009748FEF7E5FB9748FEF79AF908998D4A7F
:105E90009548FEF78BFB9448FEF7F2F9FEF7E8FB16
:105EA000FFF722BB039DCDF8009001958C48049923
:105EB0003A4632ABFEF74EFCFFF71ABB8B48FEF7B3
:105EC0006BF804F05DFE03F071FC3546FFF760B936
:105ED0001EAC2046794905F099F9FFF7DEBA8448EF
:105EE000FEF75AF804F04CFEDFF844B2AA46CBF8AD
:105EF0000000FFF7A9BA7C480293FEF74DF804F0C2
:105F00003FFECBF80000029B824662269B46FEF7CE
:105F1000B0BF484605F0BDF9764B09EB0002198881
:105F20009B7829F800109370FFF744B9039805F0A7
:105F3000B0F9704B3A1819889B7839529370FFF773
:105F400059B920466C4905F092F9002800F04E81BD
:105F500020466A4905F08BF9002800F0B2812046FE
:105F6000674905F084F9002800F05D81CDF814A0A0
:105F70000026FFF755BA25F001050690A9E5204651
:105F8000604905F074F9002840F00E810123CBF838
:105F900000305026DFF89CA1DFF894B1FFF754BA27
:105FA00026462546FEF71BBE06460546FEF717BEEB
:105FB00006460446DFF880A1FFF754B85248FDF7C3
:105FC000EBFF04F0DDFD46260546CBF80000AEE40D
:105FD00006460446DFF864A1FFF744B8CDF814A0E4
:105FE00006468246DFF848B1FFF72EBA0646044659
:105FF0008246FFF737B845480293FDF7CDFF04F01E
:10600000BFFD8DF834004248FDF7C6FF04F0B8FD2F
:106010008DF835003F48FDF7BFFF04F0B1FD8DF866
:1060200036000D9A6326110CABF800208BF8021095
:10603000029B9B46FEF71DBF0646824677E425F08D
:1060400002050590FFF7E9B93348FDF7E9FF33484A
:10605000FDF7DAFFFEF780F9FEF788FA4FF4FA70E1
:10606000FAF7EEFC2E4B6F6085F83C7050462146E7
:106070001F603E46FDF7A2FEFEF720BC2648FDF756
:10608000CFFF2848FDF7C0FFFEF766F9FEF76EFA6E
:106090004FF4FA70FAF7D4FC214B6E6085F83C603F
:1060A000504621461E60FDF7A1FEFEF707BC00BF6B
:1060B00028D20008D0D1000830D20008DCD2000875
:1060C00060C7000844D10008F0CE00081CC20008D8
:1060D00014CE0008C8CB00088CD1000824CE0008DC
:1060E000C0D0000830D1000898DF000800CF0008B9
:1060F000B0D0000820CF00086CD000087CD0000889
:106100009CD000086CCC00089CD1000888D0000806
:106110008CD0000894D0000894CD0008A8CD0008C9
:10612000F8110020DCCD000810CB000858CB000887
:1061300074030020B8CA000834CB000878CB0008EC
:10614000BF48FEF785FABF48FEF73AF80EA9BE4AE7
:10615000BE48FEF72BFABD48FEF792F8FEF788FA24
:10616000FEF7D3BE2846BA4905F081F80990002809
:1061700000F0C7802846B74905F079F804460028A2
:1061800000F0168100263446FEF768BCB248029340
:10619000FDF702FF04F0F4FCCBF80000029B069030
:1061A00064269B46FEF765BE2046AC4905F05FF8C5
:1061B000002840F02A81CBF800005026DFF8ECA23E
:1061C000DFF8ECB2FFF740B9E01C04F0D9FC0A2874
:1061D00084BF5646B2463FF6AAAB00EB800006EB02
:1061E0008003DA6856469A60FFF7A1BB9748FDF72F
:1061F000D3FE04F0C5FC42268046CBF80000CDF863
:1062000014A0FFF70DB95BF8343043F040034BF8AE
:106210003430BAE4DFF89CB25BF8343043F08003EA
:106220004BF83430A1E48E48FDF7B6FE04F0A8FC2C
:1062300044260990CBF80000CDF814A0FFF7F0B881
:10624000E01D04F09DFC0128044640F24E81B24658
:10625000FFF76DBBA01D04F093FC0A2888BF5E46C3
:10626000824688BFB2463FF662AB7E4952461EACBC
:106270001AA804F0CBFF52467B49204604F0C6FF23
:106280001AA8FDF789FE04F07BFC431E0E2B4FEA93
:106290008A0B9EBF0BEB0A0306EB83039860204634
:1062A000FDF794FE0BEB0A0306EB83031A69002843
:1062B00000F00281002642F002021A61B246FFF7A6
:1062C00036BB6A48FDF768FE04F05AFC8DF85000B2
:1062D0006748FDF761FE04F053FC8DF851006548F6
:1062E000FDF75AFE04F04CFC8DF85200149BCDF8DB
:1062F00014A01A0CABF800308BF802204326FFF7ED
:106300008FB85D48FDF748FE04F03AFC06465B484E
:10631000FDF742FE04F034FC034659480293FDF7B2
:106320003BFE04F02DFC04465648FDF735FE04F014
:1063300027FC0A905448FDF72FFE04F021FC32465A
:106340000B905249089804F061FF029B50491A468D
:10635000504604F05BFF22464D4912A804F056FF58
:106360004B490A9A13A804F051FF49490B9A14A803
:1063700004F04CFF029BA6F26C715A1E0A98CBF8EF
:106380001C10CBF810200B99099ACBF80C40CBF8D5
:106390000800CBF80410CBF80020204632461946FE
:1063A000F9F7A6FF5426CBF81800099CFEF756BB58
:1063B0003848FDF7F1FD1E220146584604F08AFFD9
:1063C0007026FEF74BBB201D04F0DAFB01283FF6D8
:1063D0003EAF314BB24603EB00139A685A60FFF7A9
:1063E000A6BAE81D04F0CCFB032805466BD9B346DA
:1063F000FEF73FBD2948FDF7CFFD04F0C1FBFCF7D8
:1064000045F9B3460890FEF734BD2046244904F010
:106410002EFF244B00280CBF9A464FF0000ADFF8ED
:1064200090B008BF5326FFF70FB81F48FDF7B4FD23
:1064300004F0A6FBFCF71CF9B3460590FEF719BD66
:1064400078C7000830D1000844D1000898DF000860
:1064500080CC0008A8CC000848D2000874CC000802
:10646000A0D00008B8D10008C0D1000888D000082A
:106470008CD0000894D0000890CC000898CC00087C
:10648000A0CC000844DF0008A4CC000850CC0008D1
:1064900054CC0008ACCC00087001002068D2000881
:1064A000C8D00008F4CB000858D20008D0CA0008B1
:1064B000740300203426002022F0020206461A61EE
:1064C0008246FFF734BA024618491AA804F09EFE25
:1064D0001AA8FDF761FD04F053FB0F2887D807EBDE
:1064E00005156860B346FEF7C4BC0246104928A8EB
:1064F00004F08CFE28A8FDF74FFD04F041FB0F28A7
:106500003FF6A5AE0B4BB24603EB04146060FFF7F9
:106510000EBA281D04F034FB03283FF668AF07EBE2
:1065200000139A68B3465A60FEF7A3BC7CD20008F9
:10653000D0D100087001002030B585B04FF4804400
:10654000684603F0E9FE0022200448F2A063C0F28E
:1065500001030121ADF80420ADF8082040F4A84063
:106560004FF480624BF6FF75ADF80650ADF80A2087
:10657000ADF80C40009303F0DDFE200440F4A84089
:10658000694603F059FE05B030BD00BF10B54FF4A9
:10659000A844C4F200042046012103F0E7FE20468F
:1065A000012103F00FFF2046002103F00BFF2046DE
:1065B00003F022FEBDE81040FFF7BEBF70B50546F0
:1065C0000E4643F2010401E0013C13D04FF4A84011
:1065D0002946C4F2000003F003FF0028F4D04FF472
:1065E000A840C4F20000314603F0FAFE0028EBD0C8
:1065F000012070BDFFF7CAFF204670BD38B50546C3
:1066000019B1BDE83840FFF7D9BF43F2010401E0FA
:10661000013C0AD04FF4A840C4F20000294603F020
:10662000DFFE0028F4D0012038BDFFF7AFFF204681
:1066300038BD00BFF8B507464FF4A840C4F20000CB
:106640000E46012115461C4603F082FE0120C1F2D0
:1066500000000021FFF7D2FF002832D04FF4A840FD
:10666000C4F2000034BB012103F08EFE4FF4A844B5
:10667000C4F200042046F9B2002203F099FE022081
:10668000C1F200000021FFF7B9FFB8B18020C1F2CC
:1066900000000021238BFFF7B1FFA8B125B1C6F39D
:1066A0000721204603F07EFE2046F1B203F07AFE79
:1066B0000020F8BD002103F067FED7E76FF001006E
:1066C000F8BD4FF0FF30F8BD6FF00200F8BD00BF1D
:1066D00030B51A4B83B01C680CB103B030BD012536
:1066E00001A81D6003F038FD29464FF4001003F0A7
:1066F0000DFF0820294603F0FBFE0820294603F081
:10670000F7FE29464FF4001003F00EFF21464FF428
:10671000001003F009FFC023ADF804304FF44060CF
:106720001C23C4F2010001A98DF8073003238DF862
:10673000063003F0ADFCFFF7FFFECEE73C0C002077
:106740002DE9F041069D1E466F1E7B427B4180462F
:10675000FFF770FF074610B13846BDE8F081802092
:106760000421C1F20000C1F20001FFF727FF002859
:106770005BD04FF4A844C4F200042046012103F08A
:10678000E7FD0120C1F200003946FFF737FF00287E
:106790004ED020465FFA88F1012203F009FE022064
:1067A000C1F200003946FFF729FF002843D0238BB0
:1067B0008DB33C4611E040200021C1F20000FFF7FC
:1067C0001DFF18B34FF4A840C4F2000003F0ECFD25
:1067D0003219AC4202F8010C1DD00134AC42EAD1AE
:1067E0004FF4A840C4F20000002103F0CDFD4FF4A7
:1067F000A840C4F20000012103F0B8FD40200021B0
:10680000C1F20000FFF7FAFE0028DBD16FF00607A7
:106810003846BDE8F0814FF4A840C4F200000121E1
:1068200003F0B2FD3846BDE8F0816FF0030793E74F
:106830006FF0040790E76FF005078DE770B51C4611
:106840000023FFF7F7FE064608B1304670BD8020F2
:10685000C1F200003146FFF7D1FE28B3049BD3B14B
:10686000049BE51801E0AC4215D04FF4A84014F8A1
:10687000011BC4F2000003F095FD80200421C1F249
:106880000000C1F20001FFF799FE0028EBD16FF084
:106890000306304670BD4FF4A840C4F20000012149
:1068A00003F064FD304670BD6FF00206CDE700BF17
:1068B00070B43A4A3A49546A0B689C4215D8956AB2
:1068C000AB4212D2D56B002D52D01C1B00FA04F43F
:1068D000344D2E6826432E601268032A32D0052AD2
:1068E00015D001330B6070BC7047D46A2B4DA342A6
:1068F000F2D32E6BB342EFD2ED6B002D3ED01C1BBA
:1069000000FA04F4284D2E6826432E60E4E7A3F134
:106910001402032A23D9A3F11804032C34D800FA53
:1069200002F2224C25681543256003F0070201247A
:1069300004FA02F458BB1E48DA08855C25EA040410
:106940008454CEE7102BCCD9142BCAD8A3F1110450
:1069500000FA04F0174A146804431460C1E7A3F175
:10696000080500FA05F5104A14682C431460DCE7AA
:106970000C4C256840EA45052560ADE70A4C2568C2
:1069800040EA45052560A7E72F2BAAD8CDE70848A0
:10699000DA08855C2C438454A3E700BF6C0C00200C
:1069A000540C0020B00C0020CC0C0020C80C00209F
:1069B000440C0020C00C002000B583B001A803F0F7
:1069C000CBFB0820012103F093FD0823ADF8043030
:1069D0004FF4406002238DF80630C4F20100042316
:1069E00001A98DF8073003F053FB03B000BD00BFD1
:1069F000F0B4294A1368002B2BD028490B68022BCE
:106A000017D0032B264B26D0264C0F682168264D25
:106A1000A0F801101E680021A0F803602E6807701E
:106A20001960467121600120296000231360F0BCC9
:106A300070471B4B1D681C68E443E4B2B4EB152F90
:106A40001BD0184C48F2EE752668AE421AD00020D2
:106A5000EBE71846EBE71D681C68E443E4B2B4EBCF
:106A6000152FF4D11C68E4B21C60104C26681D6818
:106A70000C4C45EA06251D60C7E71D68094CEDB2C0
:106A80001D60C2E70B250D601D68C5F30725256055
:106A90001D68EDB21D60B8E7D00C0020680C002026
:106AA000500C0020B80C0020BC0C0020580C00201A
:106AB0002DE9F0474FF440609E4CC4F201000821DC
:106AC00003F052FB236893B99B4E356895B99B4BF5
:106AD000002800F0C2801B68002B40F00C81984B0E
:106AE0004FF6FE711A688A4201D801321A60206896
:106AF000BDE8F087934F3A68002A70D0002800F074
:106B0000B280914A11780131C9B2E929117000F2BD
:106B100006818E4B8E495A6B09688A42E7D1996B80
:106B20000029E4D1DFF868828A49D8F800C00D68EE
:106B3000AC4500F079818848002707601B68012B6D
:106B400000F06581052B00F07A810A2B18BF292BF4
:106B500003D10068C00700F156810120022B20609C
:106B600040F09C81002A40F0028275480368B3F52A
:106B7000E16F80F01682794D794FD5F800903B682F
:106B8000DFF8F4A149F00109C5F80090CAF8003017
:106B9000C1F800C002606546724A02201060724A65
:106BA0003B601360714B1A68714B1D60714B1A602A
:106BB000236863B10B689C4500F0BA816E4A604857
:106BC0001568674FC8F8003000233D6003605B4ADA
:106BD000002313605C4A33600B60137087E7674FD4
:106BE0003B68002B00F08180584B002840F0D28099
:106BF0001A68032A00F05581DFF84C81DFF83C91D8
:106C00005A68D9F8001051488A420BD882689142DC
:106C100008D898F800C0C268944503D30269944527
:106C200040F2B3815B69494A99420BD39369994217
:106C300008D898F80010D369994203D3136A99428F
:106C400040F2A9810025356088F800500123C9F879
:106C50000030002D3FF44BAF5BE71A6801321A6039
:106C60002068BDE8F087DFF8D490DFF8DC80D9F841
:106C70000030A3F11F020A2A17D898F80020052A2D
:106C800013D90A2A11D83E493048442203F0D4FFD0
:106C90002F4A002313600122C9F8002088F8003031
:106CA0003B60002D3FF423AF33E7A3F15E02532A8C
:106CB00008D898F800202D2A00F2A080162A01D9C1
:106CC0003049E1E7A3F13C020F2A40F28A80283BD9
:106CD000162B00F2908098F80030122B40F28B8037
:106CE0001F2B00F288802849CEE7E8B9134B1A68B9
:106CF00001321A600DE7134A012313601F4AFF2176
:106D00001560144A336015601B4A15601F4A1560F0
:106D1000164A15600E4A11600B4A1370E7E60749E0
:106D200033600B601370E2E6074A01233B60137087
:106D3000EFE600BFD00C00204C0C0020C40C00205B
:106D40005C0C0020400C0020600C00206C0C00202B
:106D5000540C0020CC0C0020B40C0020BC0C0020F3
:106D6000B0010020680C0020B80C0020C00C0020EE
:106D7000500C0020580C0020B00C0020640C0020A7
:106D8000E4D30008B0D4000828D40008C80C0020C0
:106D9000AC0100208B49D3F83490D1F800C0E14514
:106DA00000F09080DFF850821A6898F800A0012A5D
:106DB0000AF1010A5FFA8AFA834888F800A000F015
:106DC0009980BAF1E90F7FF644AF09F1FF3294459B
:106DD00000F0C3807D4A00233360136088F80030E0
:106DE00085E698F800203B2A7FF671AF4B2A3FF6E4
:106DF0006EAF774948E70025356049E7592A3FF6E5
:106E000061AF744940E7744800230360D0E602682C
:106E1000013A012A88BF2360F5D9704A7048126888
:106E20000360704B1A60BDE66B480068B0F5966F62
:106E3000BFF481AE6C480768013707607EE60368DF
:106E4000012BE0D001232360684B1F7858789A7893
:106E500087EA000909F00F0989EA171787EA101075
:106E600002F00F09814501D000202060D8781F79F9
:106E70004240587982EA0703984201D000232360F8
:106E80005B4B5C4A1F681068544A38431860544B87
:106E9000052018601268534B1A6083E6052BD3D087
:106EA000BBE748490A68102A7FF4A6AEDFF81C91B8
:106EB000D9F80020053A072A79D94F4B306018706D
:106EC0000546C3E6986B01287FF46CAFDFF8FC90B1
:106ED0005869D9F80010884205D89869814298BF4E
:106EE0009A637FF6B6AE444A00233360C9F8003097
:106EF0001370FCE5BAF10B0F7FF6ABAEBCF10A0FD5
:106F00007FF65FAFDFF8D490C16AD9F80020ACF10A
:106F10000B0A614442EA0A220CF1010C0131C9F862
:106F200000200A22C0F834C0016388F8002065E61A
:106F30002A48324F05683A682748AA427FF442AE91
:106F4000026840F6C90C62459FBF294AD2F800C0CA
:106F50004CF0010CC2F800C034E69B6B002B7FF4B0
:106F600039AFC1F80090002D3FF4C1ADD1E51B4B06
:106F7000224F1B6810E60A200F3A202118601020CB
:106F80000F2AD8621963596305D80120FFF790FCD6
:106F900000233B605AE60020FFF78AFC00233B6099
:106FA00054E6174B154F1A600C4B1B68F4E5124A58
:106FB00012783B2ADFD94B2ADDD800233B6011230E
:106FC0000B6043E6540C00206C0C0020C40C002025
:106FD000F4D400086CD400085C0C0020B00C002035
:106FE000680C0020B80C0020B40C0020440C0020D9
:106FF000BC0C0020C80C0020600C0020B001002058
:10700000D00C0020F9F746B910B582B004460DF156
:107010000600F9F74FF978B1084B09491B88BDF80C
:1070200006200988D21AC2EB0212CB1A92FBF3F3A4
:107030000F2B28BF0F23236002B010BDD40C0020FB
:10704000D60C002008B50F4B1B686BB1FF23C0F2B4
:10705000020398420AD80C4B00221A800B4B40F2D4
:10706000FF321A80012008BD184608BD02220649D9
:10707000E120FCF729FBE32004490222FCF724FB72
:10708000012008BD64040020D40C0020D60C002090
:1070900008B50A4B1B680BB9002008BDE120084960
:1070A0000222FCF72BFB0028F6D00222E320054940
:1070B000FCF724FB003018BF012008BD6404002049
:1070C000D40C0020D60C002040F6D443C2F20003BA
:1070D0001888704740F6D643C2F2000318887047FC
:1070E00010B582B0F9F7D6F80A240DF10600F9F7C9
:1070F000E1F840B90A20F9F7A3FC013CF5D1054CB1
:10710000208802B010BD034CBDF806302380FFF785
:10711000BFFFF5E7D40C002010B582B0F9F7BAF83C
:107120000A240DF10600F9F7C5F840B90A20F9F76D
:1071300087FC013CF5D1054C208802B010BD034C02
:10714000BDF806302380FFF7A3FFF5E7D60C00203B
:10715000F9F730B8F0B507468DB00A20FCF7ACFC63
:10716000092828D00A2813D0072803D00024204655
:107170000DB0F0BDFCF7F6FD0A2201A900F5B670CE
:1071800004F0D6F90146384602F0B8FB7424EEE765
:10719000FCF7E8FD00F14C042021204604F05AF8E9
:1071A000014610B1002301F8013B20463A46FDF7A5
:1071B00009FB0446DBE7FCF7D5FD01AE00F5A6743C
:1071C000002502E002340A2D12D023782046022145
:1071D000002B7BD06378002B78D0F9F7C3F8A37825
:1071E0000135202B46F8040FECD103340A2DECD1E5
:1071F000029CA4F141032F2BB8D801A252F823F02E
:10720000C1720008C17200081B730008C172000837
:107210006D710008C1720008C17200086D7100082C
:107220006D7100086D7100086D710008C172000871
:107230006D710008D57200086D710008C1720008F8
:107240006D7100086D710008D5720008F5720008B4
:107250006D7100086D710008D57200086D7100082D
:107260006D7100086D7100086D7100086D71000886
:107270006D7100086D7100086D7100086D71000876
:107280006D710008C17200081B730008C17200080C
:107290006D7100086D7100086D7100086D71000856
:1072A0006D7100086D7100086D7100086D71000846
:1072B0006D7100086D7100086D710008DD720008C5
:1072C000022D7FF453AF039B3B6050E7002D3FF44A
:1072D0004DAF8DE7012D7FF449AF48E720233846B5
:1072E00000F8013B0DF109011E2203F0F3FF00231A
:1072F000FB773CE7072D7FF439AF039B03F1640272
:10730000049B7A61013B3B61059BFB60069BBB6074
:10731000079B7B60089B3B6029E7042D7FF426AF29
:10732000039B3B70049B7B70059BBB701FE700BFFA
:1073300030B53B4B87B01A68044682426DD0684630
:107340001C6002F009FF02A803F07EFA042001216C
:1073500003F0CEF80420012103F0CAF84FF4804076
:10736000012103F0C5F84FF400734FF400600325CA
:10737000C4F201006946ADF8003018238DF80330DF
:107380008DF8025002F084FE4FF480634FF40060E9
:10739000C4F201006946ADF8003048238DF803308F
:1073A0008DF8025002F074FE4FF46050C4F20100F8
:1073B000012103F087FA00234FF460501D46C4F208
:1073C000010002A9ADF80C30ADF80E30ADF8103068
:1073D000ADF814300C23ADF81230029403F0CEF95E
:1073E0004FF46050C4F20100012103F039FA4FF468
:1073F0006050C4F2010040F22551012203F03EFA30
:1074000025238DF8043001A801238DF805508DF84F
:1074100006508DF8073002F045FC07B030BD00BFC4
:10742000D80C002030B40F4A13687F2BFCD80E49CB
:107430000E4D0B685C1C7F2C45F8230098BF0C6038
:1074400001D900230B6072B613680133136062B672
:107450004FF46050C4F2010040F22771012230BCA9
:1074600003F00CBAE80E0020EC0E0020E00C002027
:1074700010B50446007828B1FFF7D4FF14F8010FC7
:107480000028F9D110BD00BF30B40D4B1A6882B18D
:107490000C490D4D0A68541C802C55F8225018BF19
:1074A0000C6009D072B61A68013A1A6062B60122FD
:1074B0000560104630BC704700220A60F2E700BF4A
:1074C000DC0C0020E00E0020F00E0020024A1368C1
:1074D000002BFCD1704700BFE80E00204FF4605035
:1074E00038B5C4F2010040F2255103F0F9F9002843
:1074F0002BD14FF46050C4F2010040F2277103F029
:10750000EFF900B938BD4FF46050C4F2010040F209
:10751000277103F00BFA234B1A68002A38D0224A4D
:10752000224C1168481C802808BF002054F8211004
:1075300010601A684FF46050013AC4F2010089B239
:107540001A60BDE8384003F0B5B94FF46050C4F29A
:10755000010040F2255103F0E9F94FF46050C4F204
:10756000010003F0ABF9124B1A687F2AC1D8114908
:10757000114D0A68C0B2541C7F2C45F8220098BFF8
:107580000C6001D900220A601A6801321A60B0E763
:107590004FF46050C4F2010040F22771BDE838405A
:1075A00003F06CB9E80E0020F0100020E00C002081
:1075B000DC0C0020E40E0020F00E002010B541F29B
:1075C000F404C2F2000402460B4620464FF48071D8
:1075D00004F0D8FA2046BDE81040FFF749BF00BFCD
:1075E0000FB400B583B004AB53F8040B19460193F4
:1075F000FFF7E4FF03B05DF804EB04B0704700BF91
:10760000FFF796BE10B584B001A803F057F801202B
:10761000014602F07BFF0023ADF80A30ADF80630DA
:10762000052301A9ADF808304FF0804040F21F3328
:10763000ADF8043002F086FF01210A464FF0804089
:1076400003F06EF801240F2368461C228DF80020F9
:107650008DF803408DF801308DF8023002F022FBE6
:107660004FF08040214603F03DF804B010BD00BF4C
:1076700038B54FF08040012103F07CF86A4B1C685C
:10768000002C34D0694B43F698211A6801328A42A3
:107690001A6000D038BD664A0120664910600C6847
:1076A000654A24180C6014680021241814601468BA
:1076B00019603C2CEED1614B11601A6812181A60E7
:1076C0005F4A10601A683C2AE4D15E4A1960136868
:1076D0001B1813601368182BDCD15B4B11601A6800
:1076E00012181A601A68072AD4D1196038BDFFF73A
:1076F000DFF950490B68012B07D9544B40F6A660BF
:107700001A68013282421A6043D0514B1A68013222
:10771000EA2A1A6054D04F4B1A680132962A1A602E
:1077200048D04D4B1A680132962A1A603CD04B4B18
:107730001A6801320F2A1A6030D03C4B43F6982069
:107740001A68013282421A60A4D1394A01201060BD
:107750000C68394A24180C6011680024091811605B
:1077600011681C602D2931D01268334B3C2A38D067
:107770001B681E2B53D03A4B1A68002A8AD01A680D
:10778000013A1A601B68002B84D1364B01221A6023
:1077900080E7354A012010601C60B6E7334A0120BB
:1077A000106000221A60C8E7314A012010600022F0
:1077B0001A60BCE72F4A0120106000221A60B0E76F
:1077C0002D4A0120106000221A60A4E72B4B1B49B0
:1077D0001C680D68AC421FBF09681960284B18600F
:1077E000C2E7164A002119601368012001331360B3
:1077F000134B186013683C2BBDD1124B11601A68F3
:1078000012181A601A68182AB5D10F4A196013683D
:107810001B1813601368072B08BF1160ABE7194BE7
:1078200001221A60A7E700BF4412002008120020BE
:10783000FC1100204C1200200C12002054120020D9
:107840001012002030120020001200202812002008
:10785000341200202C1200202012002038120020A8
:10786000B4010020F41100203C1200200826002062
:107870000C2600202412002050120020B801002005
:1078800018120020141200204DF23850C0F60000EB
:10789000704700BF40F2BC13C2F200031868704783
:1078A00041F2302141F2542241F20C23C2F2000194
:1078B000C2F20002C2F20003096842F210601268CC
:1078C0001B68C2F20000816042600360704700BF25
:1078D0002DE9F04F9DB003F08DF803F019F9012068
:1078E000014602F005FE4FF400700121C0F23000A5
:1078F00002F046FC4FF4E130FFF782FEFFF75CF840
:1079000001F044FB01F06AFBFFF77CFE0120F9F770
:10791000BBF8F8F765FDF8F781FD01F01FFDFBF7F7
:10792000ABFEF8F793FD002841F0E380C148FFF774
:107930009FFDC148FFF79CFDC048FFF799FDBE4879
:10794000FFF796FDBE48FFF793FDBE48FFF790FD99
:10795000B948FFF78DFD41F2DC20C2F20000036858
:10796000002B01F06C80B848FFF782FDB248FFF7AA
:107970007FFDB64DFBF798FD2B68002B01F056807C
:10798000B348FFF775FDAC48FFF772FD2B68002B7D
:1079900041F08C80AF4CB0482168FFF721FE22688F
:1079A00022F47F0323F47F43EBB940F2FF43C0F29C
:1079B00001039A4201F2BB8040F2FF632268C0F2E9
:1079C00001039A4201F2A980A448FFF751FD9A48A9
:1079D000FFF74EFD206801F0A9FE206801F026FEA9
:1079E0002068FFF72FFBFFF7B3FBF8F76FFD01F0FF
:1079F0008BF941F24421C2F2000101230B6001F036
:107A0000DFFE41F24422C2F2000200261660FAF7BD
:107A100003FDFAF743FE41F20423C2F200031860AB
:107A2000FAF78EFE41F24029C2F20009C9F80000BF
:107A3000FAF7BEFE41F21C2CC2F2000CCCF800009A
:107A4000FAF762FE41F2482E2B68C2F2000ECEF821
:107A5000000083B34FF480752368C0F20205AB4287
:107A60007C4F28D07E482946FFF7BAFD774B3D6012
:107A70001B68002B41F08E807A48FFF7F9FC6E48B6
:107A8000FFF7F6FC01F020FC002801F07B80FBF7FB
:107A9000DBFB002801F06E8001F0C8FE002801F039
:107AA000618001F0CBF8002801F02F804FF4807343
:107AB000C0F20203236041F218210120C2F200014A
:107AC00041F24C220860C2F20002146801460246EC
:107AD0000334FAF79FFC41F24C25C2F200052B68F3
:107AE00009A89C421ED9FEF783FF0028F3D000218D
:107AF0000A460120FAF78EFC0120F8F7AFFF09A82B
:107B0000FEF776FF002001460246FAF783FC56484E
:107B1000FFF7AEFC4848FFF7ABFC01F0DDFA08B117
:107B200001F0D2FB0020014602468346FAF772FCC0
:107B3000FCF7E4F9FCF716F94FF0010900F13C0CF1
:107B4000DFF82C81494F8246CDF818B004255C46F9
:107B5000CDF81490CDF81CC0CDF810B013A8FFF7E5
:107B6000F9FA8146002840F0E781D8F8003043B1A7
:107B700041F2482EC2F2000EDEF80030002B40F039
:107B80000881BBF1000F40F02881DAF80030002BAB
:107B900040F015863548F8F767FC002840F04C8126
:107BA00041F21820C2F20000036873B141F2DC21F7
:107BB000C2F200010B68002B40F00B8641F2182C3A
:107BC0000023C2F2000CCCF80030D8F8003073B1BA
:107BD00041F2482EC2F2000EDEF800303BB141F215
:107BE0003C20C2F200000368002B40F0B88641F24E
:107BF000F411C2F200010B688BB1DAF80430002BEB
:107C000040F02D8641F2F4120023C2F2000240F24D
:107C1000B4161360C2F2000640F6D863336041F236
:107C20001029C2F20009D9F80030002B40F05D8520
:107C300020E000BF40D5000828C7000860D5000834
:107C400080D5000838D500088CD5000864040020D1
:107C5000ACD50008BC010020C0D5000878D60008CB
:107C6000B4D60008D8D6000898D7000810260020FF
:107C70009425002041F2142EC2F2000EDEF80030EE
:107C8000002B00F0398340F27439C2F200098F4AA8
:107C9000D9F8003000211160002B00F02D8341F253
:107CA000542CC2F2000CDCF80020B2FBF3F103FB11
:107CB0001123002B40F0208340F2504EC2F2000E00
:107CC000DEF80030002B40F05D8541F2DC2CC2F282
:107CD000000CDCF80030002B00F04C8501F0F0FCCB
:107CE0007B4B7C4A064610F0010F4FEA56017A485A
:107CF00018BF1A46FFF774FCFF2E0AD03046FBF778
:107D0000C9F841F24C2EC2F2000EDEF80030063304
:107D10000693002D40F0048341F2502EC2F2000E73
:107D2000DEF80030002B40F0198341F2FC12C2F261
:107D300000021368002B40F0238341F22425C2F295
:107D400000052B68002B40F02D8301F07FF9FF2800
:107D5000054600F03283002101200A46FAF75AFB5B
:107D6000132D00F27486DFE815F0C701BA01A801EF
:107D7000430218020602E10193025602AE025A01C2
:107D80008E018101740167019B014501300172067A
:107D9000C70008A8FFF738F900283FF4F2AE40F218
:107DA000C010089AC2F200000168531C8B4203D332
:107DB0004B1C9A427FF6E5AE4848FFF711FC089B42
:107DC00040F2C011C2F20001184602250B60FAF71A
:107DD000ABFFBBF1000F3FF4D8AE41F2F812C2F294
:107DE000000213684FF0010B002B7FF4D3AEDAF8DA
:107DF00004304FF0010B002B3FF4CCAE384B394828
:107E0000C3F800B0FFF734FB3748FFF731FB3749C1
:107E1000079A0BA803F0FAF90BA8FAF7E7FF41F26B
:107E2000F413C2F2000332480425C3F800B0F8F797
:107E30001BFB00283FF4B4AE012041F2DC240146D4
:107E40000022C2F20004FAF7E5FA2368002B40F0A2
:107E5000218541F23026C2F200063368BC68244A0C
:107E60009C4200F06F85D2F804E00425D7F8189002
:107E700040F2000CC2F2000C5CF829103E68F86871
:107E800041F2002CC2F2000C7A693B698DE8114086
:107E90000396CCF8009041F2302941F2542CC2F202
:107EA000000CC2F20009C9F80040CCF800E041F231
:107EB0000C2EC2F2000E0F4802F26C720133CEF8A3
:107EC0000060FFF78DFB32246AE600BF1412002029
:107ED00020CF0008B0C60008F8DB000800DB00086F
:107EE000F81100203CDB000828C7000850DB000820
:107EF0001026002058DB0008AC48FFF7B9FAAC4860
:107F0000FFF7B6FA0126322404960025059E1BEAE7
:107F1000060F52D1002C3FF421AE013C7FF41EAE7F
:107F2000204621462246FAF775FA13A8FFF712F900
:107F3000814600283FF419AE002101200A46A9F12C
:107F40004109FAF767FAB9F1330F00F24482DFE82A
:107F500019F0AB03980393037D03420268035D03AA
:107F600042023702420242023B034202CF02420275
:107F7000B60242024202AB024E0242024202300309
:107F800025034202420242024202420242024202ED
:107F9000420242021A030B03A002420242024202C0
:107FA00042024202420242024202420242024202B1
:107FB00095024202420242024502F8F747FA0028BF
:107FC00040F0A68401260596A4E77A48FFF750FA08
:107FD0007748FFF74DFA41F24826C2F200063368AF
:107FE000002B40F0EA840025FAF7B4FE3224049511
:107FF00002258BE77048FFF73BFA6D48FFF738FA28
:1080000041F24826C2F200063368002B40F0C684D5
:108010000025FAF795FE32240495022576E7674895
:10802000FFF726FA6248FFF723FA0025FAF7DEFD8C
:1080300032240495022569E76148FFF719FA5C4884
:10804000FFF716FA0025FAF711FE322404950225EF
:108050005CE75C48FFF70CFA5548FFF709FA002681
:10806000FAF7D4FD3224049602254FE75648FFF76D
:10807000FFF94F48FFF7FCF90025FAF7D7FD322446
:108080000495022542E75148FFF7F2F94848FFF707
:10809000EFF90026FAF79AFD32240496022535E717
:1080A0004B48FFF7E5F94248FFF7E2F90026FAF7F7
:1080B000CDFD32240496022528E74648FFF7D8F97B
:1080C0003B48FFF7D5F9FAF70FFB41F20425C2F25E
:1080D00000050026286032240496042516E73E4851
:1080E000FFF7C6F93248FFF7C3F900240494FBF701
:1080F000ABF83224049D09E73848FFF7B9F92C485A
:10810000FFF7B6F940F2601CC2F2000CDCF8005038
:108110003224D5F1010538BF00250026CCF80050E7
:108120000496B5420CBF14250C25EFE62C48FFF74A
:108130009FF91F48FFF79CF941F23026C2F2000672
:108140003268284B002A00F011841A68013A1A603C
:1081500041F20C290023C2F20009C9F8003041F2B3
:10816000DC29C2F20009D9F80060002E73D1322454
:1081700004960425CAE61C48FFF77AF90C48FFF775
:1081800077F9FAF7EBFA41F240260025C2F2000631
:108190000495322430600425B8E61448FFF768F9E6
:1081A0000348FFF765F9FAF7E5FAECE748DE00085F
:1081B00028C700082CDE000810DE000848DD000893
:1081C000D0DD0008ACDD000888DD000868DD0008AF
:1081D000F0DD000868DC000858DC000848DC000816
:1081E000E8DC000830120020C8DC0008A8DC000829
:1081F000C748FFF73DF9C748FFF73AF9FAF762FABF
:1082000041F204290025C2F2000904953224C9F87C
:10821000000004257AE6C048FFF72AF9BD48FFF7B9
:1082200027F941F25420C2F200000268BB4B002A39
:1082300000F0A0831A68013A1A6041F2DC29C2F208
:10824000000941F20C21D9F800600023C2F20001BC
:108250000B60002E8BD041F2302941F2542C41F2B8
:108260000C2EC2F2000CC2F2000EC2F20009D9F8C4
:108270000010DCF80020DEF800300025A848B960C6
:108280007A603B60322401F0C5F8049504253DE690
:10829000A448FFF7EDF89F48FFF7EAF841F2302CC9
:1082A000C2F2000CDCF800209F4B162A00F2688313
:1082B0001A6801321A6041F20C2E0023C2F2000E3D
:1082C000CEF800304BE79948FFF7D2F89148FFF716
:1082D000CFF841F25423C2F200031A688F4B3A2AB6
:1082E00000F24B831A6801321A6041F20C24002319
:1082F000C2F20004236032E7049E002E7FF4DCAC5F
:10830000069E002E3FF405AD41F24C29C2F2000951
:10831000D9F80030B342FFF4FCAC049E0425069665
:108320008348FFF7A5F87B48FFF7A2F841F2302910
:1083300041F2542CC2F2000CC2F20009D9F800003C
:108340002A46DCF80010FAF779F841F2502EC2F212
:10835000000EDEF80030002B3FF4E7AC40F2601175
:10836000744BC2F20001002208681A60FAF7F6FAAC
:1083700041F2FC12C2F200021368002B3FF4DDACA4
:108380006D4B00221A6041F20C23C2F2000341F24D
:1083900024251868C2F20005FAF722FA2B68002B90
:1083A0003FF4D3AC654B00221A60F8F7C5F800F033
:1083B0004DFEFF2805467FF4CEAC00250495A5E5CB
:1083C0005F48FFF755F85348FFF752F800F084FE76
:1083D000002840F085813224FFF7C7BB139B40F291
:1083E000B412C3F56E630233C2F20002136041F2AD
:1083F000DC24C2F200042368002B40F0ED8241F23D
:108400003026C2F200063368DDF854E09E4500F0E5
:10841000E782DDF850C00425199C139E169B40F29C
:10842000000041F20029C2F20000C2F2000950F837
:108430002410CDF804E00093CDF808C00396C9F8E5
:10844000004041F23029C2F20009C9F800E0189A50
:10845000179B41F2542E41F20C29C2F2000EC2F2D7
:108460000009CEF800C0374802F26C720133C9F837
:1084700000603224FFF7B4F8FFF777BB13A8FAF7D0
:10848000B5FC314813A9FFF7ABF804253224FFF7F8
:108490006CBB1398FAF7D2F801462C48FFF7A0F806
:1084A00004253224FFF761BBFAF7CEFE2848FEF719
:1084B000DFFF1848FEF7DCFF3224FFF756BB40F21F
:1084C000601EC2F2000E139BDEF80020934282D0A1
:1084D000204A2149002B08BF1146204A204814BFDA
:1084E0000C25142513603224FFF77AF8FFF73DBB03
:1084F00041F2F41C0123C2F2000C1A48CCF80030FF
:10850000FEF7B6FF0348FEF7B3FF3224FFF72DBB9B
:1085100088DC000828C7000818DD00085412002075
:108520001026002000DD00083012002030DD000899
:1085300038DC000850120020FC110020241200201A
:10854000ACDA000854DA0008E4DA00089CD8000825
:10855000C4DA000898DE000884DE0008600100200C
:1085600060D800088CDA000813A8FAF7BFFBCC48E3
:108570009DF84C109DF84D209DF84E30FFF730F8D7
:108580003224FFF7F2BA1398FAF7F6FBC5481399AD
:10859000FFF726F802253224FFF7E7BAC248FEF7B4
:1085A00067FFC248FEF764FF3224FAF7F1FBFFF7DA
:1085B000DCBABF48FEF75CFF0124BC48FEF758FF59
:1085C00004943224FFF7D1BA139B002B00F01482DD
:1085D00041F24829B7480123C2F20009C9F8003026
:1085E000FEF746FFB148FEF743FF41F2482EC2F2C4
:1085F000000E40F2C011FF23C2F20001DEF80000BD
:108600000B603224FAF786F8FFF7AFBA1398F9F740
:10861000F1FFA9481399FEF7E3FF04253224FFF781
:10862000A4BA41F21C26C2F200061398336898429D
:108630003FF4D1AEFAF7C2F8A04A03460146A0487B
:1086400013603224FEF7CCFFFFF78FBA41F204210A
:10865000C2F2000113980B6898423FF4BCAEFAF7DF
:1086600023F8984A03460146974813600425FEF70D
:10867000B7FF3224FFF779BA13A8FAF713FB934830
:1086800076E741F24825C2F200052B68002B40F046
:10869000C0811398FAF748FB8D481399FEF7A0FFA5
:1086A00002253224FFF761BA41F24022C2F20002F1
:1086B0001398136898423FF48EAEFAF747F8854A4C
:1086C000034641F2502419461360C2F2000400230D
:1086D000814823600425FEF783FF3224FFF745BA63
:1086E00000F0F2FD3224FFF740BA7C4B002241F249
:1086F000002C41F2302E1A60C2F2000CC2F2000EC1
:1087000041F25420DCF80010C2F20000DEF8003024
:1087100040F260150268C2F20005C3EB031328683B
:1087200002EB83026E4D00F0B5FA002800F0A18044
:108730002B68DFF8D8C1D3F1010E38BF4FF0000E1F
:1087400041F2302641F254296649BEF1000FC2F2CF
:108750000006C2F2000932686348D9F8003008BF49
:108760006146C5F800E00CBF14250C25FEF738FF64
:10877000FFF780BA5D48FEF77BFE4C48FEF778FEB7
:10878000FFF7C7BA41F244200123C2F200000360A0
:1087900000F0B6FF564B574A10F0010F064641F263
:1087A000442918BF1A46C2F20009002352484FEA72
:1087B0005601C9F80030FEF713FFFFF79DBA4F4886
:1087C000FEF756FE3948FEF753FE4FF0010BFFF758
:1087D000E1B9DFF83491484600F0B0FE00283FF4DC
:1087E000EDA941F23022C2F200021368D9F808E084
:1087F0009E4500F0C880D9F804C00425BE69F86819
:1088000040F20009C2F2000959F826107A693B6962
:108810008DE80140CDF808C0386841F20029C2F265
:1088200000090390C9F8006041F2302641F2542952
:10883000C2F20006C2F20009C6F800E0C9F800C0A2
:108840003E6841F20C29C2F200092D4802F26C7216
:108850000133C9F80060FEF7C3FEFFF7AFB900208F
:1088600001460122F9F7D6FD322401F041F8FFF765
:10887000C9B9244B4CF6CD451B68CCF6CC45A5FBBD
:1088800003C5AD0805EB8505AB420CBF04250125EA
:10889000FFF7F0B91C4800F0BDFDFFF7DABA00BFE2
:1088A00034D8000884D9000838DA000828C700083E
:1088B00010D90008B0D9000810DA00081C120020F6
:1088C000E4D800080412002078D8000808D800086E
:1088D0002CD9000840120020C0D800081012002037
:1088E0006001002084DE0008B0DB00081CDC00080A
:1088F00020CF0008B0C60008D0DB00082CDB000841
:1089000084DB0008541200201026002098DE0008A6
:10891000A548FEF7ADFDA548FEF7AAFD4FF00009FA
:1089200041F2F81CC2F2000CCAF804908AF83C909C
:108930009F49A048CCF80090CDF81490FBF756FA68
:10894000FFF7E8BA41F25429C2F20009D9F8003021
:10895000D2F804E09E457FF488AAFFF787BAFEF7B5
:1089600051FB954B00221A60FFF741B917221A609C
:10897000FFF7EEBB3B221A605FE400221A60B4E40A
:1089800000221A6097E441F25426C2F200063368CE
:10899000D9F804C09C457FF430AF2FE7874A002305
:1089A00040F2C01918461360C2F20009FF23C9F84B
:1089B0000030F9F7AFFEFFF72BBB804A002340F2EF
:1089C000C01918461360C2F20009FF23C9F800302D
:1089D000F9F7A0FEFFF707BB13A800F01BFD0EE59B
:1089E00041F25429C2F20009D9F80030DDF850C034
:1089F0009C457FF410AD0FE541F2482CC2F2000C0B
:108A00006F48CCF80030FEF733FD6848FEF730FDC4
:108A1000EBE56A4A002340F2C01618461360C2F222
:108A20000006FF233360F9F775FE32E66548FEF76E
:108A30001FFD5E48FEF71CFD634CFEF7D4BF634884
:108A4000FEF716FD5948FEF713FDFEF792BF132DF2
:108A500055D80FF2080959F825F000BF0581000824
:108A6000EB800008C7800008FD810008A78100088E
:108A700083810008398100089D8200082382000854
:108A8000D38200082B8000089380000879800008BA
:108A90005F80000845800008AD8000080180000864
:108AA000D77F0008BB8A0008057F000800204649E0
:108AB0000422FAF709FEFEF76DBF41F24829C2F21F
:108AC0000009D9F8003040F2C01CD3F1010338BFCF
:108AD00000231846C9F80030C2F2000CFF2300251D
:108AE000CCF800303224F9F715FE04950225FFF783
:108AF0000DBAF7F761FCFBF7ABF9FEF717BF0026DD
:108B0000049632243546FFF701BA3148FEF7B0FC2F
:108B10002648FEF7ADFCFEF7C9BF2E48FEF7A8FCBD
:108B20002248FEF7A5FC00F063F8FEF74DBF2A4887
:108B3000FEF79EFC1D48FEF79BFC00F09BFB2748C0
:108B4000FEF796FC1948FEF793FC2068FAF7E2F965
:108B50002348FEF78DFC1548FEF78AFC00F034FE32
:108B6000FEF72ABF1F48FEF783FC1048FEF780FC83
:108B7000FEF797BF1C48FEF77BFC0C48FEF778FC1D
:108B8000FEF78ABF1948FEF773FC0848FEF770FC31
:108B9000FEF77DBF304639460422FAF7AFFD0028C4
:108BA0007EF470AFFEF768BFB4D7000828C700088E
:108BB000FCD70008F0D700083C1200204812002023
:108BC000E0D90008A0D60008BC0100209CD5000810
:108BD0006CD7000854D60008E4D5000804D6000875
:108BE00030D6000840D7000820D70008FCD600087F
:108BF00030B5104B87B01B6813B9002007B030BDEB
:108C0000BF2069461822FAF75FFD0028F5D00A4810
:108C10006A4600231478517895781C50C1EB0111F5
:108C20001C18083305EB81010332402B6160F1D140
:108C30000120E3E76404002034260020F0B548F664
:108C4000890787B0114C6A460023C8F688071919AE
:108C500048681D59A7FB00614909C1EB0116A0EB4B
:108C6000860008331570517090700332402BEED19E
:108C7000074B186838B1BF2018226946FAF73EFD45
:108C8000003018BF012007B0F0BD00BF342600201F
:108C900064040020F0B400231A4D02E00833402B96
:108CA00021D05C595E1914F0800FF7D07668964297
:108CB000F4D1C4F3C20604F0070704F0400418B16D
:108CC000D4F1010438BF0024002CE7D0BE420DD8F7
:108CD000B14234BF00260126B94288BF0026002ECB
:108CE000DCD0012000E00020F0BC7047B9428CBF0E
:108CF00000270127B14234BF3E4647F00106002E4F
:108D0000CCD0EEE734260020704700BF70B5642059
:108D1000F7F782FE4FF4406020210022C4F20100E8
:108D200001F028FA4FF40C70F7F776FE4FF440602C
:108D3000C4F201002021012201F01CFA274D142069
:108D4000F7F76AFE00264FF496732B60344603E073
:108D500004B92C682B68ABB14FF440602021C4F2F9
:108D6000010001F001FAD6F1010338BF0023002C05
:108D700008BF00230028EBD0002BEBD02E682B6817
:108D8000002BE9D13220002E18BF002C0CBF00258B
:108D9000012515D0F7F740FE4FF440602021C4F2C2
:108DA000010001F0E1F905467820F7F735FE6B1E6A
:108DB0005842C6EB040458411E2C98BF002070BDD9
:108DC000F7F72AFE4FF440602021C4F2010001F0C1
:108DD000CBF97820F7F720FE284670BD90250020BB
:108DE00010B54FF44064C4F2010420210022204653
:108DF00001F0C0F90520F7F70FFE012220212046DF
:108E000001F0B8F90A20F7F707FE2021204601F00B
:108E1000ABF904463220F7F7FFFD621E5042504185
:108E200010BD00BF70B5082401250026FFF7D8FF4C
:108E30006B0000B12E43013CDDB2F7D1304670BD6E
:108E400038B54D1E0446EDB239B101354519FFF76D
:108E5000E9FF04F8010BAC42F9D138BD70B5064604
:108E60000825012418E04FF440600022C4F20100FC
:108E700001F080F90520F7F7CFFD4FF44060202185
:108E80000122C4F2010001F075F950206400F7F7E7
:108E9000C3FD013DE4B21BD04FF44060202114EA31
:108EA0000602C4F20100DED101F064F95020F7F7A8
:108EB000B3FD4FF4406020210122C4F2010001F013
:108EC00059F905206400F7F7A7FD013DE4B2E3D1AD
:108ED00070BD00BF38B54D1E0446EDB239B1013545
:108EE000451914F8010BFFF7B9FFAC42F9D138BDB1
:108EF00010B50446FFF70AFF80B9234603F8010BBB
:108F00000133607003F8010B03F8010B03F8010B48
:108F100003F8010B03F8010B187010BD3320FFF7A5
:108F20009DFF20460821FFF78BFFFFF7EFFE012092
:108F300010BD00BF30B5144B83B01A680AB103B03E
:108F400030BD012401A81C6001F006F92020214653
:108F500001F0CEFA14234FF44060202501A98DF8CA
:108F60000730C4F201000323ADF804508DF8063039
:108F700001F08EF84FF44060C4F201002946224609
:108F800001F0F8F8DBE700BF5812002000B583B00D
:108F900001A801F0E1F80820012101F0A9FA01235C
:108FA000ADF804304FF44060022301A98DF806307B
:108FB000C4F2010010238DF8073001F069F84DF676
:108FC0006060C0F60000FEF753FA4CF22870C0F65D
:108FD0000000FEF74DFA03B000BD00BF10B50A4C0B
:108FE0002368012B0FD001214FF440600A46C4F2E0
:108FF000010001F0BFF80548FEF73AFA0448FEF711
:1090000037FA0123236010BDC401002074DE00087C
:1090100028C7000810B50A4C23687BB14FF44060A4
:1090200001210022C4F2010001F0A4F80548FEF776
:109030001FFA0548FEF71CFA0023236010BD00BF8D
:10904000C401002088DE000828C70008F0B583B0FE
:109050006846FDF7CDFC68B31C4B1D4A18681168C3
:1090600001301860002928D09DF8050000F00100AB
:1090700018490023BDF80170BDF803C09DF80040F9
:1090800010600E46184602E00130782B12D0CA5C00
:109090000633A242F8D100EB400206EB4202B2F8DE
:1090A0000150BD42F0D1B2F80320624503D0013037
:1090B000782BECD1FF2003B0F0BD9DF8053013F004
:1090C0000100D5D001231360F4E700BF5C1200203B
:1090D00060120020641200202DE9F04FDFF890812B
:1090E00000274D4D83B001263C46C2462846F9F77D
:1090F0007DFE2846FEF7BCF94848FEF7B9F96846F8
:10910000FDF776FC04EB440908EB49090AEB070577
:109110004846FDF76DFC0028FAD06A7912F001028A
:10912000F6D1C4B399F80010134602E00133A3420C
:109130002FD018F8020006328842F7D103EB430C17
:109140000AEB4C0CB9F80100BCF801E08645EDD102
:10915000B9F803E0BCF803C0F445E7D1FF2B18D001
:109160000022134602E00133A342D1D018F802C016
:1091700006328C45F7D103EB430C0AEB4C0CBCF8E0
:1091800001B08345EFD1BCF803C0F445EBD1002B0F
:10919000BED1142E37D0731E122B3BD8DFE803F05C
:1091A0002F2D2B29272523211F1D1B1917151311BF
:1091B0000F0A31001A4D01340136063796E7194D72
:1091C000F9E7194DF7E7194DF5E7194DF3E7194D93
:1091D000F1E7194DEFE7194DEDE7194DEBE7194DA3
:1091E000E9E7194DE7E7194DE5E7194DE3E7194DB3
:1091F000E1E7194DDFE7194DDDE7194DDBE7194DC3
:10920000D9E7194DD7E71948F9F7F0FD012003B068
:10921000BDE8F08F004DCEE7B0DE000828C700089B
:1092200078E0000858E0000838E000081CE000087A
:1092300000E00008E0DF0008C0DF0008A4DF00084D
:1092400088DF000874DF000860DF00084CDF0008DA
:1092500038DF00081CDF000800DF0008E4DE00083B
:10926000C8DE0008C0DE00089CDE000894E00008AC
:1092700064120020F0B5124B83B01868E8B10025E5
:10928000104F04262C46052230466946FAF71CFA90
:109290009DF800C0BDF80110BDF8032004EB4403A5
:1092A000013407F805C007EB430305360635142CD7
:1092B000A3F80110A3F80320E5D103B0F0BD00BF6F
:1092C0006404002064120020F0B5124B83B01868CB
:1092D000E8B10025104F04262C4604EB440307EBAD
:1092E000430317F805C0B3F801E0B3F803300522D3
:1092F0003046694601348DF800C0ADF801E0ADF8A4
:109300000330B6180635FAF7F9F9142CE5D103B095
:10931000F0BD00BF640400206412002010B50446B4
:1093200082B00B460092D02000222146FDF708FAB9
:10933000D0F1010038BF002002B010BD10B50446C6
:1093400082B00B460092D02000222146FDF776FA2B
:10935000D0F1010038BF002002B010BD30B583B09D
:10936000FDF7B6F93F200DF107010122FFF7D6FF07
:10937000054620B301240720244B0DEB00012246B3
:109380001C60FFF7CBFF10B39DF80730002B29D1ED
:1093900000200DF107010122FFF7C0FF0446B0B124
:1093A0009DF807301A0619D503F07F0300200DF150
:1093B000070101228DF80730FFF7C0FF0EE00E20F5
:1093C0000DF107010122FFF7A9FF044618B9002497
:1093D000204603B030BD9DF807306BB90C4B01221D
:1093E0001A60F5E7072000230DEB000122468DF8F7
:1093F0000730FFF7A3FFCBE70E200DF10701012295
:109400008DF80750FFF79AFFE8E700BFE41200204D
:10941000DC1200202DE9F04F474B89B01B681BB9C7
:10942000184609B0BDE8F08F836802690193C368EC
:1094300041690293D0F800E0013246F26763C6F258
:10944000666303926439049183FB0EBA0199DDF8D7
:109450000CB0476883FB0118029A83FB0B1B83FB4C
:1094600007C983FB022C049ACDF800B083FB02B23B
:1094700001990592039B029ADDF810B04FEAEE764F
:10948000C6EBAA06DDF814A0FD17CC178069D1172A
:10949000DA174FEAEB73C5EBA905C1EBAC01C3EBDF
:1094A000AA03DDF800C0059005EB850A03EB8300F5
:1094B000C4EBA8040090C2EBAC020198A7EB4A07EA
:1094C000DDF80CA006EB860B04EB840902EB820CA2
:1094D000AEEB4B0EA0EB4909DDF810B00298AAEBF9
:1094E0004C0CDDF800A009EB041901EB8108059C88
:1094F000A0EB4808ABEB4A0008EB01180CEB021C90
:1095000000EB03130EEB061E07EB051701340020DA
:1095100006A907228DF818E08DF819708DF81A90B9
:109520008DF81B408DF81C808DF81DC08DF81E3005
:10953000FFF704FF75E700BFDC1200202DE9F04FB4
:10954000394B8BB01B6804461BB900200BB0BDE83B
:10955000F08F002008A90722FFF7E0FE0028F4D0D2
:109560009DF825A09DF820709DF826804FEA1A1BD3
:109570009DF824304FEA171C0BEB8B0B4FEA1819A0
:10958000CDF81CB00CEB8C0C05939DF822209DF8B7
:10959000233009EB890908F00F08CDF800C0DDF889
:1095A0001CC00AF00F0ACDF80890CDF804809DF891
:1095B000215011090693DDF81490DDF80480059B15
:1095C000CDF80CA00AEB4C0ADDF808C002F00F023F
:1095D00001EB81012E091B0909F00F0B02EB410180
:1095E00008EB4C09069ADDF8008005F00F0504939E
:1095F00007F00F0706EB860603EB830305EB460631
:1096000002F1FF3C07EB48070BEB43030AF1FF3580
:1096100009F1640227606660A160C4F818C0E360C5
:109620002561626192E700BFDC12002000B50E4B9D
:1096300083B01B6853B1FF23C0F20203984207D8DE
:1096400000220120094B1A6003B000BD1846FBE759
:109650000122DF200DF10701FAF736F89DF8072007
:109660000A2A88BF0022EDE764040020E0120020EF
:1096700000B5094B094A1B68106883B08DF80730A4
:1096800040B1DF2001220DF10701FAF737F8003071
:1096900018BF012003B000BDE012002064040020C8
:1096A00041F2E023C2F200031868704710B541F29E
:1096B000E024C2F200042060FFF7DAFF206810BD4A
:1096C00000B50D4B83B01B68FF200BB903B000BD84
:1096D000112001A90222FFF721FE0028F6D09DF8F3
:1096E0000500064B9DF80420C0F340001B6840EACB
:1096F0004200C01AEAE700BFDC120020E01200209E
:1097000000B585B001A802A903AAF9F7CFFE10B9E8
:10971000FF2005B000BD029B002BF9D1024B186859
:10972000039B181AF5E700BFE812002000B50E4BA6
:1097300083B01B6853B1FF23C0F20203984207D8DD
:1097400000220120094B1A6003B000BD1846FBE758
:109750000122DF200DF10701F9F7B6FF9DF8072080
:109760000A2A88BF0022EDE764040020E8120020E6
:1097700000B5094B094A1B68106883B08DF80730A3
:1097800040B1DF2001220DF10701F9F7B7FF0030EA
:1097900018BF012003B000BDE812002064040020BF
:1097A00041F2E823C2F200031868704710B541F295
:1097B000E824C2F200042060FFF7DAFF206810BD41
:1097C0000920F9F7E5BE00BF00B5144B83B01B6854
:1097D0002BB1AA2012491022F9F776FF50B91022B6
:1097E0000F48104901F076FD0F4B01221A6000204E
:1097F00003B000BDBA2001A90222F9F765FF0028D5
:10980000EDD09DF804109DF80520074B01202D296F
:109810001A60EDD152421A600120E9E76404002089
:10982000CC010020A4E00008C801002000B5134BC3
:1098300083B01B68002B1ADB2B228DF804208DF8D7
:1098400005300F4B1B6813B9002003B000BDAA20E0
:109850000C491022F9F752FF0028F5D0BA20022255
:1098600001A9F9F74BFF003018BF0120EDE75B427B
:109870002D228DF804208DF80530E2E7C801002084
:1098800064040020CC01002040F2C813C2F200039F
:109890001868704710B5014604460A48FDF7A0FE57
:1098A00004F10C03182B0AD8074B1A68A24204D003
:1098B0001C60FFF7BBFF012010BD012010BD002080
:1098C00010BD00BFB4E00008C801002040F2CC1079
:1098D000C2F20000704700BF014640F2CC1008B54C
:1098E000C2F2000001F0CDFCBDE80840FFF79EBFCA
:1098F00040F2CC10C2F20000FAF790BA70B5284AD4
:1099000048F280131268C7F65543CB184FF46161D3
:1099100001FB023382B002AE46F8043D05463046F4
:1099200001F06CF903690446DA1E052A0CD9022BF2
:109930002BD0092B10D18369C268D21A182A03DDF3
:1099400053B98368022B07DC019B304603F5616342
:10995000019301F053F90446636904F10C006B6153
:1099600023692B61E368EB6007C8013102F26C7276
:10997000F6F7BEFCA861236A2B62A368AB6063683C
:109980006B6023682B6002B070BD8369C268D21A15
:10999000182AE1DD002BD7D18368012BD4DCDBE76B
:1099A000C801002008B5202000F05AFB28B1202073
:1099B00000F064FB014B00221A6008BDEC1200208D
:1099C0002DE9F843DFF800E10646DEF80030002B11
:1099D000FBD1002E6FD03A48770007EB060C3949CF
:1099E0008444182510F8029CA5F11803A5F110086D
:1099F000802212EA090F0CBF22243A24CC540133EE
:109A000052084345F5D110F8039CA5F108088022BF
:109A100012EA090F0CBF22243A24CC540133520815
:109A20004345F5D110F8018C802212EA080F0CBFD3
:109A300022243A24CC54013352089D42F5D10330FC
:109A400018356045CED10022CB181046985401320B
:109A5000302AFBD14FF4305001240021C4F2010020
:109A6000CEF8004000F03EFE1C200021C4F20200AF
:109A700000F0DEFABB19DB0030331C204FF6F87122
:109A80001940C4F2020000F0E9FA1C20022122462B
:109A9000C4F2020000F0D8FA1C202146C4F20200F1
:109AA00000F0C6FA4FF43050C4F201002146BDE880
:109AB000F84300F017BE334602493746C3E700BFFC
:109AC000F3120020FC140020EC120020AD2809D86D
:109AD0000A78054B00EB40001A544A781818427077
:109AE0008B788370704700BFF0120020F0B469B12A
:109AF0000A4D01EB410700230678EC18EE54467836
:109B0000033366708678BB42A670F5D10AB9F0BC03
:109B100070470846F0BCFFF753BF00BFF0120020AB
:109B20002DE9F0415D4D94B0002468462C6000F0B2
:109B300013FB0420012100F0DBFC18234FF400602C
:109B40004FF48078C4F2010069468DF80330032396
:109B50008DF80230ADF8008000F09AFA4FF4006002
:109B600022464146C4F2010000F004FB02A800F0C6
:109B7000A5FD05A800F0ACFD01214FF4006000F048
:109B8000B7FC0120014600F0A5FC4FF430505B23E8
:109B9000C4F2010002A9ADF80C30ADF80840ADF8F0
:109BA0000E40ADF80A4000F0CDFC4FF43050602379
:109BB0000126C4F2010005A9ADF81430ADF8166015
:109BC000ADF81A40ADF81C4000F01CFD4FF43050C9
:109BD0000821C4F2010000F0C5FD4FF43050C4F27A
:109BE0000100314600F0B0FD4FF43050C4F20100E6
:109BF000314600F085FD4FF4305032464FF400718D
:109C0000C4F2010000F096FD0C2301A88DF8043089
:109C10008DF805408DF806408DF8076000F042F899
:109C200009A800F0F7F91C202146C4F2020000F058
:109C3000FFF91C20C4F2020000F020F942F6344380
:109C4000C4F2010309934FF484531C200C93802326
:109C50000E934FF44053129310230B93104BC4F206
:109C6000020009A91194CDF83C8010940D9413942E
:109C70000A93274600F0AEF98DF824408DF8254070
:109C80008DF826402B68002BFCD109A8AE210122BB
:109C9000FFF72CFF14B0BDE8F08100BFEC120020EC
:109CA000FC140020C37830B47BB90378012103F0A1
:109CB0001F0201FA02F15A094FF46143CEF2000388
:109CC000203243F8221030BC70474FF46D43CEF27F
:109CD0000003DB684478DB43C3F302230F22C3F1A4
:109CE000040122FA03F304FA01F48578017803EA07
:109CF0000502224301F160431201D2B203F5614330
:109D000083F800230278012102F01F0301FA03F116
:109D10004FF46143CEF20003520943F82210D2E718
:109D200042680B6822F4702270B422F480720C79BD
:109D3000134343EA0423436086688C68CA684FF281
:109D4000FD73CFF6F1734D7922433340134343EA59
:109D5000450383600B7CC26A013B22F47002DBB2D4
:109D600042EA0353C36270BC704700BF0023036024
:109D7000037143718360C36001230374704700BFA4
:109D8000836819B923F001038360704743F001032E
:109D900083607047836843F008038360704700BFA7
:109DA0008068C0F3C0007047836843F00403836099
:109DB000704700BF8068C0F380007047836819B99E
:109DC00023F4A0038360704743F4A00383607047CB
:109DD000092970B401EB41041ED91E3C072606FA7E
:109DE00004F603FA04F4C568062A25EA060343EAE2
:109DF0000403C3601DD90C2A02EB820227D9413A21
:109E00001F2404FA02F401FA02F1C36A23EA0402ED
:109E10000A43C26270BC7047072606FA04F603FACA
:109E200004F40569062A25EA060343EA04030361EC
:109E3000E1D8013A02EB82021F2404FA02F401FA8B
:109E400002F1436B23EA04020A434263E2E7233A46
:109E50001F2404FA02F401FA02F1036B23EA04025C
:109E60000A430263D6E700BFC06C80B2704700BFF0
:109E7000036819420CBF002001207047082110B46C
:109E800004684FF6FE72C4F20201002322408842A9
:109E90000260036043608360C36050D01C23C4F23F
:109EA0000203984252D03023C4F20203984255D0A4
:109EB0004423C4F20203984258D05823C4F2020348
:109EC00098425BD06C23C4F2020398425ED0802398
:109ED000C4F20203984228D04FF48163C4F2020313
:109EE00098422AD040F21C43C4F20203984255D053
:109EF0004FF48663C4F20203984258D040F24443C0
:109F0000C4F2020398425BD04FF48B63C4F20203A5
:109F1000984201BF4FF48063C4F202035A6842F4CE
:109F2000702208BF5A6010BC70470023C4F20203BD
:109F30005A6842F070625A60F5E74FF48063C4F2E9
:109F400002035A6842F00F025A60ECE70023C4F2A1
:109F500002035A6842F0F0025A60E4E70023C4F2B8
:109F600002035A6842F470625A60DCE70023C4F2CC
:109F700002035A6842F470425A60D4E70023C4F2E4
:109F800002035A6842F470225A60CCE70023C4F2FC
:109F900002035A6842F470025A60C4E74FF48063C7
:109FA000C4F202035A6842F0F0025A60BBE74FF471
:109FB0008063C4F202035A6842F470625A60B2E7E6
:109FC0004FF48063C4F202035A6842F470425A604C
:109FD000A9E700BF8B68F0B40D6A0C694A691D439C
:109FE0002C438B691443CA6905684F6A23438E6A00
:109FF00013431F4325F4FF4525F070053E432E43D0
:10A000000660CB6843600B6883604B68C360F0BC3C
:10A01000704700BF0023036043608360C360036137
:10A0200043618361C361036243628362704700BF1F
:10A0300029B902684FF6FE73134003607047036846
:10A0400043F001030360704703681AB923EA010172
:10A050000160704719430160704700BF416070475D
:10A06000C1004CBF4FF480630023C4F202031B689D
:10A0700003420CBF00200120704700BFC3004CBF4B
:10A080004FF480630023C4F202035860704700BF9E
:10A09000CB782DE9F00303F00F06DB0648BF8B7881
:10A0A0000A8848BF1E4312F0FF0F27D0076800231D
:10A0B00001254FF00F0803E00133082B1CD00A885C
:10A0C00005FA03F42240A242F6D19C0008FA04F9F2
:10A0D00006FA04F491F803C027EA0907BCF1280F37
:10A0E00047EA040708BF4261E6D0BCF1480F08BF49
:10A0F00002610133082BE2D107600A88FF2A28D9C0
:10A100004768002301254FF00F0803E00133082BB7
:10A110001ED00A8803F1080405FA04F42240A24282
:10A12000F4D19C0008FA04F906FA04F491F803C08B
:10A1300027EA0907BCF1280F04BF426191F803C068
:10A140002743BCF1480F08BF02610133082BE0D15F
:10A150004760BDE8F00370474FF6FF7303800223AA
:10A1600083700423C3707047836819420CBF0020BA
:10A17000012070470AB9416170470161704700BF13
:10A1800030B400230028C4F2010300F44012B4BF2D
:10A19000DB695B68B2F5401F84B222D0C20217D5DA
:10A1A000C0F30342032505FA02F223EA020343F057
:10A1B000706321B1420D120104FA02F4234300221C
:10A1C000C4F201020028B4BFD361536030BC7047B1
:10A1D000420D120104FA02F223EA020343F0706313
:10A1E000E7E70022C4F20102556823F0706325F00E
:10A1F00070655560DDE700BF08B54FF4A843C4F2B1
:10A20000000398420BD001214FF4800000F08CF93C
:10A210004FF480000021BDE8084000F085B901211D
:10A220004FF4001000F080F94FF400100021BDE859
:10A23000084000F079B900BFF0B587B004468688C1
:10A2400001A80D4600F0F2F8039A4DF68363C4F2BC
:10A250001B33A3FB021326F03F06980C3604360C82
:10A2600087B23E43A680238848F2A06123F0010311
:10A270001B041B0C23802B68C0F201018B4222D8E7
:10A280005B00B2FBF3F292B201372784032A98BF36
:10A290000422A28323889BB243F0010323802388F6
:10A2A000698923F48163AA8823F002031B040A430B
:10A2B0001B0C13439BB223802A89AB8913439BB2A7
:10A2C000238107B0F0BDEE884BF6FF718E421DBFB3
:10A2D00003EB830303EB8303B2FBF3F203EB4303D0
:10A2E0000CBFB2FBF3F242F4804292B213051B0D95
:10A2F0000BB942F001024FF4967101FB00F044F6F5
:10A30000D351C1F2620181FB00318909013142F46C
:10A3100000422184BDE700BF002341F28832026081
:10A3200083804BF6FF72038143814FF48043C280E8
:10A3300083817047038829B923F001031B041B0C98
:10A34000038070479BB243F001030380704700BF56
:10A35000038829B923F480731B041B0C0380704706
:10A360009BB243F480730380704700BF038829B910
:10A3700023F400731B041B0C038070479BB243F44F
:10A3800000730380704700BF038829B923F48063FA
:10A390001B041B0C038070479BB243F48063038053
:10A3A000704700BF01827047008AC0B2704700BF8B
:10A3B0001AB901F0FE010182704741F001010182EA
:10A3C000704700BF038819B95B045B0C03807047BA
:10A3D0006FEA43436FEA53439BB20380704700BF69
:10A3E00082B000230A0F0093019301900092009B1A
:10A3F00021F07F4153B1019B14330193019B1B68F2
:10A4000019420CBF0020012002B07047019B090CCB
:10A4100018330193F2E700BF4FF48053C4F20203F4
:10A420005A6822F4404210435860704710B44FF409
:10A430008053C4F202035A6802F00C02042A01D0CD
:10A44000082A28D04FF49052C0F27A0202604FF4EA
:10A450008053C4F202035C681C49C4F303140C5D0E
:10A4600022FA04F242605C68C4F302240C5D22FA12
:10A4700004F484605C68C4F3C224095D22FA01F22A
:10A48000C2605B681249C3F38133CB5CB2FBF3F269
:10A49000026110BC70475A685968C2F383420232A5
:10A4A000CC030AD55B68990307D44FF49053C0F2EC
:10A4B0007A0303FB02F20260C9E74FF41063C0F2B3
:10A4C0003D0303FB02F20260C1E700BFE40100208C
:10A4D000E00100204FF48053C4F202035A6919B915
:10A4E00022EA00005861704710435861704700BF6E
:10A4F0004FF48053C4F202039A6919B922EA0000AA
:10A500009861704710439861704700BF4FF48053C3
:10A51000C4F20203DA6919B922EA0000D86170476F
:10A520001043D861704700BF4FF48053C4F2020358
:10A530001A6919B922EA00001861704710431861BE
:10A54000704700BF70B44FF430524FF45054C4F20F
:10A5500001020388C4F20104904218BFA0429BB2DA
:10A5600014BF0022012208D04FF48064C4F200041A
:10A57000B0F1804F18BFA04236D14FF68F754C888E
:10A580001D4045EA04034FF4A0564FF48055C4F231
:10A590000005C4F20006B04218BFA8421FBFCD8814
:10A5A0004FF6FF441C4044EA050303808B888385F3
:10A5B0000B8803855AB94FF488424FF48043C4F2A4
:10A5C0000102C4F20103984218BF904205D10B7AF0
:10A5D00003860123838270BC70474FF49043C4F21A
:10A5E00001039842F5D1F2E74FF440654FF400645F
:10A5F000C4F20005C4F20004A04218BFA842C2D1B0
:10A60000BBE700BF038C2DE9F00123F001031B041D
:10A610001B0C0384038C0D8984884F88028B2F4385
:10A6200022F0730223F002034FF450564FF43055DA
:10A6300012041B04B1F800C0C4F20106C4F2010503
:10A64000120C1B0CBFB2A84218BFB042A4B242EA1F
:10A650000C0247EA03030BD04FF488464FF48045C1
:10A66000C4F20106C4F20105A84218BFB0421ED1CF
:10A670004FF6F775B1F80AC0B1F80E808F891D400A
:10A6800045EA0C0C4FF6FB738E884FF6FF4548EAFF
:10A69000070725400CEA0303BCB233432C438480F4
:10A6A0000283CA8882860384BDE8F00170474FF4B4
:10A6B0009045C4F20105A842F1D1D9E700234FF635
:10A6C000FF7181800380C38043800372704700BFA5
:10A6D0000023038043808380C3800381438183817F
:10A6E000C3817047038829B923F001031B041B0CA5
:10A6F000038070479BB243F001030380704700BFA3
:10A70000B0F8443021B95B045B0CA0F844307047CA
:10A710006FEA43436FEA53439BB2A0F8443070475B
:10A7200083899BB21AB923EA0101818170471943D9
:10A730008181704783899BB21AB923EA0101818123
:10A740007047194381817047038829B923F080033A
:10A750001B041B0C038070479BB243F080030380F3
:10A76000704700BF038B23F008031B041B0C194325
:10A7700001837047C94389B20182704770B5038A6B
:10A78000CA8823F440531B041B0C134303828389A0
:10A7900004468A88088923F4B0530D4623F00C033D
:10A7A000498902431B040A431B0C13439BB2A38138
:10A7B000A38AAA8923F440731B041B0C86B013439D
:10A7C000A38201A8FFF732FE4FF46053A289C4F2BE
:10A7D00001039C4212B20CBF049B039B002A21DBA5
:10A7E000286803EB830303EB83038000B3FBF0F1E2
:10A7F00048F21F53C5F2EB13A3FB0102A0895209D3
:10A8000000B216016425002802FB151213DB1201A9
:10A810003232A3FB0203C3F3431333439BB22381BE
:10A8200006B070BD2A6803EB830303EB8303520079
:10A83000B3FBF2F1DCE7D2003232A3FB0213C3F325
:10A8400042133343EAE700BF4FF41652002302607D
:10A850000C228380C380038142818381704700BFC3
:10A86000838929B923F400531B041B0C838170478F
:10A870009BB243F400538381704700BF01F01F0374
:10A8800010B4C1F342110124A14204FA03F30DD024
:10A8900002290DD014302AB9026822EA03030360AA
:10A8A00010BC7047026813430360F9E70C30F2E70D
:10A8B0001030F0E7C905C90D818070478088C00558
:10A8C000C00D7047838919B95B045B0C83817047A5
:10A8D0006FEA43436FEA53439BB28381704700BFE3
:10A8E000C1F3421310B401F01F020124012B04FA3A
:10A8F00002F416D0022B0CBF028A828A92B2224046
:10A900000123090A03FA01F103889BB219420CBF23
:10A9100000200120002A0CBF002000F0010010BC24
:10A920007047828992B22240EAE700BF090A0123F8
:10A9300003FA01F3DB439BB2038070470649074AE1
:10A94000074B9A42BEBF51F8040B42F8040BF8E7DC
:10A95000044880470448004778E2000800000020CF
:10A96000B8020020F5A90008410100081F49204A4B
:10A97000002301E041F8043B9142FBD3FCF7A8FF20
:10A98000FEE7FEE7FEE7FEE7FEE7FEE7FEE7FEE79F
:10A99000FEE7FEE7FEE7FEE7FEE7FEE7FEE7FEE78F
:10A9A000FEE7FEE7FEE7FEE7FEE7FEE7FEE7FEE77F
:10A9B000FEE7FEE7FEE7FEE7FEE7FEE7FEE7FEE76F
:10A9C000FEE7FEE7FEE7FEE7FEE7FEE7FEE7FEE75F
:10A9D000FEE7FEE7FEE7FEE7FEE7FEE7FEE7FEE74F
:10A9E000FEE7FEE7FEE7FEE7FEE7FEE7B80200202F
:10A9F000782600204FF48053C4F202031968002225
:10AA000041F0010119605968CFF6FF020A405A600F
:10AA10001A68002122F0847222F480321A601A68C7
:10AA200082B022F480221A6058681A4620F4FE0090
:10AA300058604FF41F00986000910191196841F42B
:10AA40008031196003E0009BB3F5A06F09D0136853
:10AA500003F400330193009B01330093019B002B0F
:10AA6000F1D04FF48053C4F202031B6813F4003397
:10AA700008BF019301D001230193019B012B08D052
:10AA80004FF46D43CEF200034FF000629A6002B0C3
:10AA900070474FF40052C4F2020211684FF4805321
:10AAA00041F0100111601168C4F2020321F00301AA
:10AAB00011601068194640F0020010605A685A6030
:10AAC0005A685A605A6842F480625A605A6822F49E
:10AAD0007C125A605A6842F4E8125A601A6842F0CE
:10AAE00080721A600A684FF480539201C4F2020324
:10AAF000F8D559681A4621F003015960596841F0A8
:10AB000002015960536803F00C03082BFAD1B7E730
:10AB10004FF48053C4F202035A6802F00C02082A70
:10AB20001CBF4FF49052C0F27A020DD04FF4805304
:10AB3000C4F202035B681049C3F30313CB5C22FA2F
:10AB400003F20E4B1A6070475A685968C2F3834289
:10AB50000232C80309D55B68990306D44FF49053B9
:10AB6000C0F27A0303FB02F2E0E74FF41063C0F295
:10AB70003D0303FB02F2D9E7F401002004020020A8
:10AB800000210A2200F046BC08B5074B044613B169
:10AB90000021AFF30080054B1868836A03B1984722
:10ABA000204601F071F800BF00000000CCE0000872
:10ABB00070B50E4B0E4D0024ED1AAD101E4603E08D
:10ABC00056F8242090470134AC42F9D101F05EF8E8
:10ABD000084D094B0024ED1AAD101E4603E056F84F
:10ABE000242090470134AC42F9D170BDB00200205E
:10ABF000B0020020B4020020B002002038B5074B9C
:10AC000005461C68E36B1BB9242000F00DF8E063D7
:10AC1000E16B2846BDE8384000F002B86802002029
:10AC2000002200F0C3B80000024B0146186800F093
:10AC300047BA00BF6802002010B5002302E0CC5CD8
:10AC4000C45401339342FAD110BD8218034601E087
:10AC500003F8011B9342FBD1704700002DE9F74F29
:10AC6000064600F09FFF40F2B1739E42024640F359
:10AC700096806FF4F663F318A6F2B2719B1040F25F
:10AC80006D1505FB0135A6F26D716FF0630391FB45
:10AC9000F3F36FF4C861ED1871184FF4C87391FBAA
:10ACA000F3F16D18642196FBF1FC01FB1C6C96FB23
:10ACB000F3F103FB11614660D1F1010106F00306D7
:10ACC00038BF002101960346022407261F7A4A2F27
:10ACD00011D15F69019805EB070810B9BCF1000FAD
:10ACE00000D121B13B2FD4BF0027012700E00F4640
:10ACF0004744013F3FE0442F02D15F69EF193AE03A
:10AD0000019F37B9BCF1000F0CBF89464FF0010914
:10AD100000E0894623484FF0300808FB0909D3F8C2
:10AD20000CA0A846012705E009EB870B5BF804BCE3
:10AD30000137D8445745F7DB08F1040797FBF6FBCA
:10AD400006FB1B7B5F691869BAF1010FB8BF4FF0B2
:10AD5000010AB7EB0B0748BF073700F1FF3B0AF1C9
:10AD6000FF3A072000FB0B7759F82A9000E0073FD5
:10AD70004F45FCDA47449869DFF82C80013C08FB1A
:10AD80000707186A074443F81C7F9FD1936BD1696A
:10AD90009942ACBF002301231360012000E0002092
:10ADA000BDE8FE8FD0E00008805101002DE9F84396
:10ADB00080460C46174600F0F5FED8F800109B4A76
:10ADC000064691FBF2F302FB131104E001F5A831F2
:10ADD00001F5C071013B0029F8DB4FF4616091FB84
:10ADE000F0F200FB12113C20A26091FBF0F200FB9C
:10ADF0001211626021601A1D072192FBF1F001FB24
:10AE00001022002AB8BF0732002BA26140F2B275AF
:10AE10004FF4C8704FF0640CDFF81C9217DBA907E1
:10AE200004D195FBFCF20CFB125242B995FBF0F1F8
:10AE300000FB1151D1F1010138BF002100E00121D7
:10AE400059F82120934218DB01359B1AE7E7013DB1
:10AE5000AA0704D195FBFCF20CFB125242B995FBF8
:10AE6000F0F100FB1151D1F1010138BF002100E0E8
:10AE7000012159F821209B18E9D4A5F26C72626176
:10AE80006B4A4FF0300909FB01290022E36122617E
:10AE900002E001319B1A2161216959F82120934276
:10AEA000F7DA0133E360002F40F0BB8000F0A6FC2E
:10AEB000604B1B681BB373689D4205D13168D8F89D
:10AEC0000030F26931B90CE02846FFF7C7FE0028D0
:10AED000F4D110E093420CDBB26B934209DA012308
:10AEE0000BE09342FBDAB26B9342ACBF0023012329
:10AEF00003E0002301E04FF0FF33236200E027620C
:10AF0000236A4FF46160012B0CBFF36B336A256831
:10AF100093FBF0F200FB12333C2093FBF0F100FBBB
:10AF200011336068EB1A411AA0683B2BC2EB000298
:10AF300023606160A26003DD013161603C3B04E09D
:10AF4000002B03DA013961603C33236063683B2BDB
:10AF500003DD0132A2603C3B04E0002B03DA013A3E
:10AF6000A2603C336360A368172B1FDDE2690132E6
:10AF7000E261A2690132062AC8BF0022A261E2682A
:10AF8000183B0132A3602369E26059F823108A421A
:10AF900044DD0133521A0C2BE26023613ED1626919
:10AFA0000023013223616261E36137E0002B35DA6F
:10AFB000E269013AE261A269013A48BF0622A26150
:10AFC000E2681833013AE260A3603ABB2369013BAF
:10AFD00001D423611EE00B23236163695A1E12F022
:10AFE000030F626103F26B7305D1642293FBF2F1EC
:10AFF00002FB113252B94FF4C87293FBF2F102FB1B
:10B000001133D3F1010338BF002300E0012303F51E
:10B01000B673E361236959F82330E36000F0EFFB76
:10B0200001E0002323622046BDE8F883805101003F
:10B03000D0E000088425002030E1000830B5002968
:10B040003BD051F8042C0B1F1C49002AB8BF9B1899
:10B050000A6812B95A600B6030BD93420CD219686D
:10B060005818904203D15A588918426819605A609A
:10B07000124A136030BD0A46516809B19942FAD9A3
:10B08000146815199D420AD11B68E318D01888422C
:10B09000136012D108681B1813604B680CE002D9CA
:10B0A0000C23036030BD18681C188C4203D10C6857
:10B0B0004968001918605960536030BD8025002030
:10B0C000F8B5CD1C25F0030508350C2D38BF0C252F
:10B0D000002D064645DB8D4200D242E0234B1B6823
:10B0E0001C4612E02268521B0DD40B2A02D92260A2
:10B0F000A4181EE0A34203D163681C4A136021E038
:10B1000062685A601EE023466468002CEAD123E09E
:10B110003046214600F06AF838602946304600F093
:10B1200065F8431C01461CD0C41C24F0030484426F
:10B1300001D1256006E03046611A00F057F8013071
:10B14000F7D10EE004F10B00231D20F00700C31A15
:10B150000AD05A42E250F8BD054F3B68002BDCD1C3
:10B16000D6E70C2333600020F8BD00BF8025002007
:10B170007C2500201A4B10B51C68A36BD3B918208E
:10B18000FFF752FD43F20E33A06303804AF6CD333E
:10B19000438041F2342383804EF26D63C3804DF6C9
:10B1A000EC630381052343810B2383810122002368
:10B1B000C0E90423A46B0B492069626941430A4B2F
:10B1C00003FB0212A0FB03015118012200231218F5
:10B1D00043EB0103C4E9042323F0004010BD00BF8A
:10B1E000680200202DF451582D7F954C38B5064C3F
:10B1F000002305460846236000F02CFD431C02D1C5
:10B20000236803B12B6038BD742600200EB400B54E
:10B210004FF402719CB0ADF814106FF0004104912E
:10B2200007914FF6FF711DABADF81610084953F8A2
:10B23000042B02900690086802A9019300F0E6F939
:10B24000029B00221A701CB05DF804EB03B070473B
:10B2500068020020C9B2034610F8012B12B18A42DD
:10B26000F9D102E0002918BF00231846704710F8F2
:10B27000012B11F8013B012A28BF9A42F7D0D01ABE
:10B280007047034611F8012B03F8012B002AF9D16E
:10B290007047034613F8012B002AFBD1181A013816
:10B2A000704770B5A2B108E0012A03D128781B7855
:10B2B000C01A70BD013A002CF8D00B460546002A92
:10B2C000F4D010F8016B1C780131B442ECD0EDE7FA
:10B2D000104670BD30B50139034609E011F8015F31
:10B2E000013A03F8015B1C4615B99B18002205E0E2
:10B2F0001C46002AF2D1F8E704F8012B9C42FBD14E
:10B3000030BD00002DE9F74F01904148D0F8009082
:10B310000846044614F8015B09EB050677782046D9
:10B3200007F00807FFB2002FF3D12D2D03D114F839
:10B33000015B012704E02B2D04BF244614F8015BB8
:10B34000002B5ED0102B08D158E02078782801D04F
:10B3500058284ED1657810230234002F0CBF6FF0AF
:10B3600000404FF00040B0FBF3FA002603FB1A0840
:10B37000304609EB050C9CF801C00CF0040B5FFA99
:10B380008BFBBBF1000F01D0303D0BE01CF0030C38
:10B390001BD0BCF1010F14BF4FF0570C4FF0370C0E
:10B3A000CCEB05059D4210DAB6F1FF3F0AD05045BF
:10B3B00006D801D1454503DC03FB0050012601E01E
:10B3C0004FF0FF3614F8015BD3E7731C0AD1002F4E
:10B3D00001990CBF6FF000404FF0004022230B603A
:10B3E00022B912E007B140427AB106B1611E116084
:10B3F0000BE03025002BB0D10823AEE7302DACD1C7
:10B40000A3E7302DA1D00A23A7E7BDE8FE8F00BF38
:10B410006C02002030B51346044A05460C461068FD
:10B4200029462246BDE83040FFF76CBF6802002085
:10B430002DE9F74F01903D48D0F8009008460446AA
:10B4400014F8015B09EB05067778204607F008073A
:10B45000FFB2002FF3D12D2D03D114F8015B01278A
:10B4600004E02B2D04BF244614F8015B002B57D0B9
:10B47000102B08D151E02078782801D0582847D1E6
:10B480006578102302344FF0FF3ABAFBF3FA03FB5E
:10B490000AF000266FEA0008304609EB050C9CF81C
:10B4A00001C00CF0040B5FFA8BFBBBF1000F01D065
:10B4B000303D0BE01CF0030C1BD0BCF1010F14BF9E
:10B4C0004FF0570C4FF0370CCCEB05059D4210DACE
:10B4D000B6F1FF3F0AD0504506D801D1454503DCFF
:10B4E00003FB0050012601E04FF0FF3614F8015B2A
:10B4F000D3E7731C05D1019922230B60304622B992
:10B5000012E007B140427AB106B1611E11600BE052
:10B510003025002BB7D10823B5E7302DB3D1AAE7EA
:10B52000302DA8D00A23AEE7BDE8FE8F6C020020C4
:10B5300030B51346044A05460C4610682946224693
:10B54000BDE83040FFF774BF680200202DE9F047E6
:10B550008D688146AB420C4692461F463FD38A898E
:10B5600012F4906F39D0266809696369C1EB060847
:10B5700003265E43022508F1010302F4806296FB74
:10B58000F5F6DB1912B29E4238BF1E4682B1314633
:10B59000FFF796FD054600B913E021694246FFF723
:10B5A0004BFBA38923F4906343F08003A3810CE059
:10B5B000324600F022FB054638B948462169FFF7BC
:10B5C0003DFD0C23C9F8003018E025616661454453
:10B5D000C8EB06062560A6603D46AF4200D23D4658
:10B5E0002A462068514600F0EFFAA36800205B1B52
:10B5F000A36023685D192560BDE8F087A3894FF03B
:10B60000FF3043F04003A381BDE8F0872DE9F04F00
:10B610009DB003938B89064603F080031BB20D4651
:10B62000144663B10B6953B94021FFF749FD286007
:10B63000286110B90C233360D0E040236B610023F4
:10B64000099320238DF82930DFF89C813023DFF81F
:10B650009C918DF82A3023469A4613F8012B1AB98B
:10B66000BAEB040B0FD002E0252AF5D1F8E73046FB
:10B67000294622465B46FFF769FF013000F0A780AC
:10B68000099B5B4409939AF80030002B00F09F80DF
:10B6900000234FF0FF3204930793059206938DF831
:10B6A00053301A930AF1010A4FF0010B05E0C8EB81
:10B6B00000000BFA00F00343049354464A482178F3
:10B6C000052200F073FA0AF1010A049B0028EED16A
:10B6D000D90602D520228DF853201A0702D52B2235
:10B6E0008DF8532022782A2A03D0079B21460A206E
:10B6F00010E0039A111D12680391002A01DB0792E2
:10B7000004E0524243F0020307920493013408E03C
:10B7100000FB03230C4622780131303A092AF7D97D
:10B72000079323782E2B19D163782A2B09D1039BF9
:10B7300002341A1D1B680392002BB8BF4FF0FF3371
:10B740000BE0611C00230A2001E000FB03230C46F0
:10B7500022780131303A092AF7D905932348217814
:10B76000032200F023FA40B14023C9EB000003FAA2
:10B7700000F0049B01340343049314F8011B1C489C
:10B7800006228DF8281000F011FA88B1194B33B950
:10B79000039B073323F007030833039313E003AB42
:10B7A0000093304604A92A46134BAFF3008007E00C
:10B7B00003AB0093304604A92A460F4B00F092F8E1
:10B7C000431C074603D0099BDB19099343E7AB8968
:10B7D00003F040031BB20BB9099801E04FF0FF30B2
:10B7E0001DB0BDE8F08F00BF38E100083EE1000861
:10B7F00042E10008000000004DB5000870477047A6
:10B800002DE9F04715461F468A680B6906469A429D
:10B81000A8BF13462B6091F843200C46DDF820802A
:10B820000AB101332B602368990602D52B680233D5
:10B830002B60236813F0060916D094F84330226871
:10B84000003318BF0123920616D41EE001233046B0
:10B8500039465246C047013003D14FF0FF30BDE8B2
:10B86000F08709F1010901E004F1190AE1682B6888
:10B87000CB1A9945EADBE0E7E218302182F8431061
:10B8800094F84510023382F844103046394604F1EA
:10B890004302C0470130E0D023682A68E16803F022
:10B8A0000603042B08BFC2EB01052369A2680CBF85
:10B8B00025EAE57500259A42C4BFC3EB0203ED18E3
:10B8C0004FF000091A3408E0012330463946224679
:10B8D000C0470130C1D009F10109A945F4DB0020BE
:10B8E000BDE8F0872DE9FF470E7E91466E2E80461B
:10B8F0000C469A460C9D01F1430200F0AF800FD830
:10B90000632E1DD006D8002E00F0C080582E40F0C7
:10B91000D0804FE0642E1CD0692E40F0CA8018E021
:10B92000732E00F0B78005D86F2E2BD0702E40F00C
:10B93000C08043E0752E25D0782E40F0BA8041E0DB
:10B940002B6801F142071A1D1B682A6081F84230FA
:10B95000B3E021682B6811F0800F02D0191D296017
:10B9600008E011F0400F03F10401296002D0B3F99F
:10B97000005000E01D68002D45DA2D236D4284F84B
:10B98000433040E021682B6811F0800F02D0191D70
:10B99000296007E011F0400F03F10401296001D094
:10B9A0001D8800E01D68237E5F486F2B14BF0A23AB
:10B9B000082324E081F845605B4807E00B6843F00A
:10B9C00020030B607823594884F8453021682B68A0
:10B9D00011F0800F03F104062E6000D003E04F0643
:10B9E00001D51D8800E01D68CE0744BF41F020014D
:10B9F00021601DB9236823F0200323601023002158
:10BA000084F8431001E048480A236668002EA660C7
:10BA100003DB216821F00401216005B96EB104F156
:10BA20004201B5FBF3F603FB1655455D0F4601F8E1
:10BA300001593546002EF4D100E01746082B0AD1F3
:10BA40002368DB0707D561682369994203DC30234B
:10BA500007F8013C013FD21B226133E009682B68E3
:10BA600011F0800F05D0191D2960196863690B60FA
:10BA70000CE011F0400F03F10401296003D01968B4
:10BA800063690B8002E061691B6819600023236110
:10BA9000174617E02B681A1D2A601F683846FFF703
:10BAA000F8FB63682061984288BF23612369636063
:10BAB00005E004F1420784F842600123236100237A
:10BAC00084F84330CDF800A04046214603AA4B46F7
:10BAD000FFF796FE013002D14FF0FF3021E04046E3
:10BAE00049463A462369D0470130F5D02368980784
:10BAF0000ED4E068039B9842B8BF184611E00123BA
:10BB0000404649463246D0470130E5D0013502E093
:10BB1000002504F11906E168039BCB1A9D42EEDB78
:10BB2000E7E704B0BDE8F08749E100085AE1000802
:10BB300030B5141E9BB0054604DA8B2303604FF02A
:10BB4000FF301DE04FF40272ADF80C20009104911B
:10BB500001D0611E00E021464FF6FF72029105916F
:10BB6000ADF80E2028461A4669461E9BFFF74EFD8B
:10BB7000431C01DA8B232B6014B1009B00221A7046
:10BB80001BB030BD73B50093054B06460D461446F9
:10BB9000186831462A462346FFF7CAFF7CBD00BF1E
:10BBA00068020020004870477002002010B5C9B23A
:10BBB0000346821803E0047801338C4203D0934299
:10BBC0001846F8D1002010BD814210B511D28C1852
:10BBD000A0420ED253428118E418CB1801E0A15CB8
:10BBE000995412F1FF32FAD210BDCC5CC454013327
:10BBF00000E000239342F8D110BDF8B50646154683
:10BC00000C4621B91146BDE8F840FFF759BA1AB9F8
:10BC1000FFF714FA2C4612E000F013F8A8420ED2F7
:10BC200030462946FFF74CFA074638B121462A46E6
:10BC3000FFF702F830462146FFF700FA3C4620465F
:10BC4000F8BD51F8040C002802DA04390B58C0186A
:10BC500004387047094A136863B118186946884266
:10BC600098BF106004D9064B0C221A604FF0FF33C6
:10BC700018467047034B1360EFE700BF882500208C
:10BC80007426002078260020FEE700BFF8B500BF2C
:10BC9000F8BC08BC9E467047F8B500BFF8BC08BCAD
:10BCA0009E46704765617374657220646174653A7D
:10BCB00020253034642D253032642D253032640D3A
:10BCC0000A000000536F00004D6F0000446900003F
:10BCD0004D690000446F000046720000536100008F
:10BCE000537500005475000057650000546800004B
:10BCF0004443463737204572726F723A204869676D
:10BD0000682070756C7365203C3D20350000000094
:10BD10004443463737204572726F723A204869674C
:10BD2000682070756C7365203E3D20323500000040
:10BD30004443463737204572726F723A2070617201
:10BD400069747920503120696E636F727265637413
:10BD5000000000004443463737204572726F723A44
:10BD60002070617269747920503220696E636F723D
:10BD70007265637400000000444346373720457203
:10BD8000726F723A20706172697479205033206941
:10BD90006E636F7272656374000000000000000043
:10BDA0000000000006090906000000000A040A0A53
:10BDB0001F110000110E1111110E000012090909C6
:10BDC00009060000040A0A0A090A0000000000002F
:10BDD0000000000000000000000000000000000063
:10BDE0000000000000000000000000000000000053
:10BDF0000000000000000000000000000000000043
:10BE00000000000000000000000000000000000032
:10BE10000000000000000000000000000000000022
:10BE20000000000000000000000000000000000012
:10BE30000000000000000000000000000000000002
:10BE400000000000000000000000000000000000F2
:10BE500000000000000000000000000000000000E2
:10BE600000000000000000000000000000000000D2
:10BE700000000000000000000000000000000000C2
:10BE800000000000000000000000000000000000B2
:10BE900000000000000000000000000000000000A2
:10BEA0000000000004040404000400000A0A00006A
:10BEB0000000000000051F0A1F140000040E0C04FF
:10BEC000060E040009150E0E15120000040A0C15CA
:10BED000120D000004040000000000000304080824
:10BEE000080403001804020202041800040A040AE9
:10BEF00000000000000000040E040000000000002C
:10BF0000000404080000000E000000000000000013
:10BF100000040000010202040408080006090909DF
:10BF200009060000040C0404040E00000C020204C4
:10BF3000080E00000C020C02020C000002060A0FA0
:10BF4000020200000E080C02020C000006080E0996
:10BF5000090600000F010204040400000609060996
:10BF60000906000006090907010600000000040098
:10BF70000004000000000400000404080001020C9A
:10BF80000201000000000F000F0000000008040381
:10BF9000040800000E010204000400000609131545
:10BFA00017100F0000040A0A1F110000000E0A0CEF
:10BFB0000A0E00000007080808070000000E090923
:10BFC000090E0000000E080E080E0000000E080EFC
:10BFD000080800000007080B090700000009090F06
:10BFE00009090000000E0404040E0000000E020205
:10BFF000020C000000090A0C0A09000000080808E9
:10C00000080F000000111B151511000000090D0B91
:10C0100009090000000E1111110E0000000E090E9A
:10C0200008080000000E1111110E0201000C0A0C8C
:10C030000A09000000060804020C0000001F0404A6
:10C0400004040000000909090906000000090909A3
:10C0500006060000001115150A0A000000110A0466
:10C060000A11000000110A0404040000000F010678
:10C07000080F000006040404040406001008080465
:10C08000040202000C04040404040C00040A0A1153
:10C09000110000000000000000001F000804000064
:10C0A0000000000000000C020E0F000008080E093E
:10C0B000090E0000000006080806000002020E1229
:10C0C000120E00000000040E0806000003040F0416
:10C0D00004040000000007090F010E0008080A0D03
:10C0E0000909000004000C040404000002000E0210
:10C0F00002020C0008080A0C0A0900000C040404DF
:10C10000040400000000151F1515000000000A0DB2
:10C1100009090000000006090906000000000E09D8
:10C12000090E080000000E12120E020000000A0C98
:10C13000080800000000060C020C000000040F04B8
:10C1400004020000000009090B05000000000909B5
:10C1500006060000000015150E0A00000000090682
:10C16000060900000000090906061C0000000E0672
:10C17000080E00000204040804040200040404047D
:10C180000404040008040402040408000000000D74
:10C190001200000000040A0A0A0E0000000001005C
:10C1A0000100020002000300030004000400050077
:10C1B000050006000700080009000B000D000E0036
:10C1C000100012001400170019001C001F002100AD
:10C1D000240028002B002E003200360039003D00DC
:10C1E000420046004A004F00540059005E006300C0
:10C1F00069006E0074007A00800086008C00930055
:10C200009900A000A700AE00B600BD00C500CD009B
:10C21000D500DD00E500EE00F600FF00257500000A
:10C220004E6F6E65000000005261696E626F7700AC
:10C230004661646500000000526F6C6C00000000F5
:10C240004578706C6F64650052616E646F6D0000BC
:10C25000536E616B6500000054656C6574797065A0
:10C260000000000043756265000000004D617472BB
:10C270006978000044726F700000000053717565AA
:10C28000657A65004E6F726D616C0000436C6F6380
:10C290006B320000080809090A0A0B0B0C0C0D0D83
:10C2A0000E0E0F000000000000000100030A000055
:10C2B0000100040A00000100080A00000101040B4B
:10C2C0000C000101030B0C0001010C000000010136
:10C2D000030A0C000101040A0C000101080B000014
:10C2E0000101040B00000101030B0000000000002D
:10C2F00000000100030A00000100040A000001011F
:10C30000080000000101040B0C000101030B0C00EC
:10C3100001010C0000000101030A0C000101040AE4
:10C320000C000101090000000101040B00000101E3
:10C33000030B00000000000000000100030A0000E1
:10C340000100040A00000100080A00000100050ABB
:10C3500000000101030B0C0001010C0000000101B1
:10C36000030A0C000101050B00000101080B00008D
:10C370000101040B00000101030B0000000000009C
:10C3800000000100030A00000100040A000001018E
:10C39000080000000100050A00000101030B0C0069
:10C3A00001010C0000000101030A0C000101050B52
:10C3B00000000101090000000101040B000001015F
:10C3C000030B000045534B4953544C46DC4E46008A
:10C3D0005A45484E5A57414E5A49470044524549DA
:10C3E0005649455254454C0054474E414348564FD8
:10C3F000524A4D0048414C42515A57D64C46500083
:10C400005A5745494E53494542454E004B445245C3
:10C4100049524846DC4E4600454C464E45554E5620
:10C420004945520057414348545A45484E525300DB
:10C43000425345434853464D554852005745535380
:10C44000490000004F53534900000000524845493D
:10C450004E2D525548520000534348574142454ED5
:10C4600000000000000000000002000303000704B9
:10C47000010004010407020004020404020407028C
:10C48000000B030204030603040004040505050071
:10C490000405020305020405050606010406070457
:10C4A000070003070304070704080104080504093B
:10C4B00001050908030000000D1A0F1A0E1A121ABE
:10C4C000161A131A191A111A171A151A181A141AF1
:10C4D0000D0010000E0012001600130019001100CC
:10C4E00017001500180014002800000054696D653D
:10C4F0006F757400290D0A004F4B00004552524FD2
:10C50000520000002D200000495041444452455340
:10C5100053200000415020004D4F444520000000B2
:10C520006170000054494D45200000004649524DBD
:10C530005741524520000000434D442000000000B8
:10C540004854545020474554200000002D2D3E20D3
:10C55000000000003C30643E3C30613E0D0A0000AB
:10C560003C253032783E0000636170202225732222
:10C570002C22257322000000617020222573222CBA
:10C58000222573220000000074696D652022257346
:10C590002200000045535038323636204C4F474772
:10C5A00045520D0A0000000054D300085CD3000877
:10C5B00064D300086CD3000870D3000874D300085B
:10C5C00078D300087CD3000890CC000898CC0008F1
:10C5D000A0CC000844DF0008A4CC0008B0C60008C6
:10C5E000B0C60008B0C60008B0C60008B0C6000853
:10C5F0000400000002000000020000000200000031
:10C600000200000084D3000890D3000854D300082F
:10C610005CD300087CD3000888D000088CD00008C8
:10C6200094D00008F0CF000894D3000898D30008F5
:10C6300044D1000844D1000844D100089CD300082C
:10C640009CD300089CD3000854D30008A0D3000852
:10C6500034CA0008B0D300087CD3000854D30008C3
:10C66000A0D3000834CA00087CD30008BCD300085B
:10C67000C4D30008CCD30008D0D30008D8D3000816
:10C68000DCD30008F4CF00087CD300086163746930
:10C69000766500002573256400000000485454505E
:10C6A0002F312E3020323030204F4B000D0A0D0A32
:10C6B000000000003C68746D6C3E0D0A0000000034
:10C6C0003C686561643E0D0A000000003C746974BA
:10C6D0006C653E003C2F7469746C653E0D0A000069
:10C6E0003C2F686561643E0D0A0000003C626F6487
:10C6F000793E0D0A000000003C48313E0D0A000062
:10C700003C2F48313E0D0A003C6120687265663D51
:10C71000222F0000223E00003C2F613E266E6273F5
:10C72000703B266E6273703B0D0A00004D61696EAE
:10C73000000000006E6574776F726B004E65747751
:10C740006F726B0054656D7065726174757265000F
:10C750006C6472004C445200446973706C617900DF
:10C76000616E696D6174696F6E730000416E696D11
:10C770006174696F6E730000616D62696C696768EE
:10C7800074000000416D62696C69676874000000A4
:10C7900074696D657273000054696D657273000091
:10C7A0003C503E003C7472206267636F6C6F723D58
:10C7B000236630663066303E0D0A00003C74723EDF
:10C7C0000D0A00003C74643E000000003C2F7464BD
:10C7D0003E0000003C696E70757420747970653D90
:10C7E0002274657874222069643D220022206E61E3
:10C7F0006D653D2200000000222076616C75653D6C
:10C800002200000022206D61786C656E6774683DBF
:10C8100022000000222073697A653D22000000009A
:10C820003C74643E3C627574746F6E2074797065FC
:10C830003D227375626D697422206E616D653D22C3
:10C84000616374696F6E222076616C75653D227339
:10C8500061766500223E5365743C2F627574746F77
:10C860006E3E00003C2F74643E0D0A003C74616211
:10C870006C6520626F726465723D303E0D0A000087
:10C880003C2F74723E0D0A003C74683E3C666F6E2D
:10C890007420636F6C6F723D626C75653E000000C2
:10C8A0003C2F666F6E743E3C2F74683E0D0A00008C
:10C8B0003C2F7461626C653E3C503E0D0A000000E6
:10C8C0003C627574746F6E20747970653D22737567
:10C8D000626D697422206E616D653D2261637469C9
:10C8E0006F6E222076616C75653D22003C2F62756B
:10C8F00074746F6E3E266E6273703B003C2F626FE5
:10C9000064793E0D0A0000003C2F68746D6C3E0D8A
:10C910000A0000003C73656C6563742069643D2205
:10C9200000000000223E0D0A000000003C2F73654D
:10C930006C6563743E0D0A003C6F7074696F6E2005
:10C9400076616C75653D22002073656C6563746566
:10C95000640000003C2F6F7074696F6E3E0D0A001A
:10C96000266E6273703B3C696E70757420747970CA
:10C97000653D22636865636B626F7822206E616D2E
:10C98000653D2200222076616C75653D22616374ED
:10C990006976652220000000636865636B6564004A
:10C9A0003C696E70757420747970653D2272616E99
:10C9B0006765222069643D220000000022206D6925
:10C9C0006E3D220022206D61783D2200222073748A
:10C9D000796C653D2277696474683A0070783B0031
:10C9E00022206F6E696E7075743D22005F6F7574E2
:10C9F0007075742E76616C75653D00002E76616CE5
:10CA00007565223E000000003C6F757470757420DF
:10CA10006E616D653D2200005F6F757470757422E4
:10CA20003E0000003C2F6F75747075743E0000006E
:10CA30002E0D0A0044656661756C74003135000086
:10CA40003C666F726D206D6574686F643D2247456A
:10CA5000542220616374696F6E3D222F0000000034
:10CA60003C2F666F726D3E0D0A000000436F6C6FC5
:10CA7000727300003C74643E0D0A000036340000FE
:10CA8000266E6273703B266E6273703B266E627315
:10CA9000703B0D0A000000004C6561726E696E67A4
:10CAA0002049522072656D6F746520636F6E7472D9
:10CAB0006F6C2E2E2E000000537769746368696EC8
:10CAC0006720706F776572206F6E2E2E2E0000002B
:10CAD000537769746368696E6720706F7765722039
:10CAE0006F66662E2E2E00006F66666C696E65009E
:10CAF0004D696E696D756D206C656E677468206F29
:10CB000066206B65792069732031302100000000B8
:10CB100054696D65736572766572207375636365BC
:10CB2000737366756C6C79206368616E6765642EDB
:10CB30000000000053657474696E67206F66206E94
:10CB400065772074696D65736572766572206661BC
:10CB5000696C65642E00000054696D657A6F6E65BE
:10CB6000207375636365737366756C6C7920636895
:10CB7000616E6765642E000053657474696E67208A
:10CB80006F66206E65772074696D657A6F6E6520BB
:10CB90006661696C65642E0047657474696E672010
:10CBA0006E65742074696D650000000044697370DF
:10CBB0006C6179696E672074656D706572617475FA
:10CBC00072652E2E2E00000053746F726564206D06
:10CBD000696E696D756D2076616C75650000000089
:10CBE00054657374696E6720646973706C61792E23
:10CBF0002E2E0000536176696E6720736574746928
:10CC00006E6773207065726D616E656E746C792EDF
:10CC10002E2E00006874747020706174683A2027AA
:10CC20002573270D0A00000068747470207061720B
:10CC3000616D65746572733A20272573270D0A00AC
:10CC40002F000000253032642E25303264000000B1
:10CC5000253464002530326400000000616374698B
:10CC60006F6E00006C6561726E697200706F77653F
:10CC7000726F6E00706F7765726F666600000000FD
:10CC8000736176656461746574696D6500000000A8
:10CC900079656172000000006D6F6E7468000000BD
:10CCA000646179006D696E00736176657469636BA8
:10CCB00065720000576F7264436C6F636B00000015
:10CCC00056657273696F6E00454550524F4D0000B6
:10CCD000454550524F4D2056657273696F6E000086
:10CCE0005469636B65720000506F776572204F6EF8
:10CCF00000000000506F776572204F6666000000EC
:10CD00004C6561726E2049522072656D6F746520AA
:10CD1000636F6E74726F6C00656570726F6D6475B1
:10CD20006D700000454550524F4D2064756D700088
:10CD30003C503E0D0A3C666F6E7420636F6C6F72E0
:10CD40003D677265656E3E003C5052453E000000F6
:10CD50002530347800000000202000003C2F505285
:10CD6000453E0000202020002F6E6574776F726BA7
:10CD70000000000073617665776C616E0000000052
:10CD8000776C616E6D6F6465000000007373696499
:10CD900000000000576F7264436C6F636B204E6538
:10CDA00074776F726B0000003C423E436F6E6E659D
:10CDB0006374696E6720746F2041636365737320C9
:10CDC000506F696E742C2074727920616761696E8E
:10CDD000206C617465722E3C2F423E003C423E53F3
:10CDE000746174696E672061732041636365737356
:10CDF00020506F696E742C207472792061676169AC
:10CE00006E206C617465722E3C2F423E0000000063
:10CE10007361766574696D6573657276657200001D
:10CE20007361766574696D657A6F6E6500000000E8
:10CE30006E657474696D6500495020616464726543
:10CE40007373000045535038323636206669726D70
:10CE50007761726500000000574C414E00000000F1
:10CE60005353494400000000266E6273703B266EE7
:10CE70006273703B266E6273703B00004B657900F5
:10CE800054696D65207365727665720054696D65CD
:10CE9000207A6F6E652028474D54202B2900000012
:10CEA000476574206E65742074696D65000000002C
:10CEB0003C503E0D0A3C666F6E7420636F6C6F725F
:10CEC0003D7265643E3C423E000000003C2F423E05
:10CED0003C2F666F6E743E0D0A0000002F74656D66
:10CEE000706572617475726500000000736176652B
:10CEF00074636F7272727463000000007361766510
:10CF000074636F7272647331387878006469737017
:10CF10006C617974656D706572617475726500001D
:10CF20002E350000266465673B430000576F72642E
:10CF3000436C6F636B2054656D70657261747572BC
:10CF4000650000005254432074656D706572617411
:10CF500075726500445331387878000054656D70FF
:10CF600020636F7272656374696F6E205254432040
:10CF700028756E697473206F6620302E35B0432992
:10CF80000000000054656D7020636F7272656374F9
:10CF9000696F6E204453313878782028756E697433
:10CFA00073206F6620302E35B043290044697370BA
:10CFB0006C61792074656D7065726174757265005D
:10CFC0002F6C6472000000006C64726D696E00006A
:10CFD0006C64726D61780000736176656175746F61
:10CFE00000000000576F7264436C6F636B204C4409
:10CFF000520000004D696E004D6178004175746FFC
:10D000006D61746963206272696768746E657373B9
:10D0100000000000536574206173206D696E696DB6
:10D02000756D2076616C7565000000005365742095
:10D030006173206D6178696D756D2076616C7565C1
:10D04000000000002F646973706C617900000000BB
:10D0500073617665697469730000000073617665B9
:10D0600073796E63616D62690000000073617665BB
:10D070006272696768746E657373000073617665C8
:10D08000636F6C6F72730000726564006772656530
:10D090006E000000626C75650000000073617665CB
:10D0A000646973706C61796D6F6465007361766536
:10D0B00074696E74657276616C00000074657374D7
:10D0C000646973706C61790073617665616C6C0082
:10D0D000576F7264436C6F636B20446973706C614B
:10D0E0007900000045532049535400005065726D8B
:10D0F000616E656E7420646973706C6179206F660F
:10D100002022455320495354220000004469737083
:10D110006C6179204D6F64650000000055736520D7
:10D12000646973706C617920636F6C6F7273000057
:10D130004272696768746E6573732028312D3135CA
:10D14000290000003000000054656D702064697390
:10D15000706C617920696E74657276616C00000094
:10D160005465737420646973706C61790000000009
:10D170005361766520616C6C000000002F616E6960
:10D180006D6174696F6E730073617665616E696D50
:10D190006174696F6E00000073617665636F6C6F18
:10D1A00072616E696D6174696F6E0000646566001E
:10D1B00073617665616E0000737025640000000085
:10D1C00066617625640000007361766563616E00B8
:10D1D00063737025640000006364656600000000EE
:10D1E000576F7264436C6F636B20416E696D61743D
:10D1F000696F6E7300000000416E696D6174696F44
:10D200006E000000436F6C6F7220416E696D617437
:10D21000696F6E00616E256400000000646566251C
:10D22000640000003100000063616E2564000000AE
:10D2300063646566256400002F616D62696C6967CF
:10D240006874000073617665616D62696D6F646515
:10D250000000000073617665616D62696C656473DE
:10D260000000000073617665616D62696F666673C8
:10D27000657400007361766561616E00617370258D
:10D28000640000006164656600000000576F72640E
:10D29000436C6F636B20416D62696C6967687400F1
:10D2A000234C4544730000004F6666736574206F1D
:10D2B00066207365636F6E64203D203000000000BF
:10D2C000416D62696C69676874204D6F6465000028
:10D2D00061616E256400000061646566256400007C
:10D2E0002F74696D657273007361766569640000FF
:10D2F000610000006F000000662564007425640072
:10D30000576F7264436C6F636B2054696D65727301
:10D3100000000000696425640000000061256400CD
:10D320006F256400682564006D25640048545450DE
:10D330002F312E3020343034204E6F7420466F75DC
:10D340006E640000343034204E6F7420466F756E6A
:10D35000640D0A004E616D650000000056616C7539
:10D360006500000059595959000000004D4D00005A
:10D3700044440000686800006D6D000041637469FA
:10D380006F6E0000574C414E20436C69656E74000F
:10D39000415000004700000042000000363300000A
:10D3A000446563656C65726174696F6E00000000AE
:10D3B0004661766F7572697465000000536C6F7416
:10D3C0000000000041637469766500004F6E000044
:10D3D00046726F6D00000000546F0000486F757258
:10D3E00000000000010000000F0000001500000018
:10D3F000070000000B000000070000000B00000009
:10D40000070000000B0000000F00000014000000E7
:10D41000000000000F0000001400000000000000E9
:10D4200001000000000000000500000002000000F4
:10D430000B0000000C0000001A00000002000000B9
:10D440000B000000020000000B00000000000000C4
:10D45000100000001C000000280000003000000048
:10D4600001000000010000000000000002000000B8
:10D47000050000000C000000110000002200000068
:10D48000050000000C000000050000000C0000007A
:10D49000000000001000000010000000200000004C
:10D4A000200000000100000001000000000000005A
:10D4B00002000000050000000C0000001100000048
:10D4C00022000000050000000C0000000500000024
:10D4D0000C00000000000000000000000000000040
:10D4E000000000000000000001000000010000003A
:10D4F0000000000003000000050000000C00000018
:10D500000F0000001E000000050000000C000000DD
:10D51000040000000B0000000000000010000000EC
:10D52000150000002500000025000000010000009B
:10D530000100000000000000322E302E37000000F5
:10D540000D0A57656C636F6D6520746F20576F729D
:10D5500064436C6F636B204C6F67676572210000DA
:10D560002D2D2D2D2D2D2D2D2D2D2D2D2D2D2D2DEB
:10D570002D2D2D2D2D2D2D2D2D2D2D2D000000008F
:10D5800056657273696F6E3A2000000072746320F2
:10D590006973206F6E6C696E6500000072746320A1
:10D5A0006973206F66666C696E65000065657072F0
:10D5B0006F6D206973206F6E6C696E6500000000EE
:10D5C00063757272656E7420656570726F6D20761A
:10D5D000657273696F6E3A203078253038780D0A9D
:10D5E0000000000072656164696E672069722063E3
:10D5F0006F6465732066726F6D20656570726F6D04
:10D600000000000072656164696E67206469737070
:10D610006C617920636F6E66696775726174696F9A
:10D620006E2066726F6D20656570726F6D00000010
:10D6300072656164696E672074696D657365727681
:10D64000657220646174612066726F6D206565701B
:10D65000726F6D0072656164696E67206E696768DC
:10D66000742074696D6572732066726F6D206565D4
:10D6700070726F6D0000000072656164696E6720F2
:10D6800074656D7020636F6E666967757261746929
:10D690006F6E2066726F6D20656570726F6D000031
:10D6A000656570726F6D206973206F66666C696E58
:10D6B000650000007570646174696E6720454550AF
:10D6C000524F4D20746F2076657273696F6E2030F3
:10D6D00078253038780D0A0077726974696E672092
:10D6E00076657273696F6E20746F20454550524F96
:10D6F0004D206661696C6564000000007772697492
:10D70000696E6720495220636F64657320746F20CF
:10D71000454550524F4D206661696C6564000000BC
:10D7200077726974696E6720636F6E6669672074CB
:10D730006F20454550524F4D206661696C6564000D
:10D7400077726974696E672074696D657365727646
:10D750006572206461746120746F20454550524F9A
:10D760004D206661696C6564000000007772697421
:10D77000696E67206E696768742074696D652064DE
:10D7800061746120746F20454550524F4D20666191
:10D79000696C65640000000063616C6C696E6720F1
:10D7A0004952206C6561726E2066756E6374696F94
:10D7B0006E0000007573657220627574746F6E2060
:10D7C000707265737365643A20636F6E666967751E
:10D7D00072696E6720657370383236362061732047
:10D7E00061636365737320706F696E74000000007D
:10D7F000776F7264636C6F636B0000003132333497
:10D800003536373839300000636F6D6D616E643ABC
:10D810002073657420646973706C617920636F6C28
:10D820006F727320746F2025642025642025640D99
:10D830000A000000636F6D6D616E643A2073657459
:10D8400020616D62696C6967687420636F6C6F72C8
:10D850007320746F2025642025642025640D0A0040
:10D86000636F6D6D616E643A2073657420706F77BD
:10D870006572202573000000636F6D6D616E643A00
:10D880002073657420646973706C6179206D6F64B6
:10D890006520746F2025640D0A000000636F6D6DB4
:10D8A000616E643A2073657420616D62696C6967AA
:10D8B0006874206D6F646520746F2025640D0A0004
:10D8C000636F6D6D616E643A2073657420616E697B
:10D8D0006D6174696F6E206D6F646520746F2025B3
:10D8E000640D0A00636F6D6D616E643A2073657438
:10D8F00020636F6C6F7220616E696D6174696F6E09
:10D90000206D6F646520746F2025640D0A0000008F
:10D91000636F6D6D616E643A2073686F7720746514
:10D920006D7065726174757265000000636F6D6D76
:10D93000616E643A2073657420646973706C6179F8
:10D94000206272696768746E65737320746F202536
:10D95000642C2064697361626C65206175746D6FFD
:10D960006D61746963206272696768746E65737350
:10D9700020636F6E74726F6C20706572204C44521D
:10D980000D0A0000636F6D6D616E643A20736574FB
:10D9900020616D62696C696768742062726967688A
:10D9A000746E65737320746F2025640D0A00000087
:10D9B000636F6D6D616E643A20656E61626C6520A7
:10D9C0006175746F6D6174696320627269676874F0
:10D9D0006E65737320636F6E74726F6C000000006D
:10D9E000636F6D6D616E643A2064697361626C652A
:10D9F000206175746F6D6174696320627269676814
:10DA0000746E65737320636F6E74726F6C000000C8
:10DA1000636F6D6D616E643A207365742064697321
:10DA2000706C617920666C61677320746F20307848
:10DA30002530327800000000636F6D6D616E643ACE
:10DA400020737461727420646973706C61792074DE
:10DA500065737400636F6D6D616E643A20736574F5
:10DA60002074696D6520746F202573202534642D22
:10DA7000253032642D2530326420253032643A2539
:10DA80003032643A253032640D0A0000636F6D6DE8
:10DA9000616E643A207374617274206E65742074D0
:10DAA000696D65207265717565737400636F6D6D66
:10DAB000616E643A206C6561726E20495220636F1A
:10DAC00064657300636F6D6D616E643A2073617697
:10DAD0006520646973706C61792073657474696E14
:10DAE00067730000636F6D6D616E643A20707269D8
:10DAF0006E74207469636B65723A20272573270062
:10DB00006C64723A206F6C64206272696768746E2C
:10DB100065733A202564206E6577206272696768B4
:10DB2000746E6573733A2025640D0A00657370384E
:10DB3000323636206E6F772075700000657370384E
:10DB4000323636206E6F77206F6E6C696E6500001E
:10DB5000202049502025730064636637373A20251A
:10DB600073202534642D253032642D253032642015
:10DB7000253032643A253032643A253032640D0A59
:10DB80000000000072656164207274633A2025739E
:10DB9000202534642D253032642D25303264202533
:10DBA0003032643A253032643A253032640D0A004E
:10DBB000466F756E642054696D65723A2025732036
:10DBC000617420253032643A253032640D0A000039
:10DBD000676F742074656D7065726174757265200D
:10DBE00066726F6D20445331387878783A20256416
:10DBF00025730D0A00000000676F742074656D7056
:10DC0000657261747572652066726F6D205254433F
:10DC10003A20256425730D0A000000006E6F207401
:10DC2000656D706572617475726520617661696C8D
:10DC300061626C6500000000757064617465206449
:10DC40006973706C6179000049524D503A20504F11
:10DC5000574552206B65790049524D503A204F4B41
:10DC6000206B65790000000049524D503A206465F0
:10DC70006372656D656E7420646973706C61792080
:10DC80006D6F64650000000049524D503A20696E86
:10DC90006372656D656E7420646973706C61792060
:10DCA0006D6F64650000000049524D503A20646574
:10DCB0006372656D656E7420616E696D6174696F04
:10DCC0006E206D6F6465000049524D503A20696EB8
:10DCD0006372656D656E7420616E696D6174696FE4
:10DCE0006E206D6F6465000049524D503A206465A6
:10DCF0006372656D656E7420686F75720000000058
:10DD000049524D503A20696E6372656D656E74209C
:10DD1000686F75720000000049524D503A206465EA
:10DD20006372656D656E74206D696E757465000053
:10DD300049524D503A20696E6372656D656E74206C
:10DD40006D696E757465000049524D503A206465E6
:10DD50006372656D656E74207265642062726967B6
:10DD600068746E657373000049524D503A20696EB5
:10DD70006372656D656E7420726564206272696796
:10DD800068746E657373000049524D503A206465A3
:10DD90006372656D656E7420677265656E20627270
:10DDA000696768746E6573730000000049524D50D6
:10DDB0003A20696E6372656D656E74206772656581
:10DDC0006E206272696768746E657373000000008C
:10DDD00049524D503A2064656372656D656E7420DA
:10DDE000626C7565206272696768746E6573730032
:10DDF00049524D503A20696E6372656D656E7420AC
:10DE0000626C7565206272696768746E6573730011
:10DE100049524D503A2064656372656D656E742099
:10DE20006272696768746E657373000049524D5081
:10DE30003A20696E6372656D656E742062726967FF
:10DE400068746E657373000049524D503A206765DF
:10DE5000742074656D706572617475726500000080
:10DE6000706F7765725F696E697428292063616CD1
:10DE70006C656400737769746368696E6720706F9E
:10DE8000776572206F6E0000737769746368696EDE
:10DE90006720706F776572206F6666002020676567
:10DEA000742074656D706572617475726500000030
:10DEB0002020706F776572206F66662F6F6E00008E
:10DEC00020206F6B00000000202064656372656D88
:10DED000656E7420646973706C6179206D6F646520
:10DEE000000000002020696E6372656D656E74200D
:10DEF000646973706C6179206D6F64650000000067
:10DF0000202064656372656D656E7420616E696D55
:10DF10006174696F6E206D6F646500002020696E0A
:10DF20006372656D656E7420616E696D6174696F91
:10DF30006E206D6F64650000202064656372656DFE
:10DF4000656E7420686F7572000000002020696E95
:10DF50006372656D656E7420686F757200000000F5
:10DF6000202064656372656D656E74206D696E75E1
:10DF7000746500002020696E6372656D656E7420A3
:10DF80006D696E7574650000202064656372656D4F
:10DF9000656E7420726564206272696768746E656C
:10DFA000737300002020696E6372656D656E742066
:10DFB000726564206272696768746E6573730000CD
:10DFC000202064656372656D656E74206772656597
:10DFD0006E206272696768746E657373000000007A
:10DFE0002020696E6372656D656E74206772656569
:10DFF0006E206272696768746E657373000000005A
:10E00000202064656372656D656E7420626C756551
:10E01000206272696768746E657373002020696E90
:10E020006372656D656E7420626C756520627269DD
:10E030006768746E65737300202064656372656D34
:10E04000656E7420676C6F62616C206272696768CC
:10E05000746E6573730000002020696E6372656DD5
:10E06000656E7420676C6F62616C206272696768AC
:10E07000746E6573730000002020746F67676C65B1
:10E08000206175746F206272696768746E6573735E
:10E090000000000020205468616E6B20796F7521AC
:10E0A000000000003139322E35332E3130332E311D
:10E0B000303300004E65772074696D657A6F6E6548
:10E0C0003A2025640D0A00004300000008020020E9
:10E0D0001F0000001C0000001F0000001E000000C8
:10E0E0001F0000001E0000001F0000001F000000B5
:10E0F0001E0000001F0000001E0000001F000000A6
:10E100001F0000001D0000001F0000001E00000096
:10E110001F0000001E0000001F0000001F00000084
:10E120001E0000001F0000001E0000001F00000075
:10E130006D0100006E010000232D302B2000686C63
:10E140004C0065666745464700303132333435361A
:10E150003738394142434445460030313233343553
:10E1600036373839616263646566000020202020FC
:10E170002020202020282828282820202020202077
:10E180002020202020202020202020208810101057
:10E1900010101010101010101010101004040404AF
:10E1A0000404040404041010101010101041414124
:10E1B000414141010101010101010101010101018F
:10E1C0000101010101010110101010101042424222
:10E1D000424242020202020202020202020202025F
:10E1E00002020202020202101010102000000000C1
:10E1F000000000000000000000000000000000001F
:10E20000000000000000000000000000000000000E
:10E2100000000000000000000000000000000000FE
:10E2200000000000000000000000000000000000EE
:10E2300000000000000000000000000000000000DE
:10E2400000000000000000000000000000000000CE
:10E2500000000000000000000000000000000000BE
:10E2600000000000000000000000000000000000AE
:08E27000D01EFF7F0100000039
:10E27800E0BC0008C8BC0008E4BC0008E8BC000812
:10E28800ECBC0008D8BC0008DCBC0008FF0000009B
:10E29800FF000000E80300000100000084C200083D
:10E2A800000000000000000000000000B8CC0008DA
:10E2B8000000000000000000000000008CC2000800
:10E2C80000000000000000000000000028C2000854
:10E2D8000400000004000000010000000500000028
:10E2E80020000000200000000300000020C20008F9
:10E2F800891000080400000004000000000000006D
:10E3080030C20008FD1000080800000008000000E6
:10E318000300000038C20008C11B00080400000008
:10E32800040000000300000040C200086D19000846
:10E3380004000000040000000300000048C20008B8
:10E34800CD0D0008040000000400000000000000DB
:10E3580050C20008611E000804000000040000000C
:10E368000300000058C20008C11800080800000097
:10E37800080000000300000064C20008FD16000841
:10E388000400000004000000030000006CC2000844
:10E39800C921000806000000060000000300000074
:10E3A80074C200081D1500080400000004000000E5
:10E3B800030000007CC20008A51300080800000044
:10E3C80008000000030000000F000000200000000B
:10E3D8000100000020000000050000003C000000D3
:10E3E80020C2000801000000010000000000000039
:10E3F80028C200080400000004000000010000001A
:10E408000F00000001000000160000003CC40008D6
:10E4180044C400084CC4000858C40008FFFF0000AA
:10E42800FFFF0000D80E0000FF000000FFFFFFFF05
:10E43800FF000000FF000000010000003139322E0B
:10E4480035332E3130332E313033000000000000D8
:10E45800020406080000000001020304010203048C
:10E46800060708090000000000000000010203047C
:10E478000607080900A24A04000000000000000086
:10E488000000000000000000000000000000000084
:10E498000000000000000000C8E0000800000000C4
:10E4A8000000000000000000000000000000000064
:10E4B8000000000000000000000000000000000054
:10E4C8000000000000000000000000000000000044
:10E4D8000000000000000000080200206BE10008B6
:10E4E80001000000000000004A00000000000000D9
:10E4F8000000000000000000000000000000000014
:10E50800000000004A0000000000000000000000B9
:10E5180000000000000000000000000000000000F3
:08E5280011010008ED000008DC
:0400000508000000EF
:00000001FF
